:1000000000400020512000008D2000008F200000C3
:1000100000000000000000000000000000000000E0
:10002000000000000000000000000000912000001F
:100030000000000000000000932000009520000058
:10004000972000005D6D0000452300009720000010
:1000500097200000000000005118000097200000C9
:1000600097200000B9240000997700009720000035
:1000700097200000972000009720000097200000A4
:100080009720000097200000972000009720000094
:100090009720000097200000972000009720000084
:1000A00097200000972000000000000000000000E2
:1000B0000000000000000000000000000000000040
:1000C00010B5064C2378002B07D1054B002B02D02E
:1000D000044800E000BF0123237010BD000200208F
:1000E000000000007C06030008B5084B002B03D07D
:1000F0000748084900E000BF07480368002B00D10B
:1001000008BD064B002BFBD09847F9E70000000024
:100110007C06030004020020000200200000000012
:10012000164B002B00D1144B9D46402292029A1A86
:10013000924600218B460F461348144A121A24F0A7
:1001400042FA0F4B002B00D098470E4B002B00D0EB
:1001500098470020002104000D000D48002802D01F
:100160000C4800E000BF24F057F82000290001F0FF
:10017000D7FD01F066FFC0460000080000400020E7
:1001800000000000000000000002002030200020DD
:10019000000000000000000038B5064B1D1C0C3BA1
:1001A0001C1C3035281C0C3D01F078FBA542F9D110
:1001B00038BDC046340200209621F0B51D4F97B0DF
:1001C000381C890101F030FA07A81B4901F0ACFB8B
:1001D0000DAC0AA8194901F0A7FB10AD201C184965
:1001E00001F0A2FB13AE281C164901F09DFB301C48
:1001F000154901F099FB154B391C0293144B07AAC2
:10020000049300940AAB01950396124800F010FF86
:10021000301C01F043FB281C01F040FB201C01F0C6
:100220003DFB0AA801F03AFB07A801F037FB17B025
:10023000F0BDC04670020020A4B70200B1B70200B2
:10024000C2B70200CCB70200D7B7020034020020C8
:100250005B0700001C0200201FB5082004F0E2FB31
:1002600001280ED1084901A801F05EFB07480021D2
:1002700001AA00F057FC01A801F010FB044801F0AE
:1002800011FD05B000BDC046EAB702001C02002007
:100290001027000070B51F4C201C08F02BF91E4DD4
:1002A000201C2A1C1D4908F0F9F81D4C1D49201C72
:1002B00001F03AFB201C1C4E0C30311C01F034FBC9
:1002C000201C311C183001F02FFB201C311C243065
:1002D00001F02AFB201C311C303001F025FB2A1CC8
:1002E0001249002008F0DAF8114C201C00F04EFBF7
:1002F0002A1C201C0F4908F0D1F80F4C0023201CA9
:100300000121022201F074F82A1C201C0B4908F07C
:10031000C5F870BD30020020000000200D860000EE
:1003200034020020F2B7020086BC020099010000EE
:100330001C020020B50900007002002071150000A9
:100340001FB5084901A801F030FB074B01A81B6944
:1003500098470022054B01A81A7101F09FFA05B0D9
:1003600000BDC046D0020020B4020020C802002018
:100370001FB5084901A801F018FB074B01A8DB686D
:1003800098470022054B01A8DA7001F087FA05B002
:1003900000BDC046D0020020B4020020C8020020E8
:1003A0001FB5084901A801F000FB074B01A89B6895
:1003B00098470022054B01A89A7001F06FFA05B02A
:1003C00000BDC046D0020020B4020020C8020020B8
:1003D0001FB5084901A801F0E8FA074B01A85B68BE
:1003E00098470022054B01A85A7001F057FA05B052
:1003F00000BDC046D0020020B4020020C802002088
:100400001FB5084901A801F0D0FA074B01A81B68E5
:1004100098470022054B01A81A7001F03FFA05B079
:1004200000BDC046D0020020B4020020C802002057
:1004300030B58DB0011C8468684601F0B6FAD24927
:1004400009A801F071FA002209A9684601F072FBBF
:10045000051C09A801F022FA02226B1C28D1CB4905
:1004600009A801F061FA684609A9002201F062FBBF
:10047000051C09A801F012FA6B1C09D00222C44B1A
:1004800052421A60231C09A80B3B69460B3204E157
:10049000C04909A801F048FA684609A9002201F0FC
:1004A00049FB051C09A801F0F9F96B1C07D00322D0
:1004B000B74B1A60B849B94801F089FA5FE1B84909
:1004C00009A801F031FA002209A9684601F032FBBF
:1004D000051C09A801F0E2F904226B1C00D0F4E02D
:1004E000B04909A801F020FA002209A9684601F0E4
:1004F00021FB051C09A801F0D1F905226B1CD7D1FD
:10050000A94909A801F010FA684609A9002201F0DA
:1005100011FB051C09A801F0C1F96B1C06D00523CD
:100520009B4A5B421360A14A1370C3E7A04909A824
:1005300001F0FAF9002209A9684601F0FBFA051C4E
:1005400009A801F0ABF906226B1CB1D1994909A8A1
:1005500001F0EAF9684609A901F0FCFA051C09A8AE
:1005600001F09CF96B1C5AD0631E072203A8694650
:1005700001F0F6FA904909A801F0D6F909A903A8F3
:1005800001F0E8FA041C09A801F088F9231C06A868
:1005900003A9002201F0E4FA059B621C013B09A8B3
:1005A00003A901F0DDFA09A97C4801F008FA09A8BD
:1005B00001F074F90024814B814A18685B681B1AAA
:1005C0009B1053439C4228D20C216143411806A83A
:1005D00001F08CFA00281ED07A4BA200D358002BD1
:1005E00019D0794BE25C002A15D10132E254042C77
:1005F00011D8201C75491FF065FF030507090B0082
:10060000734806E0734804E0734802E0734800E072
:10061000734802F07FF90134CDE70A22A7E071495F
:1006200009A801F081F9002209A9684601F082FABF
:10063000051C09A801F032F904226B1C00D037E731
:10064000694909A801F070F9684609A9002201F07A
:1006500071FA051C09A801F021F96B1C07D00722CB
:100660004B4B09A81A606946A31E023A15E05F4980
:1006700009A801F059F9684609A9002201F05AFABF
:10068000051C09A801F00AF96B1C0ED00822694666
:100690003F4B09A81A60A31E033A01F061FA3F48D4
:1006A00009A901F08CF909A867E0514909A801F0EE
:1006B0003BF9684609A9002201F03CFA051C09A88B
:1006C00001F0ECF86B1C02D003225242F0E64949DB
:1006D00009A801F029F9684609A9002201F02AFABF
:1006E000051C09A801F0DAF86B1C48D0631E032230
:1006F00003A8694601F034FA2F4909A801F014F95A
:1007000009A903A801F026FA041C09A801F0C6F8FB
:1007100006A803A90022231C01F022FA06A83649E4
:1007200001F0F2F900280ED0059B621C013B09A8DC
:1007300003A901F015FA09A9184801F040F909A820
:1007400001F0ACF812E006A82C4901F0DDF9002810
:1007500002D012482A4907E006A82A4901F0D4F934
:10076000002803D00D48284901F031F90922084B2F
:1007700006A81A6001F092F803A801F08FF8684605
:1007800001F08CF80DB030BDFCB7020006B80200D5
:100790000800002010B8020086BC0200D002002031
:1007A0001AB8020026B8020030B80200FC0200208D
:1007B0003AB8020044B8020004B80200F002002077
:1007C000ABAAAAAAB4020020C8020020C92B0000CC
:1007D00001040000D1030000A10300007103000028
:1007E0004103000000B802000AB802004CB8020041
:1007F00052B80200ADB9020058B802005CB802005D
:100800005FB802005DB8020078B802007FB501262B
:10081000354D2B6833420AD1344C3549201C01F048
:1008200083F8201C3349344A2E6007F037FE334CDE
:1008300023681D79002D34D023681868002851D012
:1008400003689B68984700284CDD23681868036894
:100850009B689847002820D0236818680368DB68E5
:100860009847061E15DB214DC1B2281C01F0DAF8AD
:100870000D2E0ED1291C01A801F097F801A8FFF751
:10088000D7FD01A801F00AF8281C194901F09FF8CA
:1008900003E0012001F006FAD7E7012001F002FA97
:1008A000CAE7174C201C03F085FB211C021C2B1CE3
:1008B000684603F043FD009B0C4C191D201C01F001
:1008C00086F8211C01A801F070F801A8FFF7B0FD1F
:1008D00001A800F0E3FF201C054901F078F8684604
:1008E00003F052FD7FBDC04604030020DC0200205F
:1008F00086BC02009D18000000000020E8020020D5
:100900002805002008B5FFF781FF012002F0DAF882
:10091000F9E770B5041C05684668B54204D0281C88
:1009200000F0BCFF0C35F8E72068002801D007F084
:10093000BCFD201C70BD0000F8B50122041C0E4D4A
:100940000E4B291C0E481A6001F041F8201C291C8E
:10095000083001F03CF80B4B1D681F1C2C1C5E6816
:10096000B44204D0201C00F099FF0C34F8E70022B8
:10097000054B7D601A70F8BD86BC0200080000209F
:10098000D0020020F0020020FC020020002310B55D
:10099000041C036003710549083000F0C5FF044BD7
:1009A000201C1C60FFF7C8FF201C10BD86BC020085
:1009B000E802002010B5041CFFF7BEFF201C083021
:1009C00000F06CFF201C10BD08B5044B1B68002B09
:1009D00002D0081C111C984708BDC0460003002027
:1009E00030B585B000201B4C2056053003282CD88C
:1009F000194B1D681FF066FD1A120A02174901A85B
:100A000000F092FF281C01A9022216E0144901A857
:100A100000F08AFF281C01A903220EE0114901A859
:100A200000F082FF281C01A9042206E00E4901A85B
:100A300000F07AFF281C052201A95242FFF7C4FFEB
:100A400001A800F02BFF00232370052001F02AF9F4
:100A5000C8E7C046FC020020E80200208DB8020072
:100A6000B9B80200FEB8020031B9020070B58AB010
:100A7000041C0E1C07A8111C151C00F096FF23492E
:100A800007A800F0F8FF011C01A800F08EFF07A8DE
:100A900000F004FF1E4904A800F046FF291C04A82A
:100AA00000F0DBFF1B4900F0E6FF1B4900F0E3FF0D
:100AB000311C00F0D2FF194900F0DDFF011C07A82E
:100AC00000F073FF07A90022201CFFF77DFF07A895
:100AD00000F0E4FE04A800F0E1FE2379002B04D02E
:100AE000206801A900F00AFE0BE0019907A803F0B5
:100AF00067FC0B4807A9022203F080FB07A803F05C
:100B000043FC01A800F0CAFE0AB070BD57B902004C
:100B100059B902005FB9020063B90200C4040300BE
:100B200028050020F0B52E4E8BB0346873681B1B6F
:100B30002C4C9B10634399424FD22B4B1B78032BB9
:100B40004BD10F1C041C294904A8151C00F0ECFE15
:100B5000274901A800F0E8FE0C217943336801A879
:100B6000591800F07AFF234E311C00F084FF291C35
:100B700000F073FF311C00F07EFF011C07A800F09D
:100B800014FF04A907AA201CFFF770FF07A800F0B4
:100B900085FE01A800F082FE04A800F07FFE164C3E
:100BA0002368251C052B09D0012001F07BF8236860
:100BB0005A1DF4D1114A1370FFF712FF01F06AF8C1
:100BC000041C2B680A2B08D0012001F06BF801F0FF
:100BD00061F80B4B001B9842F3D90BB0F0BDC04637
:100BE000F0020020ABAAAAAA04000020A1B90200CA
:100BF000A9B9020004B8020008000020FC0200208D
:100C0000B80B000030B5051C87B0294B1A681C1CB6
:100C1000042A16D06846274900F086FE03A8264914
:100C200000F082FE694603AA281CFFF71FFF03A8F5
:100C300000F034FE684600F031FE642001F032F826
:100C4000E3E72368072B16D068461C4900F06CFECA
:100C500003A81B4900F068FE694603AA281CFFF799
:100C600005FF03A800F01AFE684600F017FE642096
:100C700001F018F8E5E70422124B684612491A7091
:100C800000F052FE6846114900F0E7FE011C03A87F
:100C900000F08BFE03A90022281CFFF795FE03A895
:100CA00000F0FCFD684600F0F9FD002007B030BD03
:100CB00008000020B4B9020000B80200B9B902006F
:100CC0000AB8020004000020C5B90200D0020020CA
:100CD000F0B5284D8BB02C780023042C46D10F1C86
:100CE000161C041C244901A800F01EFE234907A875
:100CF00000F01AFE391C07A800F0AFFE204900F0F2
:100D0000BAFE311C00F0A9FE1E4900F0B4FE011C21
:100D100004A800F04AFE01A904AA201CFFF7A6FEC1
:100D200004A800F0BBFD07A800F0B8FD01A800F082
:100D3000B5FD154E3368082B0AD0012000F0B2FF34
:100D40003368DA1CF5D1114A13700133FF330DE01B
:100D50000F4907A82B7000F0E7FD201C07A900220F
:100D6000FFF732FE07A800F099FD002358B20BB040
:100D7000F0BDC04604000020EFB9020014B8020024
:100D800092B9020004B8020008000020FC02002012
:100D9000FCB90200F0B52B4E8BB033780024051C53
:100DA000022B4BD1284F3A687B689B1A274A9B102D
:100DB00053439C4233D2264901A800F0B5FD254992
:100DC00007A800F0B1FD0C2161433B6807A8591842
:100DD00000F043FE204900F04EFE011C04A800F084
:100DE000E4FD01A904AA281CFFF740FE04A800F0B6
:100DF00055FD07A800F052FD01A800F04FFD174F68
:100E00003B68032B09D0012000F04CFF3B681A1D02
:100E1000F5D1134AFC24137010E00134C2E7032318
:100E2000104907A8337000F07FFD281C07A9002295
:100E3000FFF7CAFD07A800F031FD002460B20BB037
:100E4000F0BDC04604000020F0020020ABAAAAAA10
:100E500017BA020020BA020004B8020008000020FD
:100E6000FC02002028BA0200F7B5436802680E1C95
:100E70009A1A254B92105A43041C24490123002A34
:100E800003D053000D1C934202D38B4238D91F4D1F
:100E90000C20684307F00DFB071C63682268981A52
:100EA0003818002802D0311C00F07FFD381C636820
:100EB00026680193031C0C330093019B9E4207D0CC
:100EC000002802D0311C00F070FD0C360098F1E7CC
:100ED000636826680193019B9E4204D0301C00F099
:100EE000DDFC0C36F7E72068002801D007F0DDFABA
:100EF000009B276063600C235D437D19A560F7BDEF
:100F00001D1C1F1EC9D0C3E7ABAAAAAA555555156B
:100F1000F0B53E4C8FB0267802940025082E72D191
:100F20000F1C061C1C1C3C3303920193201C3849E7
:100F300000F0EAFD002811D1364D6868AB68984290
:100F400008D0002802D0211C00F02FFD6B680C3364
:100F50006B6003E0281C211CFFF786FF019B0C340B
:100F60009C42E3D12C4905A800F0DEFC2B490BA8DC
:100F700000F0DAFC14990BA800F06FFD284C211C3E
:100F800000F079FD159900F089FD211C00F073FD3A
:100F9000391C00F062FD211C00F06DFD039900F08A
:100FA0005CFD211C00F067FD011C08A800F0FDFCA1
:100FB00005A908AA301CFFF759FD08A800F06EFC2F
:100FC0000BA800F06BFC05A800F068FC154C23682A
:100FD000022B09D0012000F065FE23689A1CF5D190
:100FE000114AFE2513700EE0029A10490BA81370E7
:100FF00000F09AFC301C0BA90022FFF7E5FC0BA8BF
:1010000000F04CFC002568B20FB0F0BD04000020D9
:1010100086BC0200F00200204DBA02005ABA02005B
:1010200004B8020008000020FC02002062BA02009E
:10103000F0B50125041C0F1C161C85B00571039327
:10104000FFF77AFC104B11491D701148276001F021
:1010500061FC201CFFF7D6FD201C311C039AFFF712
:1010600037FE00280ED10D9B201C00930E9B0A9981
:1010700001930B9A0C9BFFF74BFF002802D1201C19
:10108000FFF788FE05B0F0BD04000020C92B00006A
:101090000509000038B50F4D281C07F02BFA0E4C3F
:1010A000281C221C0D4907F0F9F90D4D0D49281C8B
:1010B00000F03AFC281C221C0B4907F0EFF9002332
:1010C0000A480B49036043608360221C07F0E6F97D
:1010D00038BDC046EC020020000000200D86000054
:1010E000D002002086BC02009D180000F002002003
:1010F000130900000A4B1B6898420DD1094A0A4B9C
:1011000011781B78994207D013780849C85C137886
:101110000133DBB2137001E0012040427047C0464A
:10112000080300200C0300200D0500200D03002003
:10113000F7B5021C72B6C38F0120002B02D150609C
:10114000181C6EE0141C403424786408044001D05C
:10115000C943C9B2C220556B324E800035500120C0
:10116000A0250196177CED05B840002C02D0A127E0
:10117000FF0000E02C4FE851181C0138C046C04663
:10118000C046C046C046C046C046C046C046C0462F
:10119000C046C046F1D10825177C0120BC46A027D7
:1011A0006646FF05014203D0B040A126F60001E0EB
:1011B000B0401D4EB851181C0138C046C046C0464C
:1011C000C046C046C046C046C046C046C046C046EF
:1011D000C046F1D1013DEDB24908002DDCD101211D
:1011E000A020157CC005A940002C01D00E4C01E0C8
:1011F000A124E4000151516BC12201989200815059
:10120000181C0138C046C046C046C046C046C0464D
:10121000C046C046C046C046C046C046F1D162B6D0
:101220000120FEBD006000400C050000084B1B685B
:10123000984209D1074B084A19781278914203D095
:101240001B78064AD05C01E0012040427047C0464E
:10125000080300200C0300200D0500200D030020D2
:10126000464BF7B51C68002C00D186E0271C4037A0
:101270003B78201C9B0704D500F08AF9431E984157
:1012800003E000F085F943425841C0B2002800D184
:1012900073E0C2223A4B616B92009950208F019308
:1012A00000280DD00138C046C046C046C046C046E2
:1012B000C046C046C046C046C046C046C046F1D142
:1012C00008260025608F00280DD00138C046C04692
:1012D000C046C046C046C046C046C046C046C046DE
:1012E000C046C046F1D1C046C046C046C046C04612
:1012F000C046C046C046C046C046C046C046C046BE
:10130000C046C046C046201C6D0800F041F90028C8
:1013100003D080235B421D43EDB2013EF6B2002EA6
:10132000D0D13B789B0701D5ED43EDB2154A164964
:10133000137809780133DBB28B4204D0117813485B
:101340001370455403E001223B7813433B70A08F98
:1013500000280DD00138C046C046C046C046C04631
:10136000C046C046C046C046C046C046C046F1D191
:10137000C123626B01999B00CA50F7BD080300208E
:10138000006000400D0500200C0300200D0300202C
:10139000064B021C1B6800209A4206D1044B054AEA
:1013A0001B781078181AC005C00D7047080300207C
:1013B0000D0500200C030020094B1B6898420DD13D
:1013C000C222416B074B92009950002206490A70D5
:1013D00006490A70C122416B920099507047C0467D
:1013E00008030020006000400D0500200C030020D1
:1013F000F0B585B00393FA23071C00259B00041C5D
:101400008360154B154E0833143701914560036016
:10141000311C381C029200F087FA0120221C03992B
:10142000403201408140137825878343001883436D
:101430000B436587A587E587381C1370311C00F0C6
:10144000C6FA6A461279A31CDA776A46201C127A19
:10145000631CDA7705B0F0BDD8BA0200B2B9020059
:10146000002330B50B495A008C1865780C1C002DF0
:1014700008D1515C814205D00133042BF2D1012007
:10148000404206E00025A118A054034A9B0098584A
:101490004D7030BD1C0000200C00002038B5064DFA
:1014A00000242B68834205D10233D87F00F0A4F9D1
:1014B0002C600134201C38BD08030020002370B5C7
:1014C000828F9A4231D01A4E326882422DD0041C4B
:1014D0009A4202D0101CFFF7E1FF221C0125403286
:1014E00013781449AB43137000220A701249346018
:1014F0000A70A61CF07F9B070CD5FFF7B1FF606355
:10150000431C01D1012310E0F07F0C49042200F0BC
:10151000FDF8F7E7FFF7A4FF6063431CF2D0F07F0C
:101520000649032200F0F2F82B1C181C70BDC046BF
:10153000080300200D0500200C03002061120000AC
:1015400010B5041CFFF7AAFF00230234E07F074A0E
:1015500059008C5C844205D1012053185870FF2338
:101560008B5402E00133042BF1D110BD1C0000208C
:1015700010B5041C054B08330360FFF7E1FF201C86
:10158000143000F08BF9201C10BDC046D8BA020000
:1015900008B50230C07F03F085FA08BD70B501269A
:1015A000031C0C1C311C40331B78051C5B08994341
:1015B000201C03F01DFA201C311C03F055FA064BC9
:1015C000A200D3589E402B74E301E402E41A034BBB
:1015D000EE62E4182C6370BD80BA0200080500506A
:1015E00038B5051C0C1C081C002103F03DFA2B1C0F
:1015F00040331B789B0703D4201C012103F0F8F92A
:10160000AB1CDC77064BA200D258012393406B62DF
:10161000E301E402E41A034B6A74E418AC6238BDD7
:1016200080BA020010050050F8B5051C1435041CE2
:101630000F1C281C244900F067FA244E00280ED104
:10164000311C281C00F060FA631CD97F002803D0ED
:10165000201CFFF7A3FF07E0201CFFF79FFFA31C40
:10166000D97F201CFFF7BCFF381C20F02DF8011C8F
:10167000FE2080051FF066FB15491FF055FD1FF089
:1016800079F9420883B2023A22875A1EE3876287B9
:10169000A387181E0DD00138C046C046C046C046BC
:1016A000C046C046C046C046C046C046C046C0460A
:1016B000F1D1281C311C00F027FA002802D1201C8F
:1016C000FFF7FCFEF8BDC04653DF02007DBA020002
:1016D00000247449F7B5061C0D1C0C1C8B180193D3
:1016E000019B671B9C4207D0336821781B68301C24
:1016F000984701340028F3D1381CFEBD0B1C10B5EF
:101700000268096854689A68A04710BDF8B5314F5F
:101710000D1C3968041C161C002921D110222E48EA
:1017200022F051FF7F2240212C4B1A705A708032D8
:101730009A70DA702A4B2B4AD967C0235B00D150CC
:101740008533FF33D3589C466046274B03408020A7
:10175000C0030343C12080001350012311603B608C
:10176000142C36D8214BA400E458032E05D0042EA7
:1017700005D0022E2DD1032002E0022000E001203E
:101780000022164B99564E1C1ED113499C549300AF
:101790005D501749174D5B18A221C9005E582402FD
:1017A00035405D50F8256D015E582C400004204303
:1017B0003043585001205C5804435C50C123904092
:1017C0000B499B00C85004E0A142DED00132042A3C
:1017D000D7D1F8BD100500201405002024000020FA
:1017E00004E100E000E100E0FFFF00FFF8BA0200C2
:1017F00000600040FFE0FCFF10B514281FD8104B1C
:101800008000C15800230F4A9856884214D1FF2106
:101810000020D1540C499A00A22450500B49E400F6
:10182000521801211059884399401051C2220B1CB3
:10183000064992008B5002E00133042BE3D110BD26
:10184000F8BA0200240000201405002000600040C7
:1018500038B500240D4BA200D5182B68012B11D1EF
:10186000C121A3400A488900415819420AD0094BB6
:10187000E356013304D0084BD358002B00D09847CF
:1018800000232B600134042CE4D138BD00610040FA
:1018900000600040240000201405002010B5041C46
:1018A000006801F0ABFA201C10BD10B5041C0068E4
:1018B000002801D001F0A2FA00232360A360636036
:1018C00010BD38B5041C0D1C0068013101F0BEFAD2
:1018D000031E01D0012028C438BD036810B5002BB9
:1018E00002D043688B4209D2041CFFF7EAFF0028AC
:1018F00005D0A368002B01D122681370012010BD10
:1019000070B50E1C111C041C151CFFF7E6FF002807
:1019100003D1201CFFF7C9FF04E0A5602068311C3B
:1019200023F0BAFC201C70BD38B50023041C0D1E2A
:101930000360436083609D4207D0081C24F03AF99D
:10194000291C021C201CFFF7DBFF201C38BD38B50A
:10195000051C00680C1C00280CD06B688A68934238
:1019600006D3096823F098FCA368AB6000230AE063
:1019700001F044FA23682B6063686B60A368AB6076
:10198000002323606360A36038BD10B50B1C041EE8
:101990008C4208D00968002903D09A68FFF7B0FF8D
:1019A00001E0FFF782FF201C10BD002310B5041CCE
:1019B000036043608360FFF7E8FF201C10BD10B593
:1019C000041E8C4201D0FFF7C2FF201C10BD38B5A9
:1019D000041C0D1E08D0081C24F0ECF8291C021C65
:1019E000201CFFF78DFF01E0FFF75FFF201C38BDD3
:1019F000F8B58568002901D1002711E00127002AE8
:101A00000ED055190E1C291C041CFFF766FF002878
:101A1000F2D02368A268311C981823F03DFCA56021
:101A2000381CF8BD07B5002201AB19705A70191C9B
:101A30000132FFF7DDFF0EBD1FB5041C0A22081C92
:101A4000694600F033F9684624F0B4F86946021C90
:101A5000201CFFF7CDFF04B010BD0B1C10B50968AA
:101A60009A68041CFFF7C4FF002802D1201CFFF76E
:101A70001CFF201C10BD38B5041C0D1E09D0081C0D
:101A800024F098F8291C021C201CFFF7B1FF002845
:101A900002D1201CFFF709FF201C38BD10B5041C23
:101AA000FFF7CAFF002802D1201CFFF7FEFE201C12
:101AB00010BD08B503680A1C0968002B02D0002974
:101AC0000ED107E000290FD09368002B0CD00978C5
:101AD00048420AE08268081C002A06D0187804E010
:101AE000181C23F0CBFB00E0002008BD826808B57D
:101AF00094468A680023944504D1FFF7DAFF4342F5
:101B00004341DBB2181C08BD08B58368002B04D123
:101B1000012000290DD00B7808E0002902D10368CC
:101B20001B7803E0006823F0A9FB031C58425841CE
:101B3000C0B208BD836810B59A4208D2046809682B
:101B4000A01824F052F8002801D0001B01E0012069
:101B5000404210BD08B50022FFF7ECFF08BD0000B1
:101B6000F7B5071C0E1C151C1C1C9A4201D9251C1C
:101B7000141C381C0C49FFF7D7FEB3689D4211D2E4
:101B80009C4200D91C1C3368381C1B191A7801921E
:101B900000221A7033685919FFF719FF6A46336833
:101BA00012791A55381CFEBD86BC0200704770477A
:101BB000704770477047704710B5041C06F075FCFD
:101BC000201C10BD10B5041C06F06FFC201C10BDBD
:101BD00010B5041C06F069FC201C10BD10B5041CD7
:101BE00006F063FC201C10BD10B5041C034B036001
:101BF000403002F0C9FB201C10BDC04658BB02009B
:101C000010B5041CFFF7F0FF201C06F04EFC201C52
:101C100010BD0000C31F0020122B02D8014A9B00F8
:101C20009858704760BB020008B5024803F0FCF802
:101C300008BDC0462405002010B5054C201C03F04B
:101C40003FF8201C0349044A06F028FC10BDC0469A
:101C5000240500205D1C00000000002010B5041CBD
:101C60009130FF3001F0C6FA201C6930FF3001F0DE
:101C7000C1FA201CF03001F0A1FB201CD03001F093
:101C800037FF201C643000F05DF8201DFFF7ACFF2B
:101C9000201C10BD08B500F07DFCFA2189001EF063
:101CA00025FC08BD08B500F00DFF08BDF0B58DB0EE
:101CB000071C0E1C0192081E29D0131C023B002099
:101CC00003AC222B23D8002F12D0381C01991EF010
:101CD00093FC381C0D1C01991EF008FC631C071CAA
:101CE000092D01D8303500E0573525701C1CEAE776
:101CF00003AB9C42E9D0331C03AA944204D9013CB3
:101D000022781A700133F7E70022301C1A700DB0E8
:101D1000F0BD08B5FEF7A0FA142000F0D3FEF9E7F5
:101D200008B5FFF781FFFEF747FA0448044900F0C1
:101D3000F1FDFA20800000F0C5FEFAE7131D000057
:101D4000C92B000010B5041C034B083303601C3082
:101D500000F04FFA201C10BDB0BB020010B5041CEF
:101D6000FFF7F0FF201C06F0A0FB201C10BD0000B8
:101D70000023C35610B5041C013304D1054806499D
:101D80002C2200F055F8636960681B681840431EF8
:101D9000984110BDC0BB0200D8BB020070B5051C45
:101DA000041C0E4B0E1C083308C5281C00211822E9
:101DB00022F009FC0023201C311CE36123626363D1
:101DC000A363E364064A231C1C3000F011FA281CAC
:101DD000311C00F068F8201C70BDC046B0BB02008A
:101DE000191E000008B50430FFF7C2FF08BD08B592
:101DF000043000F0D9F908BD08B54369011C002B77
:101E000004D10368002B06D0984704E0006800283E
:101E100001D00431984708BD08B5012903D0022933
:101E200004D1383000E02030FFF7E6FF08BD0000A5
:101E300038B5051C0C1C131C291C0248221C00F080
:101E400003F838BD56BC02000FB4012008B500F0FD
:101E5000F8F8000038B50023C356041C0D1C0133EC
:101E600004D1064806492422FFF7E2FF6368002DEB
:101E700001D0E26800E02269136038BDC0BB0200F7
:101E8000D8BB020070B50D1C041C161C00F074F9C0
:101E90006B1C07D0201C002100F08CF9201C311C89
:101EA00000F082F970BD08B50322FFF7EBFF08BD13
:101EB00008B5FFF7E7FF08BD70B50D1C041C161C24
:101EC00000F05AF96B1C0BD0201C311CFFF7C2FF2D
:101ED000201C012100F06EF9201C002100F064F9A3
:101EE00070BD08B50022FFF7E7FF08BD08B5054B38
:101EF0001B68002B04D104481821192200F0B6F900
:101F000008BDC046A40900202420002008B5031CF9
:101F10000020022B0DDD0749033B9B005A58585007
:101F2000824204D01368101C5B68984701E00120CE
:101F3000404208BDA408002070B50C1C151C0228E6
:101F400010DC0F4B1B68002B01D1FFF7CFFF661988
:101F5000B44205D021780B4800F078FA0134F7E755
:101F6000281C0BE00338084B8000C058002803D021
:101F700003681B68984701E00120404270BDC046DD
:101F8000A409002024200020A408002010B50C1C67
:101F900002280BDC0C4B1B68002B01D1FFF7A6FFBE
:101FA0000A4800F045FA207001200BE00338084B86
:101FB0008000C058002803D003689B68984701E060
:101FC0000120404210BDC046A4090020242000206A
:101FD000A408002008B5031C0120022B0BDD033BE5
:101FE000054A9B009858002803D00368DB6898478F
:101FF00001E00120404208BDA408002008B5031CF0
:102000000020022B0BDD033B05489B0018580028DD
:1020100003D003681B69984701E00120404208BDD6
:10202000A408002008B5022804D880239B014B6037
:10203000002005E021F0C2FC09230360012040429A
:1020400008BD08B5002801D003F06EF8FEE70000D7
:102050000848026803210A4302600749074A084BFF
:102060009B1A03DD043BC858D050FBDC0548804771
:102070000548004724050040B0060300000000208A
:10208000000200209920000021010000FEE7FEE789
:10209000FEE7FEE7FEE7FEE72D4B10B51A78012AB2
:1020A00019D12C4A1268120715D12B4AE024116865
:1020B000F022081C104021420BD128490968114226
:1020C00009D12749274A11608021274A0902116056
:1020D00001E03028F1D01A78012A0DD11D49096894
:1020E000090709D1F0201C4909680140402903D1A2
:1020F0001A490968014223D01B68DBB2012B25D1A4
:10210000144B1B681B0721D1134B1A68F0231A408C
:10211000A02A04D1114A12681A4203D016E0D02A2C
:1021200014D1F7E7114B1A68012A03D1C022104BD2
:102130001A600BE00F4A1A601A68012AFCD1F5E711
:10214000C1218020C900C0054250D5E710BDC0465E
:10215000E00F00F0E40F00F0E80F00F0EC0F00F0EB
:10216000DFFF07C004050040186C004000EC06408B
:1021700014EC06407593000001704B1C0AD001233B
:102180008B404360044BC360044B0361044B4361C9
:10219000044B83607047C046080500500C05005092
:1021A000100500501405005008B5007840B200F04A
:1021B00023F808BD38B50023C356051C0C1C013399
:1021C00004D1094809492A22FFF732FE002C01D028
:1021D000012C07D10023A022EB56D205C133FF33D7
:1021E0009B009C5038BDC046C0BB020087BC0200AB
:1021F000704770477047000038B5041C0D1C431C25
:1022000004D10A480A491A22FFF712FEA023A400AB
:10221000DB05E018E0230C21DB00C258AD008A4347
:10222000C250C2581543C55038BDC046C5BB020098
:1022300002BD0200012310B50A4ADC00A458A142E5
:1022400007DA013BDB00D3185A680168064BCA5015
:1022500007E00133112BEFD180210268024B4905C1
:10226000D15010BD7CBD020024050000F8B50F1C44
:102270000121254BB9400360A023244CDB05161C2B
:102280001A59051C0A4380211A511A5909060A4392
:102290000121B1401A511A598A4396211A511A59EB
:1022A0008901520052081A51FFF7C4FF002204208E
:1022B0002B6817495A506C395850012199601960A0
:1022C000191CFC31CA6013495A506A6014391F3214
:1022D0005A5011495F5009185A501E517B1C03D0A7
:1022E000381C0321FFF788FF731C03D0301C032127
:1022F000FFF782FF0122094B291C1A6008480732A8
:1023000022F044F9F8BDC04600200040140500004A
:102310006C0500001C0500000C050000A40900204D
:102320002420002008B59623DB00994202DDFFF748
:1023300081FF04E09E210268014BC902D15008BD13
:102340002405000008B5C1230D4A9B00D158090699
:1023500003D50C49096A002908D1D3585B070DD56C
:10236000084B0021DB68002B01D107E00121064B5F
:102370001868002802D0054B1B68984708BDC04666
:1023800000200040FC200040A8090020AC090020EB
:10239000034B1960436803499B005A507047C0467D
:1023A000AC090020A809002000681E4B70B5C318B6
:1023B0005C4263415B00002A1AD0002903D0012946
:1023C00005D1802100E00421C12292008150FF2527
:1023D000C021C0245BB2DE00B540B1401248A40069
:1023E0000259AA430A43025101229A40026018E0AE
:1023F000002908D0012914D1C222802492008450DF
:102400008258920806E0C22204219200815082582C
:102410000339D209914304D001229A40131C034A84
:10242000D36770BD00E0FFBF00E100E004E100E021
:1024300003681A1CFC32D1680129FAD10021D1604D
:10244000A322D2009858C0B27047000003681A1C3B
:10245000FC32106A0128FAD100201062014AC9B288
:10246000995070471C05000001230E4A10B5936473
:1024700080230D499B00CB670C49101C0C6D0C4A46
:10248000002C04D000240C65116801311160094949
:102490000B601368A922D2008058190C80B21B046B
:1024A000184310BD0090004004E100E0FC900040A3
:1024B000B409002000E100E0F8B50F4C636C002B7C
:1024C0000FD000270D4E67643378BB4209D00C4B08
:1024D0001D68FFF7C9FF2D1ABD4202DC377002F0FC
:1024E000C9FE236D002B06D0064A13680133136022
:1024F0000022014B1A65F8BDFC900040B90900208C
:10250000B0090020B40900201B4970B50C78002CDC
:1025100030D10120194B1A4A586054608024E405D8
:10252000206050680028FCD00022012404251548B2
:102530001A500C30DC601D5008381A501248C22561
:102540001A50C1228020920000039850802040023F
:1025500098500E48AD0046590D4A3240C02636020A
:10256000324342518022893D9200FF3D4251026038
:102570001C600C7070BDC046B8090020009000407F
:10258000FC000040040500004C05000000E100E0F4
:10259000FF00FFFF08B5044B1B78002B01D1FFF7AC
:1025A000B3FFFFF761FF08BDB8090020104B70B5FD
:1025B0001B78041C002B01D1FFF7A6FF0D4D0E4E1A
:1025C0002B78002B02D033689C4210D0FFF74CFFD1
:1025D000201A0A2803DCFFF747FF0A30041C0123F6
:1025E0002B70A823054A3460DB00A4B2D45070BD20
:1025F000B8090020B9090020B0090020009000406F
:102600007047704708B58368984708BD704710B594
:10261000041C05F04AFF201C10BD0000F0B585B079
:102620001F1C0AAB1B88061C0D1C02920393002F73
:102630001AD0282005F03DFF6B46041C1A89039B25
:10264000A9B200933B1C00F02BFC3368301C5B6884
:10265000211C9847002808D0201C00F038FC201CC2
:1026600005F023FF024800E0024805B0F0BDC04677
:1026700016FCFFFF17FCFFFF72B601650B68002B0D
:1026800003D143658365086007E05A6D002A01D0D5
:10269000131CFAE758658365426562B67047036D9F
:1026A000002B12D072B6826D436D002A01D05365A3
:1026B00001E0026D1360436D002B01D0826D9A65BD
:1026C000002343658365036562B6704738B50B4BDD
:1026D0001C68002C10D0656D00F0CCFCA36C0029A8
:1026E00001D1834206D8201CFFF7D9FF201C0449E2
:1026F000FFF7C2FF2C1CECE738BDC046E409002000
:10270000EC090020F0B5041C93B00793230C02934E
:10271000284B04901C68284B05911E68069285B2D0
:102720000027002E43D0002C2DD0636D2349039346
:10273000A36C9AB21B0C8D4211D121498A420ED151
:10274000002B02D0029A93421BD1002F18D1201CDB
:10275000FFF7A5FF201C1B49FFF78EFF10E0002AA2
:1027600001D0AA420DD1002B02D0029A934208D187
:10277000201CFFF794FF201C1249FFF77DFF00E0AB
:102780000127039CCFE7104BEB18012B0FD9102327
:10279000291C0093029A0D4B08A800F081FB3368B6
:1027A000301C9B6808A9984708A800F090FB13B05C
:1027B000F0BDC046E0090020F0090020FE03000043
:1027C000FF030000EC09002002FCFFFF05270000CA
:1027D00010B572B60B4B1C68002C03D0201CFFF701
:1027E0005EFF08E062B65C2005F063FE00215C221B
:1027F000041C21F0E8FE0023E364034B201CE36388
:1028000010BDC046BC09002000400020024B1878D3
:10281000012318407047C046C0090020F7B5061CC8
:10282000FFF7F4FF041E33D11A4D2E60FFF7D0FFDF
:10283000194B1A491860FFF71FFFFFF7C9FF184B24
:102840001860184B4363184B8363286800280ED028
:10285000C027164E1649221C331C0097FFF7DEFED8
:10286000009728681349221C331CFFF7D7FE0C2061
:1028700005F01FFE0023838083710F4B03600F4B15
:10288000836000F00FFC01210D4A13780B43137095
:10289000F7BDC046F0090020C4090020EC09002063
:1028A000F4090020FC3F0020A92C000005270000AF
:1028B000FF030000FE03000010BE0200CD26000052
:1028C000C0090020F7B5002801D1002019E0002937
:1028D000FBD00193171C0D1C061CFFF779FF041E8B
:1028E000F3D0084B019A4363066045608760064B4E
:1028F000002A00D0054B201CA3630549FFF7BCFE4E
:10290000201CFEBDFC3F0020F12B0000912C00009C
:10291000EC09002038B5051C0C1CFFF777FF031EDF
:1029200005D00022281C211C131CFFF7CBFF38BD4B
:1029300070B5061C0C1C151CFFF768FF031E05D0A4
:10294000301C291C221C0123FFF7BCFF70BD38B5C9
:10295000051CEFF30884C36B006C1C1B6B6C1B1A0B
:10296000A3420CD21F2320349C43002801D000F046
:1029700045FA201C00F00EFA041928646C6438BD76
:10298000024B1868434258417047C046EC0900208A
:10299000002310B504499C006258002A01D001337D
:1029A000F8E76050101C10BDC8090020002310B5C6
:1029B000044A99008C58844201D00133F8E7002082
:1029C000885010BDC809002010B50024074BE058FE
:1029D000002802D003685B6898470434182CF5D1AE
:1029E000034B1B68002B00D120BF10BDC80900207D
:1029F000EC090020F8B5FFF709FF002855D02B4E51
:102A00003468351CE36CDA0718D502273B43E364CE
:102A1000274B1D680423EA6C281C1343EB64636B8B
:102A2000EB63FFF794FF281C696C02F090F83068A4
:102A3000C36C3B4239D002F0C4F836E01D4F1E4E45
:102A40003A68002A01D1326806E0216DB94203D10B
:102A5000616D002900D00A1C2A602A6831688A4208
:102A600008D11B0706D52C60FFF7AEFF3B68002B93
:102A7000FAD02B602B68A34217D03268934204D15E
:102A80000E4A5A630E4A9A6305E0944203D100202D
:102A9000191C021C06E0201CFFF759FF2B68201CA4
:102AA000191C626C5B6C02F011F8F8BDC4090020BF
:102AB000E8090020EC090020F4090020FC3F002078
:102AC000A92C000038B5114B051C1C68FFF79EFEB1
:102AD000002803D1281C02F0E0FB16E0E36CDB07C2
:102AE00006D5FFF775FE0A4B1860002800D0041CBD
:102AF00000F0C0FA2818A064201CFFF7D0FD201CAD
:102B00000449FFF7B9FDFFF775FF38BDC409002080
:102B1000E8090020E4090020F0B51E4B85B01C68D0
:102B20001D4B1A680393002A05D00F1C051CFFF7E4
:102B30006DFE002801D119482AE0E36CDB070ED5B1
:102B4000FFF746FE164B061E186008D0FFF7A7FDDC
:102B5000301C1449FFF790FD341CFFF74BFF3B047A
:102B60002B43A364201CFFF79AFD201C0E49FFF79E
:102B700083FD0E4B0020EB18012B09D9C0230093D5
:102B8000039B291C18683A1C094BFFF747FD0020DE
:102B900005B0F0BDC4090020F009002016FCFFFFBD
:102BA000E8090020EC090020E009002002FCFFFFFA
:102BB0000527000010B5FFF7AFFF041E01D1FFF796
:102BC00019FF201C10BD000010B5FFF71FFE0028E4
:102BD00009D0054C2068FFF762FD20680349FFF724
:102BE0004BFDFFF707FF10BDC4090020BC09002002
:102BF00010B50C1C8047A047FFF7E6FF10BD08B5D5
:102C0000FFF704FE002801D0FFF7DEFF08BD00003B
:102C1000F7B500282FD00C1C051CFFF7F7FD002886
:102C20002BD00726164F3868C36C1E4006D0281CD0
:102C3000211C144AFFF77CFE00261FE001F0A9FFCB
:102C400002213A68D36C1940019103D003218B43D0
:102C5000D36413E001263343D364201CA8473A68A9
:102C6000D36C191CB143D164019E5B0706D5201CAF
:102C7000FFF7C5FF02E0044E00E0044E301CFEBD2D
:102C8000C4090020FF2B000017FCFFFF16FCFFFF0C
:102C900038B5141C031C101C0D1C9847201CA84799
:102CA000201CFFF7ACFF38BD08B5FFF78DFEFFF71E
:102CB000A1FEFAE770B5124E051C3278022A1AD02E
:102CC00081421AD90C1A072C17D9081C0323284350
:102CD000034012D172B60B48D200155082185160D1
:102CE0008022A408120614432C603278013232701C
:102CF00062B6181C02E0044800E0044870BDC046FB
:102D0000F9090020FC09002013FCFFFF17FCFFFF5E
:102D1000031C70B58208980702D1181E01D137E054
:102D20000132541C72B621C9A84219D20368002B83
:102D300013DA5B005B08990041180E68002E01DA77
:102D4000A94202D3A34208D30DE080217600760881
:102D50009B19090619430160EDE79B00C018E3E7E2
:102D600062B6002014E00232934203D99200821826
:102D7000954204D803685B005B08036006E080218D
:102D80001B1B0906043A0B431360046062B604304F
:102D900070BD000070B5134A061C1378141C124D48
:102DA000002B0CD1114812492B70FFF783FF114BF8
:102DB000984202D11E2002F0EFFA01232370002472
:102DC0002B789C4209DA0C49E300C918301CFFF744
:102DD0009FFF002805D10134F2E7142002F0DCFA4D
:102DE000002070BDF8090020F909002030200020E3
:102DF0000038002017FCFFFFFC09002038B5002830
:102E00001FD0104B1C780023A34217DA0E49DA00BA
:102E10005558A84210D98A18526890420CD2041F03
:102E20002368002B02DC1E2002F0B6FA8023226801
:102E30001B061343236004E00133E5E71E2002F084
:102E4000ABFA38BDF9090020FC09002070B5041C5C
:102E5000081C0E1CFFF79EFF051C002C0ED000283E
:102E60000CD0231F1A689200B24200DD321C281CCD
:102E7000211C21F08BFB201CFFF7C0FF281C70BD1C
:102E800008B5081CFFF786FF08BD08B5081CFFF74A
:102E9000B5FF08BD08B5081C111CFFF7D7FF08BD1A
:102EA000F7B51D1C08AB1B88041C1030161C0F1C2A
:102EB000019301F0E7FA6A46002392882780668032
:102EC000A560201CE360A28063622362FEBD10B592
:102ED0008388041C9B0702D5806805F0E6FA201C55
:102EE00010BD82B030B5046A87B00B93051C0A92FE
:102EF0000123002C14D10AA9102202A821F046FBBC
:102F0000182005F0D6FA041C04A90822684621F00E
:102F10003DFB029A039B201C01F0E4FA2C621BE0AB
:102F20002269002A02D00133141CF9E7092B13DCB3
:102F30000AA9103202A821F029FB182005F0B9FADD
:102F4000051C04A90822684621F020FB029A039B75
:102F5000281C01F0C7FA256107B030BC08BC02B0DC
:102F60001847000070B5002816DD0C4B051C1A68C8
:102F70001C1C0B4E002A02D0306802F017F8FA2110
:102F8000256000243068074B89008361C46269436F
:102F900002F014F8201C00E0034870BD480A00202D
:102FA0000C0A00205130000017FCFFFFF8B5114F4C
:102FB000061C3D68002D0AD1302005F07AFA041C69
:102FC00002F06AF80C4BA5612360E5623C600B4D92
:102FD0002B68002B09D1102005F06BFA041C02F0BD
:102FE00048F8201C2C6002F01EF8301CFFF7BAFFD6
:102FF000F8BDC0460C0A0020D8BF0200380A0020E5
:10300000014B18687047C046480A002070B50D4C47
:103010002368002B03D00C4B1B68002B02D1062029
:10302000FFF7C4FF206802F015F8021C0749C31718
:103030000D684E685219734120680A604B6002F0B7
:103040000FF870BD380A00200C0A0020400A00204A
:1030500010B5FFF7DBFF0024054BE058002802D035
:1030600003681B6898470434282CF5D110BDC0466E
:10307000100A002008B5FFF7C9FFFA22034B92009F
:103080001868596800231DF02BFC08BD400A002079
:1030900008B5FFF7BBFF024B1868596808BDC0466A
:1030A000400A00200B4B10B51B68041C002B03D0FA
:1030B000094B1B68002B02D10620FFF777FF002386
:1030C000064A99008858002801D00133F8E78C504F
:1030D00010BDC046380A00200C0A0020100A00204B
:1030E000002310B5044A99008C58844201D0013362
:1030F000F8E70020885010BD100A0020082370B5A2
:10310000C3568AB0041C013304D1364836492C22F8
:10311000FEF78EFEE369E2681B68651D1A4204D162
:10312000EB7F0B2B06D8013303E0EB7F002B01D0A4
:10313000013BEB77EB7F082B0DD90123A2791A42D3
:1031400009D11A43A271A1881A1C06A801F0BAF984
:10315000FFF790FF2062EB7F012B26D80123A27995
:103160001A4222D00025A188A57102A8022201F0EE
:10317000A9F9A31DDE7F012E17D1FFF77BFF2B1CC2
:10318000226A801A994100900191019BA18806A8AA
:10319000AB4203D1154B009A9A4202D90422012373
:1031A00001E00322331C01F08DF90323A2791340BF
:1031B000012B14D1FFF75EFF0023226A801A994188
:1031C000994202D10A4B984209D90222A379A188D7
:1031D0001343A37106A80332012301F073F90AB067
:1031E00070BDC046C0BB0200D8BB0200E7030000B0
:1031F000DB05000010B5041C034B08330360FFF728
:103200006FFF201C10BDC04620BE020010B5041C7C
:10321000FFF7F0FF201C05F048F9201C10BD00004E
:10322000F0B5071C00250E1C85B002930AAB1B7875
:1032300008370393104B041C083303600192858008
:103240008571291C381C182221F0BDF9381C311C4D
:10325000039AFEF72DFE6B466A469B88127AA3807E
:10326000A31DE671DA77631D2562201CDD77FFF769
:1032700019FF201C05B0F0BD20BE02000630C1774A
:10328000704710B518C96210E10701D58158CB58B5
:103290008018984710BD08B5406C002102F03CF83A
:1032A00008BD0000F0B5041C85B0637A9C46002B75
:1032B00003D1201CFFF7EFFF69E0A37A01210193FE
:1032C0001023266F019AF35600259B18994002910E
:1032D000291CF3680393039B9D4231DAB368019A7A
:1032E0006B439B1872695B00E77AD3181A78587899
:1032F000E379012F04D15F1E3F1A101C3A1C0EE027
:10330000022F05D15F1EBA1A277A013F381A06E04C
:10331000032F04D1277A013FBF1A021C381C5B001F
:103320004343606F8218D3189B79634500DD634681
:10333000627B1A4202D00123AB4019430135CAE730
:103340001123C943F356606C994023691940029BCD
:10335000194301F0E1FFA37B072B18D8627B581CAF
:10336000520062730B499A00A073022B03D888584D
:1033700001F088FF99E7084B201C23630023636357
:10338000064B8958E4622364143001F017FE05B03F
:10339000F0BDC04650BE0200A532000083320000DE
:1033A00010B5041C044B036001F000FE201C01F06A
:1033B00097FE201C10BDC046D8BF020010B5041CEB
:1033C0000E4B08330360FFF78BFE201C743001F0B6
:1033D0009CF8201C603001F098F8201C583000F058
:1033E000D3FF201C503000F0CFFF201C044B1430C2
:1033F0006361FFF7D5FF201C10BDC04638BE020038
:10340000F0BF020010B5041CFFF7D8FF201C05F028
:103410004CF8201C10BD10B5041CFFF7C1FF201C88
:1034200005F043F8201C10BDF8B50025041C314BF5
:1034300085800833036085711430161C0F1C01F061
:103440002BFE201C2C4BE56263612564503000F09C
:10345000F1FF201C583000F0EDFF201C603001F01F
:1034600061F8201C33682667590009B20423F25E14
:10347000743001F0DBF83378226FE3717368A78052
:1034800023721023E572A5722561D35691685918ED
:103490008B4204DA0120984001330543F8E71123F9
:1034A000D168D35659188B4206DA01229A40206916
:1034B000013302432261F6E7142004F0FAFF226987
:1034C00000212A430123061C01F012FFFF22627231
:1034D000221C00230125483266646573A37323739D
:1034E000201C1370A366FFF7DDFDA379201C2B437E
:1034F000A371F8BD38BE0200F0BF0200F7B5437AF1
:10350000041C002B03D1201CFFF7C5FE64E0837A66
:1035100001219C461023066F0025F3566344994011
:103520000091291CF3680193019B9D422CDAB3683A
:1035300072696B4363445B00E77AD3181A78587852
:10354000E379012F04D15F1E3F1A101C3A1C0EE0D4
:10355000022F05D15F1EBA1A277A013F381A06E0FA
:10356000032F04D1277A013FBF1A021C381C5B00CD
:103570004343606F8218D3189B79002B02D001233C
:10358000AB4019430135CFE71123C943F356606CB3
:10359000994023691940009B194301F0BDFE667AEA
:1035A000B31EDBB2FC2B14D8FFF72AFD0B4B051C16
:1035B000236300230A4863630A4BFF21E462236408
:1035C00070431DF023F8291C4143201C143001F0E6
:1035D000F5FC637A012B96D9F7BDC04697320000FF
:1035E000B6030000833200001FB501228188131C3E
:1035F000684600F067FF012268460349131C00F08B
:1036000061FF05B000BDC046FE03000070B5051C9B
:10361000041C74350121281C01F040F9221C56328B
:1036200013780133DBB21370E17901318B4225D17C
:103630000023261C1370226D54360221525E3388FB
:103640002021934205DA201C19B2503000F0F8FE18
:10365000011CE2790023281C01F0D6F8226D338882
:103660000221525E934207DD231C002248331A7068
:10367000201CFFF7B9FF01E00133338070BD70B546
:10368000051C061C826D5C350221525E2B88041CD1
:1036900074362021934204DA19B2583000F0D0FE7B
:1036A000011C0022301C131C01F0AEF8A26D2B8807
:1036B0000221525E934207DD231C002248331A7018
:1036C000201CFFF791FF01E001332B8070BD73B523
:1036D000041C061C251C7436301C643500F030FFB9
:1036E0000023EA5E211C002360310093301C00F0AF
:1036F000F9FF002804D1231C6C331B78002B04D164
:10370000231C66331B78002B07D1231C002248336F
:103710001A70201CFFF768FF06E02A885BB29B182E
:103720002B8001236C34237073BDF0B5061C00217F
:10373000051C041C6636006E7156408864350023F3
:10374000EA5E4B1D1B1A201C85B06C3003909A4218
:1037500002DC0378002B24D1271C7437002A04DDF7
:10376000494209B2381C01F099F80023EA5E211C95
:103770000023381C0093603100F0B4FF0023F3569F
:10378000002B05D1221C48321370201CFFF72CFFA0
:103790000123039A137000222B88B256D3182B8072
:1037A0000DE0251C48352B78062B03D1201C7430E6
:1037B00000F0C6FE0023201C2B70FFF715FF05B09C
:1037C000F0BD38B5051C48352B78002B34D0041CCF
:1037D000FFF716FC221C4C321388C018231C80B241
:1037E00010804A331B88834226D8002313802B780D
:1037F000022B02D1201CFFF709FF2B78032B02D1EB
:10380000201CFFF73CFF2B78042B02D1201CFFF774
:103810005EFF2B78052B0BD02B78062B08D02B784E
:10382000072B09D10023201C2B70FFF7DDFE03E0DE
:10383000201CFFF77AFFF2E738BD1FB5036F827ACD
:103840009B68041C01339A4207D181880123684692
:10385000022200F037FE002306E0FFF74FFE201C97
:10386000FFF7AFFFA37A0133A3721FBD10B58379B1
:10387000DB0721D5027B041C022A02D1FFF7DDFF02
:103880001AE0837A016F0133DBB2837289688B425D
:1038900001D100238372002A02D1201CFFF72EFEE3
:1038A000237B012B05D163730023201CA373FFF737
:1038B000F9FC201CFFF785FF10BD00001FB5031C9D
:1038C00048331A78041C002A0DD000221A700132E5
:1038D0008188131C684600F0F5FD01226846044902
:1038E000131C00F0EFFD201C743000F029FE1FBDFA
:1038F000FF03000073B5079C051C002C09DB061CA8
:1039000048363078002806D03078012803D00D489A
:1039100016E00D4814E0069812B2C0B20090281CC0
:103920001BB2743000F0DEFE0020844207D02B1C56
:103930004A331C8007234C352880337000E0201C5C
:1039400076BDC04612FCFFFF17FCFFFFFF2902D81F
:103950004172002000E001487047C04617FCFFFF9D
:10396000407A704708B5743000F0EAFD08BD006980
:10397000002904DD002802D00139406AF8E77047C9
:10398000F8B5002927D00D1C071C00260469002C5F
:103990001ED00222A988A3884B40134216D111429F
:1039A00003D1AB889B0707D510E0A068A96801F098
:1039B000D0FC002804D1F4E7A368AA68934205D19B
:1039C0002B88002B09D022889A4206D0646ADEE751
:1039D000201C002E18D10D4816E06B88002B02D059
:1039E00062889A42F2D1EB68E268934201D0002BE0
:1039F000ECD17B68002B01D0201C9847A388044A97
:103A000001361343A380E1E7F8BDC04617FCFFFF72
:103A10000080FFFFF0B585B0002956D00D1C061CB4
:103A20000469002C1DD0AA880023920702D5A38820
:103A30009B07DB0F226829688A4210D1002B0AD02D
:103A4000A068A96801F085FC002808D0EB68E2684E
:103A5000934204D13BE0A368AA689342F6D0646A1B
:103A6000DFE730692A88071C031E22D0198891429B
:103A700005D2596A1F1C00290DD00B1CF6E7191C32
:103A80003B1C08E00C88944207D14F886C88A74201
:103A900003D80B1C496A0029F4D183420BD1198841
:103AA0008A4205D3914206D158886988884202D952
:103AB0006B62356102E0596A69625D626846094974
:103AC000012300F0FFFC002009E0074807E0A3887D
:103AD0001AB2002A02DA5B045B0CA380034805B02B
:103AE000F0BDC046FD03000017FCFFFF16FCFFFF02
:103AF000064B10B51A1C041C08322C33026083607C
:103B00000830FEF753FF201C10BDC04670BE0200F7
:103B100008B4024B9C46083808BC6047F13A0000E4
:103B200010B5041CFFF7E4FF201C04F0BEFC201CB1
:103B300010BD000008B4024B9C46083808BC604722
:103B4000213B000037B58388041C5A070FD59A061D
:103B500046D4DA060BD5011C08221831684620F03D
:103B600015FD22696369201CFFF7BBF938E00422C8
:103B70001343A380A3889A070BD5211C68461831EC
:103B8000082220F003FD22696369A06801F0CCFBE4
:103B900010E0DB0708D5E368206900936169A2693A
:103BA000E369A568A84705E020696169A269E3693E
:103BB000A568A8471022A38813420ED0256A002DBD
:103BC0000BD0A018291C20F0E1FC2B69281C2362D3
:103BD00004F06BFCFEF70EFFCCE704229343A380B6
:103BE00037BD00000C4A0023111C2C32083110B5DF
:103BF0004360838183738260036143618361C38314
:103C00000160041C0830FEF7C3FE044B1A68002A4A
:103C100000D11C60201C10BD70BE0200580A00209C
:103C2000031C72B64069002807D002695A61002A55
:103C300000D19A61DA8B013ADA8362B67047F7B540
:103C40000025071C2E1C0469002C1AD0A288636A68
:103C500011B2002911DA52070FD4002E01D13B61B5
:103C600000E07362636A201C0193FFF730F9201CA7
:103C700004F01BFC0135341C00E00193261C019C60
:103C8000E2E7281CFEBD0000F7B50E1C0125046903
:103C90000192002C37D0238832889A4201D0002B21
:103CA00026D1638872889A4201D0002B20D1FEF77A
:103CB000ADFD0123002806D0A288BF331340C03BCE
:103CC0005A425341DBB2019A934210D1A7883BB2CA
:103CD000002B0CDB201C311C1030102220F056FC75
:103CE0007B0607D4FEF792FD002803D006E00025EE
:103CF000646ACEE7201CFFF725FFF9E7211C034883
:103D0000FEF786FFF4E7281CFEBDC046453B0000D9
:103D100070B5012286B0041C0D1C8669FFF7B4FF44
:103D2000002827D1E38B092B24D8291C102202A8B4
:103D300020F02CFC182004F0BCFB051C04A96846EC
:103D4000082220F023FC029A039B281C00F0CAFBE7
:103D500072B6002E03D163692B61656102E033699D
:103D60002B6135612B69002B00D1A561E38B0133F9
:103D7000E38362B606B070BD82B008B502A90292B4
:103D80000393FFF7C5FF002008BC08BC02B018472A
:103D900038B5051CFFF753FF281CFFF741FF041E31
:103DA0000BD0211C0022281CFFF76EFF201C04F002
:103DB0007CFBFEF7E5FD0028EED138BD08B4024BD0
:103DC0009C46083808BC6047913D000010B518C9F2
:103DD0006210E10701D58158CB588018984710BD73
:103DE000F0B585B0041C01F079F8214B1B785B0716
:103DF0003CD50025236CC6B20227DF5FBD420EDA38
:103E0000201C29B2403000F01BFBB04205D101223A
:103E100068462021131C00F055FB0135EEE7251CF8
:103E2000231C4E3528884C33197801301CF0D4FC03
:103E3000231C50331B8889B28B4211D02B88A26C73
:103E4000D654636C2980002B10DB2A889A420DD14E
:103E5000012302225B426364684620219B1803E031
:103E6000684620210322012300F02CFB05B0F0BDA1
:103E70004C0A00200121024A13780B43137070474B
:103E80004C0A00200221024A13780B43137070473A
:103E90004C0A00200121024A13788B4313707047AB
:103EA0004C0A00200221024A13788B43137070479A
:103EB0004C0A002008B5002903DB024B196001F011
:103EC0004BF808BD500A002070B5041C1E1C04AB42
:103ED0001D7800F0F9FF201C0E4B4030236000F0ED
:103EE000A9FA231C01364C330135221C1E701D73A8
:103EF0000023E1214E32A3646365138053809381D4
:103F0000D381013B201C63644902FFF7D3FF201CCF
:103F100070BDC04658BB020038B5012A12D0031C40
:103F20004E33051C1888023B40181978141C1CF0ED
:103F300053FC69640025022C05D1211C2020FEF7CA
:103F400039FE00E0014D281C38BDC04617FCFFFFBC
:103F500070B5051C041C0A1C5035002907D1031C30
:103F60004E331B882A889A4212D111481FE001293A
:103F700006D12A88231C4E331B889A42FAD007E0C8
:103F8000022905D1031C4E331B88298899420AD087
:103F9000A36C28884C341E5C217801301CF01CFC7A
:103FA000301C298003E00121FFF7B6FFF0E770BD68
:103FB0000CFCFFFF4C3000787047031C50331A880C
:103FC000023B19881B888A4204D94C300078801A39
:103FD000C01800E0981A7047021C031C5C325A3368
:103FE00011881B88994205D9583011880278501AD7
:103FF000C01801E01088181A704710B5041C012978
:1040000005D1201CFFF7E8FF0028FADC04E00229B4
:1040100002D10020FEF756FD10BD08B50430002285
:10402000FEF7C2F908BD0000F0B5061C071C5C369F
:104030005A3733883A8885B09A421FD0104B1B7884
:104040001B071BD5041C3388426DD15C00F04AFF6E
:10405000231C30885833197801301CF0BDFB3B8895
:104060008DB2AB4209D1074968460222012300F014
:1040700029FA201C0121FFF7D0FF358005B0F0BDE3
:104080004C0A0020FF030000F8B5114D041C2B78EA
:104090001B0705D50121FFF7C0FF606DFEF7AEFEDF
:1040A0000827231C2E785833BE432E701878FEF74D
:1040B00071FE6065002808D0231C00205A335C3450
:1040C0003E4318802E70208000E00248F8BDC046B4
:1040D0004C0A002013FCFFFFF7B50F1C08A9051CB4
:1040E00009780430002A01D1DC070FD5002F0DD04C
:1040F000182618244E43AE1973614B1C5C43054BC4
:104100002C193261F7600122A36000E00022FEF763
:104110004BF9F7BDCD3D0000F0B5041C002589B07A
:10412000039104920593049B9D420EDA261C231CE6
:104130005A36378858331978781C1CF04DFB231CED
:104140005C331B8889B2994207D1059B012B0BD0A8
:1041500002210B48FEF7E0FC06E0039B626D5B5D0D
:104160000135D3553180DEE70123201C0093211C4B
:10417000044A0023FFF7B0FF281C09B0F0BDC04679
:10418000FF03000029400000F7B5194C2578AD0762
:1041900029D4002A29DD002927D01F1C161C0191D3
:1041A000051CFFF76FFE23781B0701D5002407E0ED
:1041B000281CFFF769FF0028F8D017E0B4420DDA99
:1041C000019B321B1919281C3B1CFFF7A5FF391C4A
:1041D0002418281CFFF711FF002FEFD1281CFFF730
:1041E00061FE201C02E0034800E00348FEBDC0461B
:1041F0004C0A00200DFCFFFF17FCFFFF10B5131C3D
:104200000A68111D0224125FFFF7BEFF10BD0000F7
:10421000F0B5174E87B03378051C5B0705D5002134
:10422000FFF7FBFEA86CFEF7E9FD04273378BB43DC
:1042300003936B461B7B33702B1C4C331878FEF7B3
:10424000A9FDA864002810D02B1C00244E331C802C
:104250005C80039B281C1F433770291C0094054A6F
:10426000231CFFF739FF201C00E0034807B0F0BD16
:104270004C0A0020E13D000013FCFFFFF7B52C4C79
:104280002578ED0751D41F1C161C0191051CFFF762
:10429000F1FD23785B0703D5002F14D13C1C0AE005
:1042A000281CFFF7B5FF0028F6D03FE0B44237DA0C
:1042B000019B18550134281C0021FFF749FE1D4BB6
:1042C0009842F3D12CE0019C012F0ED1019BE31AFF
:1042D000B34206DA281C0121FFF73AFE20700134B0
:1042E000F4E7F443E41734401AE00024022F17D116
:1042F000281CFFF762FE864207DD281CFFF75DFEE3
:104300003A1C311A281CFFF707FE0024B44207DAD2
:10431000281C0221FFF71CFE019B18550134F5E70C
:10432000281CFFF7B7FD201C00E00348FEBDC04677
:104330004C0A00200CFCFFFF0DFCFFFFF7B5151C1D
:1043400000AF7B602B1C0E1C69460833DB08DB00CA
:10435000CB1A9D4601320021041C684620F033F937
:10436000301C69462A1C7B68FFF788FF002803DCA5
:10437000201C00F05FF804E002B26946201C00F047
:104380002FF8BD46201CFEBD10B5041C006800F0CF
:104390001EFB201C10BD70B5061C081C0D1C21F056
:1043A00009FC041C0530FEF7F5FC306000F002FB50
:1043B0003068291C4480621C043020F0E7F870BD8E
:1043C00010B5041C002902D00B78002B02D1034B3E
:1043D000236001E0FFF7DFFF201C10BDACBE020030
:1043E000F8B5051C0E1C141C00290AD00B78002BF4
:1043F00007D0002A05D0081C97B221F0DBFB8742CA
:1044000002D90B4B2B6010E0601DFEF7C3FC286047
:1044100000F0D0FA2868221C4780311C043020F0BC
:10442000B5F82B681C1900232371281CF8BDC04661
:10443000ACBE0200014B03607047C046ACBE020038
:104440000023994207DB02680223D05E00238842E2
:1044500001DD51180B79181C7047000010B5054894
:10446000054C206000F0A9FA201C0449044A04F01D
:1044700015F810BDACBE0200540A002089430000AC
:1044800000000020002310B503804380041CFEF7C9
:10449000FFFDA060E160201C10BD0000084B73B55B
:1044A0001D68002D0BD0011C041C2E680831082249
:1044B000684620F06BF80CCC3168281C884773BD27
:1044C000580A002038B501804280041C1D1CFEF7EC
:1044D000DFFDA060E160002D02D0201CFFF7DEFFB1
:1044E000201C38BD82B010B5041C03930292FFF764
:1044F000C9FF201C02A9102220F048F80023201C2C
:10450000236110BC08BC02B0184710B5041C006839
:1045100000F05DFA201C10BD08B50A1C002120F037
:1045200052F808BD014B03607047C046B4BE02009C
:1045300010B5041C0868206000F03FFA201C10BD74
:1045400008B503685988981D9B885943FFF7E4FF15
:1045500008BD000030B504686088814206DAA5888D
:10456000AA4203DA002901DB002A01DA034804E049
:104570005043611808188371002030BD17FCFFFFFD
:10458000F0B5071C85B00D1C1E1C002923DD002A78
:1045900021DD002B1FD0046863880391994200DD60
:1045A0000393A38802929A4200DD0293002306340B
:1045B0000193019B029A93420BD0201C311C039A59
:1045C0001FF0E4FF3B6876195B88E418019B013318
:1045D000EEE7002000E0014805B0F0BD17FCFFFF4A
:1045E000F8B5041C0E1C151C1F1C002901DB002A39
:1045F00002DA0D4B236015E0101C48430630FEF72D
:10460000C9FB206000F0D6F92368201C5E809D80E5
:10461000002F05D0311C2A1C3B1CFFF7B1FF01E025
:10462000FFF78EFFF8BDC046B4BE020010B5041CF3
:104630000023FFF7D5FF201C10BD0000F7B5051CB7
:104640000C1E05D000200F1C061C0190011C15E05B
:10465000234B036041E03022524294469C44624620
:10466000092A14D90A2B0DD1019B36180133019365
:10467000B14200DA311C0020061C01373B78002BC8
:10468000E9D106E00028F8D001360020F5E7012046
:10469000F3E76A46928809B212B2281CFFF7A0FF1E
:1046A0002B689A1D01235B422078002815D0011C3D
:1046B0003039092909D8591C4E1EB14149420B40D5
:1046C0000A214B431B18303B05E0591C03D01370E3
:1046D000012301325B420134E6E7281CFEBDC046DF
:1046E000B4BE0200F0B5071C89B00EA80078059191
:1046F00007903868049046880020B24200DB81E0D1
:10470000049CA488A34200DB7CE00D6803956D88BF
:10471000AC46151C65440195854273DD039DAD884B
:104720005919069181426DDD002A05DA019902913D
:10473000B14207DD029605E0B11A0291614501DD43
:1047400061460291002B05DA06990191A14206DD2E
:10475000019404E0E11A0191A94200DD019555425E
:10476000D01728400025039C0634AB4202DA61468C
:104770004D425D4328182118D443E41722400024F9
:10478000049803910630A34201DD73431C1C079B70
:10479000A2188418002B02D1059D1E1C1BE00022CC
:1047A000101C019B9A422DDA002302998B4207DAF2
:1047B0000399CD5C002D01D0E55401300133F4E7BD
:1047C000059B03991B6801325B88CB1803933B68F8
:1047D0005B88E418E5E7019B9E420EDA201C029AF2
:1047E00003991FF0D3FE2B68039A5B880136D31818
:1047F00003933B685B88E418EDE7D843C017184083
:10480000029B584309B0F0BDF0B5041C87B004A862
:10481000151C1E1C0F1C00F0C1FE23685A8895420F
:1048200008DA9B889E4205DA1F2F03D9059B009367
:104830009F4201DD18482DE005230021203F7B43E6
:104840000193049B0293019A029B9B185B5C0022DC
:1048500003938B199C4653192768009378888342E9
:1048600002DABB889C4507DB0132052AF3D101310E
:104870000529E8D100200DE063465843009BFB1852
:10488000102717411818039B1F407B1E9F417F4232
:104890008771E9E707B0F0BD17FCFFFFF7B50368C4
:1048A0009E1D5B885A1A019200291CDD0C1C051CF8
:1048B0000027994202DBFFF743FE12E02B689B883A
:1048C0009F420EDA3119301C019A1FF05FFE019BE6
:1048D000211CF018FFF720FE2B6801375B88F618C3
:1048E000ECE7002000E00148FEBDC04617FCFFFFDA
:1048F00010B50548054C206000F05FF8201C044905
:10490000044A03F0CBFD10BDB4BE02005C0A0020D7
:104910000B4500000000002010B5041C006800F0EA
:1049200056F8201C10BDF8B5D443E4171440071CFA
:10493000201C0C301E1C0D1CFEF72CFA386000F0F9
:1049400039F83B681C7238684660002D04D0093085
:10495000291C221C1FF01AFEF8BD0A1C002110B5EC
:10496000041C0B1CFFF7DFFF201C10BD10B5054C0D
:104970000121201CFFF7F1FF201C0349034A03F02B
:104980008DFD10BD600A00201949000000000020C4
:1049900008B5074A03880120934208D0834202D019
:1049A0000020DB0703D41E2000F0F6FC002008BD29
:1049B000FFFF000003230380704710B5041CFFF7BE
:1049C000E7FF002802D123880233238010BD10B5F1
:1049D000041CFFF7DDFF002809D12388023B9BB2AE
:1049E000012B01D0238002E0201CFEF707FA10BD46
:1049F00038B5142811D8094B8000C5580C1C281C48
:104A0000FDF708F9002808D0054B5A5D002A01D0AF
:104A100000225A55211C02F097F838BD10BF020041
:104A2000640A0020F8B5142801D9002016E00C4BC8
:104A30008000C558281CFDF7EDF8041EF5D0094E7E
:104A4000775D002F07D102F0C1F8201C391C02F05D
:104A500001F901237355201C02F0B8F8F8BDC046D7
:104A600010BF0200640A002000B5142816D80C4AB2
:104A700083009B58032911D8A022081CC133FF339F
:104A8000D2059B001BF01EFD02080406002104E075
:104A90000C2102E0042100E00321D15000BDC046FA
:104AA000BCBE0200031C0020142B0BD8A222A021A4
:104AB000D200C9058A5804499B0058580123C240B6
:104AC000101C18407047C046BCBE0200002815D01C
:104AD000006041608260C360046145618661C761B6
:104AE000444604624C464462544684625C46C46256
:104AF000644604636E46466374468463002A06D0A7
:104B0000C46B043C043A25681560B442F9D18C6B3F
:104B1000A6464E6BB546002B06D0CC6B043C043B3E
:104B20001D682560B442F9D10C6BA446CC6AA3463B
:104B30008C6AA2464C6AA1460C6AA046CF698E696F
:104B40004D690C69CB688A680868496870470060DD
:104B500041608260C360046145618661C76144460B
:104B600004624C464462544684625C46C4626446B5
:104B700004636E46466374468463C46B043C043924
:104B800025680D60B442F9D1C76986694569046931
:104B90007047006041608260C36004614561866166
:104BA000C761444604624C464462544684625C4693
:104BB000C462644604636C46446374468463046957
:104BC0007047846BA646446BA546046BA446C46A32
:104BD000A346846AA246446AA146046AA046C769FD
:104BE000866945690469C3688268006841687047DE
:104BF00010B518C96210E10701D58158CB5880184B
:104C0000984710BD08B500F0C3FB08BD82B030B5B1
:104C100085B00892051C082202A809931FF0B6FC73
:104C2000039B029C5810DB0701D52B581C592D18EB
:104C30000AA9684608221FF0A9FC089A099B281CAB
:104C4000A04705B030BC08BC02B0184782B01FB501
:104C5000041C06920793120C1A2A14D00AD8042AAC
:104C600023D0052A27D1E6235B0001A8E15801F0F3
:104C700078F820E01B2A18D01C2A1CD1E130FF3024
:104C800002F0D2FA17E06930FF300021FEF7F6FAA1
:104C9000201C9130FF300021FEF7F0FA201CB930C3
:104CA000FF30012101F074FE05E0E4235B0001A860
:104CB000E15800F0E4FE1FBC08BC02B01847000039
:104CC0001423F0B5041C97B0192200931821043066
:104CD000FFF7FAF8231C251C261C6433181CB43576
:104CE00013211493B836FDF759F8281C02F04EF939
:104CF0001E210022301C01F021FC201CD030FEF7C8
:104D000071FF231CF033181C0621444A1593FEF74B
:104D10008BFB201C002701226930131C00971121F6
:104D2000FF30FEF77DFA201C913000971A210222F5
:104D30000123FF30FEF774FA201CB9300121022252
:104D40001A23FF3001F07CFE301C00F097FCE423B6
:104D50005B00E050301C00F02DFFE6235B00E050CC
:104D6000011C201C043BD130E2580095159BFF30FC
:104D700001F0A4FB201CE130291C1C22FF3002F0B2
:104D80001FFA0A23201C009301330193013302937D
:104D900001330393013304930133059301330693E5
:104DA00001330793013308930133099301330A93C5
:104DB00001330B9301330C9301330D9301330E93A5
:104DC00001330F930833109301331193F9300133FA
:104DD0000822129307211A3BFF3001F016FCD6235C
:104DE0009B00E0181D2101F053FF14982770032148
:104DF000FCF7FDFF231C221C201C09499C33A03218
:104E00001C6011605760074A80305A6102210122FC
:104E1000FDF7F0F9201C17B0F0BDC04694BF0200AA
:104E2000054C0000F14B00000123F0B5057885B07A
:104E30001D4040D1031CD0330090181C0193FDF796
:104E4000EDFC00F087FB282003F033FB041C10303E
:104E5000FFF718FB194B65802380182003F029FB0E
:104E6000061C071C164B291C0293009B102208C627
:104E7000301C03951FF0A7FB02A9301C08221FF06D
:104E800085FB104B01987B611223A760E560A3802E
:104E900025626562211CFEF7BDFD002805D0201C9F
:104EA000FEF715F8201C03F000FB0122009B1B7885
:104EB0001343009A137005B0F0BDC046FD03000017
:104EC0004D4C00000D4C000010B5041C00F026F8FD
:104ED000014B201C236010BDB8BF020008B500F0D4
:104EE00043F808BD08B500F044F808BD18234A1C73
:104EF0005A438218926810B55943002A05D14118C7
:104F0000CB68002B08D0984706E04318D8680028E3
:104F100002D0191C1031904710BD000038B50C4B61
:104F2000041C0360002343608360C3600362436228
:104F300083639623051D9B01C363281CFDF796F927
:104F4000281C0449221CFDF723FA201C38BDC0464A
:104F5000C8BF0200ED4E000038B50D1C041C043023
:104F6000FDF7E0F9E56338BD08B50430FDF760FAF8
:104F700008BD10B50C1C0430FDF768FA201C10BDEC
:104F800010B5041C43694268991800F09BF8E36A65
:104F9000002B04D1A369002B07D0984705E0A06936
:104FA000002802D0211C1C31984710BD10B5041CEC
:104FB00000F090F80023A361E36210BD38B5051C32
:104FC0000C1C00F087F86C61286900F04AF901199F
:104FD000281C00F077F838BD08B5C36A011C002B07
:104FE00004D18369002B06D0984704E0806900282B
:104FF00001D01C31984708BD10B5041C044B036058
:10500000FFF7D4FF201C00F06BF8201C10BDC04639
:10501000D8BF020010B5041CFFF7EEFF201C03F000
:1050200044FA201C10BD036810B5002B06D1041CE7
:10503000C06800F016F901236060236010BD10B550
:10504000041C0068002804D0E06800F00AF96368D6
:10505000C01A10BD10B58468FFF7F1FF201810BD0D
:1050600010B5041CC06800F0FCF800236060A36069
:1050700010BD002310B5036043608360041C00F082
:10508000F5F8E060201CFFF7EBFF201C10BD08B511
:1050900003689B68984708BD084B10B50833036048
:1050A000002343608360C360041C00F0DFF8044900
:1050B000206100F072F8201C10BDC04600C0020044
:1050C0008F50000008B50A1C031C011D006900F088
:1050D00090F808BD08B5011D006900F0A6F808BDEC
:1050E00010B5041C034B08330360FFF7F3FF201CCB
:1050F00010BDC04600C0020038B50023C356041CD2
:105100000D1C013304D1064806492422FCF790FE09
:105110006368002D01D0E26800E02269136038BDA9
:10512000C0BB0200D8BB020000B599B0684603219D
:10513000FCF7D7FE06A80221FCF7D3FE0CA801213C
:10514000FCF7CFFE12A81021FCF7CBFE6846012128
:10515000FFF7D2FF06A80021FFF7CEFF0CA8002121
:10516000FFF7CAFF12A80121FFF7C6FF962000F043
:1051700094F868460021FFF7BFFF06A80121FFF75A
:10518000BBFF0CA80121FFF7B7FF12A80021FFF712
:10519000B3FF962000F081F8D8E738B5041C0D1C49
:1051A00003681B68984763681D6038BD38B503689D
:1051B000041CDB68984763685A682368002A02D198
:1051C0009B68984714E05B681568984763682D1AD8
:1051D000002D08DC5A68916859601B68002BEAD0E2
:1051E00050689847E7E75A68216810680B69984744
:1051F00038BD70B50D1C72B64B60002346680A605E
:105200007468002C05D02168511A02D4231CA468AC
:10521000F7E7002B05D1036875601B69101C9847E0
:1052200000E09D60AC6062B670BD08B572B64268C1
:1052300053688B420CD19B6853600268002B02D1EB
:10524000936898470BE012691868904707E0131CB1
:10525000002B04D09A688A42F9D18A689A6062B6B3
:1052600008BD08B503685B68984708BD00487047EB
:1052700028C0020008B50248FFF798FF08BDC046E5
:1052800028C0020038B5041CFDF784F9051CFDF7A1
:1052900081F9401BA042FAD338BD08B5FA239B0020
:1052A0005843FFF7EFFF08BD10B5002906D00129CC
:1052B0001DD1002310E001311F2918D001238B409C
:1052C00002691A42F7D002688B00D31800221A60D4
:1052D000F1E701331F2B0AD001210A1C9A4004690F
:1052E0001442F6D004689A00A2181160F1E710BDCC
:1052F0000261064A08B54260054A01738260054AA8
:10530000191C0260FFF7D0FF08BDC046040500501D
:105310001005005000070050426800691368014002
:10532000834319431160704782B073B5041C061D96
:10533000069208A96846082207931FF027F96569B5
:10534000311C069A079B2068A84773BC08BC02B0B2
:105350001847026808B594460A680023944507D1A7
:105360000430043110221FF002F943424341DBB202
:10537000181C08BDBFF34F8F024A034BDA60BFF31E
:105380004F8FFEE70400FA0500ED00E000207047B3
:1053900008B5FFF7EFFF0000F0B597B01822002125
:1053A000061C10A81FF00FF910A81321FCF77BFDB5
:1053B00010A80321FCF7F8FE01225C4B00921B6849
:1053C000002B01D0DBB2009300240BA80021584A27
:1053D0000123FFF78DFF221C564BB342624153421B
:1053E0001E4072B6544B1022211C07A81F681FF0E4
:1053F000EAF8524B6421301C07931BF007F90A218D
:105400001BF0EAF905251031694379180891301C21
:105410000A211BF0FBF80A211BF0DEF91031694369
:1054200079180991301C0A211BF0D6F9802310311C
:105430004D439B017F190A970193009B002B57D086
:1054400000263F4B751E1D4004D50423013D5B42E1
:105450001D430135B300049300230293032C03D1B1
:10546000802300249B010193049A07ABD758354A47
:1054700063000133D318002203921878385C05903A
:10548000581E00788446102061460841059908425C
:1054900004D0012090400399014303910132063367
:1054A000092AEAD1039B07AAD943274B09011940CE
:1054B000AB009B589F4205D1029B312B02DC0BA80D
:1054C000002102E0019B0BA81943FA27FFF724FFF4
:1054D000FF0010AB1B785BB2013304D11B481C49A1
:1054E0002C22FCF7A5FC159B119A1B681A4201D1CE
:1054F000FFF740FF013F002FEBD1019B01345B0020
:105500000193029BE4B201330293FA23029A5B00F7
:105510009A42A3D10136042E93D1044B1B68002B71
:105520008BD0009B013BDBB2009386E7840A00200E
:10553000F0FF0000E7030000280000206EC002001A
:105540000300008030C00200F01F0000C0BB02005A
:10555000D8BB0200002201210D4B30B51A600D4A64
:10556000042411601A1C196800200B4B58605D68F8
:105570000848002DFBD0A123DB00C3580902013CE1
:105580001943002CF0D101231160436030BDC046A7
:10559000880A002000D00040FCD00040021C10B55A
:1055A000014B12CB12C210BD8C0A0020034A044BDF
:1055B00012681A607E225A607047C0462800002098
:1055C0008C0A002038B50368041C01811B6A9847C7
:1055D0002368051C5B69201C98472081281C38BD66
:1055E0000089704738B50368041C81721B6A9847AC
:1055F0002368051CDB69201C9847A072281C38BD55
:10560000807A70470048704716FCFFFF00487047DB
:1056100016FCFFFF704710B5041C02F046FF201C6B
:1056200010BD00008280142210B5134C00230834F2
:1056300004600281041C021C416202218371303229
:105640003634C360036143618361C3610362817265
:1056500013705370227843868A43F1310A4083865F
:105660002270021C40321370021DD387013343871E
:105670008387C38710BDC04668C20200F0B5061C10
:1056800097B0FCF787FF504B9842FAD94F4F3B68D1
:105690000593002B00D08BE006AC21211C220B339C
:1056A000201C01F005FA0EAD22211D220B230AA8B1
:1056B00001F0FEF923211B220B23281C01F0F8F92D
:1056C000082002F0F6FE0121059B0A1C049001F05F
:1056D000E7FD301C3A2102F031FE00281CD0A388DF
:1056E00012ADAB80A3795C20AB71394B1293A368E8
:1056F0001493237B2B73637B6B73A37BAB7302F0DD
:10570000D8FE3A230093363B0193311C2A1C049B9C
:10571000041C02F0E5FD21E0301C322102F08AFB7E
:1057200000281DD0A38812ADAB80A3795C20AB719B
:10573000274B1293A3681493237B2B73637B6B73A8
:10574000A37BAB7302F0B5FE322300932E3B019393
:10575000311C2A1C049B041C02F03EFB3C6027E029
:10576000301C3C2102F07CFA002821D0AB8812AC1E
:10577000A380AB79A420A371154B1293AB6814934B
:105780002B7B23736B7B6373AB7BA37302F091FE64
:105790003C23051C0093383B019301330293311CD9
:1057A000049B221C02F01CFA0A4B3D6044351D602C
:1057B000084B064C1868002802D0216800F0BCFA9B
:1057C000206817B0F0BDC0464FC30000940A002007
:1057D00058C20200980A0020C2680169436949431F
:1057E00052435B438818C01870470000F0B5604909
:1057F000C56885B08D4206DA031C36331A78022359
:1058000013400BD117E0C82200235200954212DD4D
:10581000031C36331A78002392070CD40123061C8C
:105820001F1C363632785408A7433C1C02279C4084
:10583000BA432243327004698C4205DA021C3632C4
:105840001278520709D415E0C8225200944211DDA3
:10585000021C3632127852070CD4061C012236364E
:1058600033789F08BA439700042293431A1C0123FC
:105870003A43327042690192021C019E40328E42CC
:1058800005DA011C3631097809070AD415E0C82168
:10589000019E49008E4210DD011C3631097809074E
:1058A0000BD4061C012136363378DF08B9430827AC
:1058B000C900BB430B43337001E0002B18D01378B1
:1058C000032B15D80133DBB21370012B03D1002158
:1058D000031DD9870CE0042B0AD1021C01213632AA
:1058E000137804300B4313700023C3870B333CE061
:1058F00013780293002B1BD0061C0127011DCB8FB0
:10590000363601339BB2CB8703963678BC46374098
:1059100008D01D2B0CD963469E43039B1E700023A9
:10592000CB8704E0092B03D9029BCF87013B13707F
:10593000FFF752FF0F4A0723904216D90E49043B46
:105940008D4212DBC8220133920095420DDC023BEE
:105950008C420ADB013B944207DC01980433884205
:1059600003DB0133904200DC0023181C05B0F0BDBE
:1059700070FEFFFFFF700200E0FCFFFF7FB5041C1C
:10598000FFF72AFF251C9023061C31351B04984283
:105990002AD9638F002B07D1013368461B210822C7
:1059A000FEF790FD0123638790239B049E4219D943
:1059B000A38F002B07D1013368461B210922FEF774
:1059C00081FD0123A3878023DB049E420AD9E38F54
:1059D000002B07D1013368461B210A22FEF772FD16
:1059E0000123E38700232B702B78042B02D801338B
:1059F0002B7003E00023E387A3876387201CFFF756
:105A0000F5FE021E0B2A13D0231CA18E30338142D7
:105A100004D11A78042A04D8013201E00022A086B9
:105A20001A70A28E618E914208D01B78042B05D982
:105A3000628668461B210123FEF744FD7FBD30B519
:105A4000041C036A8BB0009302AD616A8269C3696A
:105A5000281C01F068FC231C0C3307CD07C302226D
:105A6000A379201C9343A371FFF788FF0122A1882B
:105A700006A8131CFEF726FD00200BB030BD38B57C
:105A80000C1C051C0B68081C5B6A9847211C2B1C0E
:105A90000C3115C915C3281C38BD10B5041C03688A
:105AA0005B6A9847E06810BD10B5041C03685B6A28
:105AB0009847206910BD00000048704716FCFFFFA2
:105AC00038B50368041C01811B6998472368051CCD
:105AD0009B69201C98472081281C38BD008970478D
:105AE0000048704716FCFFFF704710B5041C02F019
:105AF000DCFC201C10BD30B5041C436BC26801697E
:105B00009A1A83698BB05A43836B92125B1AC169EC
:105B100042634B439B128363C16B406902AD091A18
:105B2000206A41438912E1630091281C216C01F035
:105B3000FAFB231C283307CD07C30122A18806A83E
:105B4000131CFEF7BFFC00200BB030BD002310B5C6
:105B50008371643303810368041C81801B69984747
:105B60000222A3799343013A1343A37110BD0000AD
:105B7000002310B5041C838083710D482164083014
:105B800020608020C000A061E0612062E360201CF2
:105B9000236163616362A362E36223636363A3635C
:105BA000E3636364111CFFF7D1FF201C10BDC046E6
:105BB000A0C20200F0B5061C97B0FCF7EBFC4F4BFF
:105BC0009842FAD94E4F3B680593002B00D08BE0EA
:105BD00021211C220B3306A80AAC00F069FF0EAD90
:105BE00022211D220B23201C00F062FF23211B22F7
:105BF0000B23281C00F05CFF082002F05AFC012156
:105C0000059B0A1C049001F04BFB301C1D2102F087
:105C1000ADFA00281CD0A38812ADAB80A379602018
:105C2000AB71384B1293A3681493237B2B73637B64
:105C30006B73A37BAB7302F03CFC1D230093183BFA
:105C40000193311C2A1C049B041C02F065FA21E01C
:105C5000301C3C2102F0A4F900281DD0A38812AD0D
:105C6000AB80A3796020AB71264B1293A368149389
:105C7000237B2B73637B6B73A37BAB7302F019FCE9
:105C80003C230093373B0193311C2A1C049B041CCA
:105C900002F05CF93C6027E0301C3C2101F0E0FFA1
:105CA000002821D0AB8812ACA380AB79A420A371CB
:105CB000144B1293AB6814932B7B23736B7B63732E
:105CC000AB7BA37302F0F5FB3C23051C0093383B30
:105CD000019301330293311C049B221C01F080FFCD
:105CE000094B1D6044353D60074B1A68044B002A80
:105CF00001D019684A64186817B0F0BD4FC300009E
:105D0000980A002058C20200940A002084B030B5DE
:105D10000693031C0491059204AC0C3326CC26C3D5
:105D200026CC26C322681A6002228379134383712A
:105D300030BC08BC04B018474164704773B50C1CF4
:105D4000051C161C0B68081CDB699847E36B281CB4
:105D500001960093626BA36B216C01F0A5FA281CDD
:105D600076BD38B50C1C051C0B68081CDB69984710
:105D7000211C2B1C283115C915C3281C38BD82B025
:105D800030B585B00892051C082202A809931EF0C0
:105D9000FDFB039B029C5810DB0701D52B581C59B7
:105DA0002D180AA9684608221EF0F0FB089A099BE4
:105DB000281CA04705B030BC08BC02B01847F8B595
:105DC0000A6803680E1C071C981A1BF07DFC726899
:105DD0007B68051C981A1BF077FCBB68041CB06834
:105DE000181A1BF071FC291C061C281C1BF09CF9BE
:105DF000211C051C201C1BF097F9011C281C1AF003
:105E000025FE311C041C301C1BF08EF9011C201CCB
:105E10001AF01CFEF8BDF0B585B001900291039216
:105E2000FFF7CDFF0125041C071C039B9D4216DADA
:105E30000C216943029B01985918FFF7C0FF211CF0
:105E4000061C1AF025FD002800D0341C301C391C1B
:105E50001AF032FD002800D0371C0135E5E7381C68
:105E6000211C1BF093FA05B0F0BDF0B58BB009937F
:105E70008023DB000025C360036143610023041C11
:105E80000791089205604560856085610293119BCA
:105E90009D4217DA0C216943109B07A85918FFF798
:105EA0008EFF1DF077FA1AF0B9F91DF0CFF91BF04B
:105EB0000BFC0299061C1AF0FFFC002800D0029689
:105EC0000135E4E700270023109D05930197009713
:105ED0003E1C059B119A93425EDA291C07A8FFF726
:105EE0006EFF1DF057FA1AF099F91DF0A7FA03900A
:105EF000039902981AF026FFFE2189051BF046FA45
:105F000004901BF0C1FB0690301C1BF0BDFB069EED
:105F1000864200DA061C301C1BF0D6FB2B68079A61
:105F2000061C981A1BF0D0FB03991AF00BFF4100D6
:105F3000490804981BF0F8F8011C00981AF086FD37
:105F4000089B00900693069A6B68981A1BF0BCFB9E
:105F500003991AF0F7FE4100490804981BF0E4F891
:105F6000011C01981AF072FDAB68019009980C357C
:105F7000181A1BF0A9FB03991AF0E4FE4100490826
:105F800004981BF0D1F8011C381C1AF05FFD059B2A
:105F9000071C013305939CE70098011C1BF0C4F813
:105FA000051C0198011C1BF0BFF8011C281C1AF0ED
:105FB0004DFD391C051C381C1BF0B6F8011C281CB3
:105FC0001AF044FD1DF0E6F91AF028F91DF036FA32
:105FD000051C291C00981AF0B5FE011C301C1BF092
:105FE000A3F8FE2189051AF031FD8921C9051BF0AE
:105FF0009BF81BF049FB291CE06001981AF0A2FEF7
:10600000011C301C1BF090F8FE2189051AF01EFDC2
:106010008921C9051BF088F81BF036FB291C20617B
:10602000381C1AF08FFE011C301C1BF07DF8FE217D
:1060300089051AF00BFD8921C9051BF075F81BF0C5
:1060400023FB079B60612360089B029800936360B9
:10605000099BA3601BF018FBA061201C0BB0F0BDD6
:10606000F0B50026041C151C0B1C371C301C321C00
:106070008FB00591AA4208DA1968013240185968B0
:106080007F1899680C337618F4E7291C1AF0BEFAC9
:10609000291C2060381C1AF0B9FA291C6060301CD9
:1060A0001AF0B4FA0599A0602A1C201CFFF7B3FE71
:1060B0000026069004960396C8235B420293C823E9
:1060C0005B420193C8235B420093221C0BAB83CA43
:1060D00083C32268029B944663440B93019A1F1C5E
:1060E00063680599D318A268079394460C93009BA4
:1060F0000BA863442A1C08930D93FFF78CFE0699A6
:1061000009901AF0C5FB002805D0079B089E049350
:10611000099B03970693009BC8330093C823009AFA
:106120005B009A42D1D1019BC8330193131C019AA1
:106130009A42C7D1029B019AC83302939342BED1BF
:10614000039B2268934206D1049B6268934202D16A
:10615000A3689E4205D0039BA6602360049B6360F6
:10616000AAE7201C0FB0F0BD70B5041C0E1C151C56
:1061700086B003A8FFF774FF201C009601950399D1
:10618000049A059BFFF771FE201C06B070BD00004D
:1061900082B0F0B5041CEBB0642071937092FFF7ED
:1061A0007CF805210EA80A1CFEF740FA0FA89149B9
:1061B000FEF744FA002300251FAA9D50D21855600F
:1061C000956096220C3352009342F4D1143AFF3A70
:1061D000291C11A81EF0F7F9A068FDF7C1FB2E1CC1
:1061E0000990FF21A068FDF7B1FB834FA068FDF780
:1061F00065FB07950895804A3BB2934202D07F4ADF
:10620000934205DAA068FDF7ADFB6427002606E09F
:10621000002F01D00F2E02D1A068FDF74FFB032203
:10622000089B606801331A400892FFF736FC051C92
:106230006068FFF739FC0022714B06929D4210DB2B
:10624000013206922A1CC8320BDB04220692AA22D3
:106250009200954205DC03220692C82D01DC013A2A
:10626000069200220492984210DB01230493031C3F
:10627000C8330BDB04230493AA239B00984205DC5C
:1062800003230493C82801DC013B04930EA8FEF706
:1062900057F9002511ABEB5C012B08D1594A6B0073
:1062A000D15CD3185A780EA8FF23FEF753F90135B5
:1062B000192DEFD16B461821595E6B460EA810229E
:1062C0009A5E089BFEF746F93BB2002B01DB0F2ECE
:1062D00007D90023A068009374300EA91A1CFEF79A
:1062E00001FA00230593059B464A5B00995C0698DA
:1062F000814224D1D3185B78049A93421FD12C2178
:1063000006AB059A5B189B5C012B18D00C25079BEC
:106310000AA85D4321680022FFF710FD1FAB5D193D
:106320000AAB07CB07C52C20012306AA0599121832
:106330005354079B0133DBB20793731CDEB2059BFA
:1063400001330593192BCED16420FEF7A6FF3B1C29
:10635000643B9FB2079B182B00D84CE718A81FA9D5
:106360001A1CFFF701FF6A461BAB23CB23C21B6835
:1063700013601899199A1A9B2068FFF7C7FCE56803
:10638000002D0CD0204910A8FEF71AF8281C10A9DF
:1063900018AA1C2300F006FF10A8FDF7F5FFA0685F
:1063A000FDF7E0FA0FA910A8A568FEF7C1F80023D1
:1063B000164A009310A90192281C1A1CFDF79AFA9C
:1063C00010A8FEF7A2F8FA204000FEF766FFA068CA
:1063D000FDF7C8FA0999A068FDF7B8FA0FA8FEF70B
:1063E00094F80EA8FEF791F86BB0F0BC08BC02B0B0
:1063F0001847C046FEC202008C3C0000D18AFFFF55
:1064000058FDFFFFCCC2020043C30200DC050000C0
:10641000F0B587B001930EAB1B88061C03930D9B50
:106420000D1C0093019B02920C9F002B3DD0002F6E
:1064300002D1009BDB0738D5282002F03AF8041C73
:106440001030FEF71FF86B461B89258063801820EB
:1064500002F02FF80497071C051C009B00210593F0
:10646000019B102208C7381C1EF0ADF804A90822B1
:10647000381C1EF08BF80E4B02226B610023A560C6
:106480000399E3602362636233680A43A2805B6816
:10649000301C211C9847002808D0201CFCF717FD51
:1064A000201C02F002F8034800E0034807B0F0BDEA
:1064B0007F5D000016FCFFFF17FCFFFF70B58CB07E
:1064C0008360109B01604260C360041C1849181C63
:1064D00000F062FD051E14D0011C1C22103105A81D
:1064E0001EF054F86A4608AB43CB43C21B681360E6
:1064F00020680599069A079BFFF708FC281C01F005
:10650000D4FF0C4B186800280ED00B4A05AB05923F
:10651000002206926A4622CB22C2C02305210293A2
:106520000322231CFFF774FF201C0CB070BDC04673
:1065300043C30200580A00209161000010B5041CFA
:1065400000F004FF0023201C237510BD13B5041CAC
:1065500004A800780090201C00F036FF002801D12C
:10656000207500E0004816BD0EFCFFFF13B5041CAB
:1065700004A800780090201C00F00EFF002801D134
:10658000207500E0004816BD0EFCFFFF1FB503ACF0
:106590006370002322700093221C0233FFF7E6FF92
:1065A00004B010BD7FB50D1C111C0F226A44061CDF
:1065B0001C1E117015D0089B002B12DD0123291C15
:1065C0000093FFF7D3FF002801D007480AE00090AE
:1065D000291C301C221C089BFFF7B8FF002801D0A3
:1065E000F3E7024804B070BD0EFCFFFF17FCFFFF8D
:1065F0001FB50F2401236C440093231CFFF7D2FF27
:10660000002800D1207804B010BD70B5041C161C01
:106610001D1C03220F2300F04BFA201C311C022208
:106620000F23103000F044FA201C291C01220F23F4
:10663000203000F03DFA201C049904220F23303052
:1066400000F036FA201C059905220F23403000F097
:106650002FFA201C069911220B23503000F028FA43
:10666000201C07990C220B23603000F021FA0B222A
:10667000201C0899131C703000F01AFA201C09998C
:1066800012220B23803000F013FA201C0A990A22F0
:106690000B23903000F00CFA201C0B9906220F23DC
:1066A000A03000F005FA201C0C991A220B23B03000
:1066B00000F0FEF9201C0D9914220B23C03000F0CD
:1066C000F7F9201C0E9917220B23D03000F0F0F9B7
:1066D000201C0F9916220B23E03000F0E9F9201C52
:1066E000109915220B23F03000F0E2F9601C11998B
:1066F00010220B23FF3000F0DBF9201C113012991F
:1067000000220B23FF3000F0D3F9201C2130139915
:106710001E220B23FF3000F0CBF9201C31301499DE
:106720001C220B23FF3000F0C3F9201C41301599C7
:106730001D220B23FF3000F0BBF9201C51301699AD
:106740001B220B23FF3000F0B3F9201C70BD82B078
:1067500030B585B00892051C082202A809931DF0E7
:1067600015FF039B029C5810DB0701D52B581C59C1
:106770002D180AA9684608221DF008FF089A099BEF
:10678000281CA04705B030BC08BC02B018470289DD
:10679000031C8A4202D18079012305E0428900204E
:1067A0008A4202D198790223184070470289031C5B
:1067B0008A4202D18079042305E0428900208A427E
:1067C00002D198790823184070470289031C8A4235
:1067D00002D18079102305E0428900208A4202D14B
:1067E0009879202318407047038910B58B4207D150
:1067F00083790124002A01D0234300E0A34383715D
:1068000043898B4207D183790221002A01D00B43AF
:1068100000E08B43837110BD038910B58B4207D113
:1068200083790424002A01D0234300E0A343837129
:1068300043898B4207D183790821002A01D00B4379
:1068400000E08B43837110BD038910B58B4207D1E3
:1068500083791024002A01D0234300E0A3438371ED
:1068600043898B4207D183792021002A01D00B4331
:1068700000E08B43837110BD82B0F0B589B00E92F9
:106880000F93078995B2041CBD4200D147890EAB16
:106890005E88022E25D0052E11D0012E73D1201C2A
:1068A000291C321CFFF7A0FF201C391CFFF76FFFCB
:1068B000002868D0A18804A8321C331C0EE0201CDC
:1068C000291C0122FFF7A8FF201C391CFFF76EFFCF
:1068D000002858D0321C0123A18804A8FDF7F2FD3E
:1068E00051E0201C391CFFF752FF002816D0321C43
:1068F000A18801236846FDF7E5FD201C291CFFF750
:1069000055FFA68800282ED0201C391CFFF74EFF0B
:10691000002828D004A8311C042227E0201C291CB0
:10692000FFF753FF00280ED1267B012E0BD1201C30
:10693000291CFFF73BFF002821D0291C042204A8B2
:10694000331CFDF7BFFD201C291C0022FFF74CFF64
:10695000201C291C0022FFF75FFF201C291C00229D
:10696000FFF772FF0FE0311C032204A80123FDF79B
:10697000A9FD201C391C0122FFF766FFE3E704A8EC
:10698000291C0322DCE709B0F0BC08BC02B01847A0
:1069900001737047F0B587B001930EAB1B88061CDE
:1069A00003930D9B0D1C0093019B02920C9F002BE7
:1069B0003DD0002F02D1009BDB0738D5282001F005
:1069C00078FD041C1030FDF75DFD6B461B892580AA
:1069D0006380182001F06DFD0497071C051C009BC7
:1069E00000210593019B102208C7381C1DF0EBFD08
:1069F00004A90822381C1DF0C9FD0E4B02226B6150
:106A00000023A5600399E3602362636233680A434D
:106A1000A2805B68301C211C9847002808D0201CED
:106A2000FCF755FA201C01F040FD034800E0034844
:106A300007B0F0BD4F67000016FCFFFF17FCFFFF1B
:106A4000F0B5041C161C00258380164A164B857170
:106A50000260218146810573186889B08C46A8427E
:106A60001DD0124A059504926A4604AB82CB82C2BD
:106A7000C023614602932A1C231CFFF78BFF0B4A9D
:106A8000094B06926A461868079506AB82CB82C20C
:106A9000C023311C02932A1C231CFFF77BFF201C00
:106AA00009B0F0BD58C30200580A00207968000000
:106AB00030B5002403730123034D84710560818088
:106AC00082734373846030BD58C2020038B5837945
:106AD000041CDB0702D5806801F0E7FCA3799B0763
:106AE00002D5A06801F0E1FCA3795B0707D5A023DC
:106AF0000021144ADB00D150A06801F0D6FCA37934
:106B00001B0708D5A568002D05D0281C00F02AFF1A
:106B1000281C01F0CAFCA379DB0605D5A068002873
:106B200002D00368DB6898476023A2791A4205D037
:106B3000A068002802D003685B6898470023A36020
:106B4000A37138BD00700040F7B50227037B3B42BC
:106B500030D0012930D800918579041C3D4015D1F1
:106B6000FFF7B4FF182001F0A4FCA37B291C182216
:106B7000061C01931DF027FD6B460421301C59565D
:106B8000FBF7AFF9A379A6603B43A3710023A46888
:106B9000E356013304D1094809492422FBF748F997
:106BA000009A6368002A03D0E2681360002004E0C2
:106BB0002269FAE7034800E00348FEBDC0BB0200BB
:106BC000D8BB020016FCFFFF17FCFFFFF7B501273B
:106BD000037B3B4236D061238579041C1D4018D1CC
:106BE000FFF774FF182001F064FCA37B291C0093BD
:106BF000637B1822061C01931DF0E5FC6B46002107
:106C0000301C5956019AFBF753F9A379A6603B4310
:106C1000A3716023A2791A4203D0A068FBF7E2F8BF
:106C200011E00023A468E356013304D10648074964
:106C30002C22FBF7FDF8636960681B681840431E4F
:106C4000984100E00248FEBDC0BB0200D8BB020074
:106C500016FCFFFF10B50124837941731C4004D05A
:106C60008068FBF7A1FA002007E06022134203D0FE
:106C70008068FBF7BCF8F6E7004810BD16FCFFFF84
:106C8000704710B5041C01F010FC201C10BD000062
:106C900070B5041C00250D4B0E1C083385808571D2
:106CA0000360211C183000F0C8F8201C211C203083
:106CB00000F0E6F8064BA680A571E5712572E56047
:106CC00025616561201C1C6070BDC04668C3020060
:106CD0009C0A00208379DB0702D5C160002000E018
:106CE0000048704716FCFFFF8379DB0701D5C068B9
:106CF00000E001487047C04616FCFFFF38B5456903
:106D0000002D22D0037A032B21D8041CFFF7ECFFBF
:106D1000A8622C2001F0CDFB2C220021051C1DF0C7
:106D200052FC0023626953622369002B01D1226166
:106D300005E0596A002901D00B1CFAE75A62237A50
:106D4000656101332372002002E0024800E002483E
:106D500038BDC04617FCFFFF13FCFFFF154B70B595
:106D60005A68154D002A03D000225A600132AA60E9
:106D70001B69114E002B1CD000210E4B0F4C1961CA
:106D80008023DB00F358012B0ED1A923DB00F1583F
:106D900020684942FFF79EFF2068FFF7AFFF236896
:106DA0005A69074BF25002E02068FFF793FF012376
:106DB000AB6070BDFC100040001000409C0A002039
:106DC00004050000031C0069002809D00221054ABF
:106DD000D167426A1A611A7A013A1A72024B196033
:106DE0007047C04604E100E000E100E030B5041C5B
:106DF00085B02569002D1ED0EA78012A06D0022A26
:106E000009D1201C203000F03FF80AE0201C183087
:106E100000F017F805E092B268461E210123FDF745
:106E200051FB23699D42E4D1201CFFF7CBFF281CB6
:106E300001F03BFBDDE705B030BD0023016043609E
:106E400070471FB5041C0068FFF7BCFF0023626891
:106E500043629A4201D160600BE0516A002902D07E
:106E600001330A1CF9E7032B02DD01F01EFB06E0EB
:106E70005062012268461D21131CFDF723FB1FBD34
:106E8000002341600370704738B5041C4068FFF769
:106E900099FF0123051C23700430FDF7FFFA00233E
:106EA000281C237001F001FB38BD13B50C1C01A890
:106EB00001F052FA01A8211C01F058FA13BD73B574
:106EC0000D1C161C1C1C01A801F046FA311C2A1CC2
:106ED00001A8231C01F082FA73BD07B5019280223C
:106EE00000915205136952696946133A5A430223C5
:106EF000FFF7E5FF07BD84B010B50492802203912F
:106F000005935205146953695169113B0A1C133AE0
:106F100062435C430F9B03A91B1BD2180C23FFF792
:106F2000CEFF10BC08BC04B018470000F7B580279E
:106F30007F053D697C690822113C6C43061C211CBD
:106F400068461DF023FB104B009A9A4219D000931B
:106F5000002301937969301C13396943FFF7A5FFBA
:106F6000019A301C0099FFF7B8FF301C211CFFF775
:106F70009CFF7969AB0813396943301C221CFFF769
:106F80009EFF0198FEBDC046FECA000010B5041C5D
:106F9000FFF7CCFF201C10BD80235B05F7B51A69F5
:106FA0005B690191113B1D1C5543FFF7BFFF071E95
:106FB00020D0302001F07DFA00213022041C002670
:106FC0001DF001FB0835BE420ADA291C201C3022C4
:106FD0001DF0DCFA0198211C1EF050F9002806D1A2
:106FE000201CBE4206D101F060FA002002E03035DC
:106FF0000136E8E7FEBD0000F0B50D1CABB00D9208
:1070000000213022061C12A80B931DF0DCFA281C6C
:107010001EF0D0FD431C0C93102B00DDB6E00B9B43
:10702000202B00D9B2E0301C291CFFF7B5FF071E4A
:1070300029D1291C0C9A12A81DF0A8FA0D990B9AB7
:1070400016A81DF0A3FA80235B051F695A69301C3E
:10705000113A7A435D690D92FFF768FF0D9B00219D
:1070600008333022041C1EA80F931DF0ACFA291C13
:1070700013397943301CFFF718FF0F9B0B93002344
:107080000C930E9335E010300D990B9A1DF06FFAAA
:10709000041C381C01F009FA002C7AD0C9E70B99BE
:1070A0001EA830221DF072FA1EA812A91EF0E6F8E2
:1070B000002822D13849301C221C10911194FFF76E
:1070C0000CFF6A460B9B099315AB23CB23C223CB42
:1070D00023C223CB23C2301C149B1299139AFFF7AF
:1070E0000AFF01230E930B9B30330B930C9B013350
:1070F0000C930C9BA342D2DB10E06A460B9B0993D6
:1071000021AB23CB23C223CB23C223CB23C2301CEE
:107110001E991F9A209BFFF7EEFEE4E7E54330211E
:10712000ED1725404D430F9B5D190E9B002B1BD186
:10713000B81E19F0DBF984422AD017490134301CFB
:10714000221C10911194FFF7C8FE6A46099515ABF1
:1071500023CB23C223CB23C223CB23C2301C1299BF
:10716000139A149BFFF7C7FE301C0D99FFF79DFE85
:1071700080235B0559690C23634313397943023338
:10718000301C0D9AFFF79BFE002402E0034C00E048
:10719000034C201C2BB0F0BDFECA000017FCFFFF03
:1071A00013FCFFFF08B509680431FFF725FF08BD90
:1071B000704710B5041C01F078F9201C10BD0000C8
:1071C00038B58280FA2200230D4D92000835056003
:1071D00041618371C26083604382041C081C0949B9
:1071E000FFF7DAFE051E09D0011C201C10311230F9
:1071F00002221DF0CBF9281C01F057F9201C38BDE4
:1072000088C3020080C3020010B5041CFBF732FFE4
:107210000023A46801228B4203D1A0425B415B4260
:107220001A40101C10BD000030B50225837985B0CE
:10723000041C2B4204D1FBF7ABFBA3792B43A371B6
:10724000201CFFF7E1FF00281DD001220F4B1A6020
:107250000F4B5A68002AFBD0002201255A600D4BC3
:107260000A4A1B685560DA17920FD3189B102382C5
:10727000FBF700FFE368A1881818A0602A1C684685
:107280002B1CFDF71FF9002005B030BD00C00040E9
:10729000FCC0004008C5004008B5FFF7C5FF08BDA9
:1072A000017042704360704782B0F0B50592021CD5
:1072B000069308AB1B7805ACE0CCE0C2002B2ED0C7
:1072C0004A78002A05D0069A52424260079A5242F2
:1072D00082604A68022A08D0032A0DD0012A10D100
:1072E000026841685242016004E002685242026052
:1072F00042685242426004E04268016852420260C1
:107300004160012B04D0022B09D143685B4202E0AB
:10731000426803680260436083685B428360F0BC3C
:1073200008BC02B0184782B037B5041C181C07937C
:107330000B7806920193089B0093031C201CFFF717
:10734000B3FF201C3EBC08BC02B0184770B5041C3B
:107350000E1C151C002110221DF035F9054B201CB8
:107360002361311C2A1C00F0C1F8034B201C1C6057
:1073700070BDC046A0860100A00A002038B5054DAA
:107380002B68834204D0041C216900F069F82C604A
:1073900038BDC046A00A0020F0B585B01C1C0AAB61
:1073A000061C0F1C03921D78FFF7E8FF01235D40C8
:1073B0000095231C301C391C039A00F093F9201A05
:1073C000441EA04105B0F0BDF0B585B01C1C0AAB51
:1073D000061C0F1C03921D78FFF7D0FF01235D40B0
:1073E0000095231C301C391C039A00F029F9201A3F
:1073F000441EA04105B0F0BD084B0068C150084BC9
:10740000021CFC32116A002904D1013B002BF7D188
:10741000012001E0002010627047C0461C050000FA
:10742000D107000010B50368002A03D08022022093
:107430009200985001221A62084A1C1CFC34E06831
:10744000002804D1013A002AF7D1012005E00020EC
:10745000A322E060D2009B580B7010BDA1860100F2
:1074600010B50B4C02680B4BA14204DC0A49816049
:10747000CC2149040AE0094CA14203DC084981609F
:10748000802102E007498160CD21C904D15010BD9F
:107490008FD0030024050000A08601007F1A06009B
:1074A00090D00300801A060070B5041C101CA025A3
:1074B000C026C130FF30F600ED0580004651081CA3
:1074C000C130FF3080004651A1252068ED004251B7
:1074D000054A8150191C201CFFF7C2FFA02305217B
:1074E0002268DB00D15070BD0C050000F8B50E1C01
:1074F000151C041C00F0FCF92648F2B20378011CAC
:10750000DBB2012B06D14778974203D18778E8B2E6
:10751000874211D02048EFB20378012B05D1437880
:10752000934202D18078B84211D00878002806D161
:1075300001230B704A708F706373184B15E0164B64
:107540001978002907D1013119705A709F700223F0
:107550006373134B09E01348FAF776FC0023FC220F
:107560002360657126719362FFDE191C0022FC31D5
:107570002360657126718A62A021C9005A500A49A8
:10758000201C5A5001325A50311C2A1C074BFFF75D
:107590008BFFF8BDA40A0020A80A0020003000409C
:1075A00000400040A0C30200FC0F0000A0860100C4
:1075B000026808B5031C101C0021FC308162A02069
:1075C000C00011500648115001311150042105220C
:1075D00059569A56181C9B68FFF766FF08BDC046AF
:1075E000FC0F0000036800211A1CFC3210B59160EA
:1075F00001315961074B9168002904D1013B002BEF
:10760000F9D1012004E000240473FFF7D1FF201C0E
:1076100010BDC046A1860100036810B5191CFC31DD
:107620008A6A0020012A08D1044C1C5988625A61D8
:107630000238A40701D40120404210BDC404000058
:10764000F7B50192B1221F1C03684910D20099506E
:107650008021012289005A50191C0025041CFC318C
:10766000CD601A607E1E019BB54213DA5919201CA9
:107670000022FFF7D7FE00280AD0201CFFF7CCFF1E
:10768000071C201CFFF794FF2E1C002F26DA1CE09D
:107690000135E7E79919201C0122FFF7C3FE0028F6
:1076A00003D0201CFFF784FF18E0089B3E1C002B32
:1076B00014D0FAF76FFF051C2368FC339B68002B7E
:1076C00005D000222368FC339A603E1C06E0FAF7DE
:1076D00061FF034B401B9842EEDDF2E7301CFEBD1C
:1076E0003F420F00F8B5171CB1221D1C0368D200E1
:1076F000491099508022002492009C500122061CBF
:107700009A60AC4211DA395D301CFFF775FE002833
:1077100009D0301CFFF74CFF301CFFF77DFF00281D
:107720000EDA041C0CE00134EBE7069B2C1C002B4A
:1077300006D0301CFFF756FF002801D00124644218
:10774000201CF8BD0023104A30B5D356834205D023
:107750000123D3560121834215D100E000210B1CE7
:1077600045330A4C0A48FF339B001C5001231D1C63
:107770004C00601C8540A340A120064C2B43C00058
:107780002350FF23535430BD2F000020031F02005D
:107790000060004000F00140A820012210B510490F
:1077A000104B0C88C0005A601C5048880E49585035
:1077B0008021082089005850802009310003FF31C2
:1077C00058500A490878A221C90058500849088829
:1077D000084958501A600022FC331A6510BDC04693
:1077E0003200002000A00040440500002E000020D0
:1077F0002C0000204C05000008B5407840B2FFF78F
:10780000A1FF08BDA0230021364ADB00F0B5D45803
:10781000D150A023E0213448DB05C9005E58585000
:1078200078315D58585080210638FF38C905195005
:107830000121195004200138C046C046C046C04648
:10784000C046C046C046C046C046C046C046C04608
:10785000F1D1A227FF00D859800F084205D0D8598E
:107860001323084202D0012030E01323013B002BF8
:107870002BD0A02101271D48C9050F500420013835
:10788000C046C046C046C046C046C046C046C046C8
:10789000C046C046C046C046F1D1A120C0000F502E
:1078A00004200138C046C046C046C046C046C04657
:1078B000C046C046C046C046C046C046F1D1A22020
:1078C000C00009584900D1D5CDE7181CA023E021FC
:1078D000DB05C9005E5078315D50A023DB00D45039
:1078E000F0BDC046004000400D0600000C05000041
:1078F000A023E021134ADB05C90010B55A507831A6
:107900005A50114B0022191CFC31CA600A62A12195
:107910001E20C9005A500D4A0D4C9850CC200D4ADB
:1079200040049850A2200C4AC00014500B4C0C4844
:10793000145001205050A0220521D2009950FFF789
:1079400061FF10BD0C060000004000400C05000067
:10795000384100402405000000F001401C40004078
:107960001405000010B5041CFFF746FF201C10BDD5
:1079700008B503685B6A984708BD000008B4024B6D
:107980009C46443808BC604771790000F8B5FA237A
:107990000189DB00041C5943324800F076FDFA21CE
:1079A000890018F0A3FD304F2081A17A381C00F027
:1079B0006CFD231C251C261C22894C33A0728C359F
:1079C0001A80A036317828682A220023FEF7DEFDCF
:1079D000002801D0254844E0317828685B221F2325
:1079E000FEF7D4FD0028F5D1317828685C222023E9
:1079F000FEF7CCFD0028EDD1317828682C22012338
:107A0000FEF7C4FD0028E5D1317828682D22012336
:107A1000FEF7BCFD0028DDD1317828682E22012335
:107A2000FEF7B4FD0028D5D1A17A381C00F028FD5E
:107A30003178C3B20E222868FEF7A8FD0028C9D10C
:107A4000FA2321899B005943064800F019FD0123C0
:107A50001843C3B2317828682A22FEF797FD002820
:107A6000B8D1F8BD78C40200F4C302000EFCFFFFD9
:107A700008B4024B9C46443808BC60478D7900002E
:107A8000074B10B51A1C041C08323C3302604364D7
:107A90004430FEF729F8201CFDF7BCFD201C10BD6A
:107AA00018C4020008B4024B9C46443808BC604726
:107AB000817A000010B5041CFFF7E2FF201C00F0E3
:107AC000F4FC201C10BD000008B4024B9C46443856
:107AD00008BC6047B57A0000F0B50425837989B009
:107AE000041C2B4204D1FAF753FFA3792B43A37153
:107AF000201C9030FFF76AF8061E62D1231CA033C9
:107B000019780C230093231C05AD8C3318680122CF
:107B10002B1CFEF747FD002801D02C4E52E00A2313
:107B200002AA9B182A785A706A781A700022995E05
:107B30000291AA785A70EA781A70287900215A5E60
:107B40005870687952421870A87900215F5E5870A9
:107B5000E87918700021585E0390287A5870687A86
:107B600018700021585EA97A5970ED7A1D700025B1
:107B70005D5FA37A5A43D117C90E8C4662445211F5
:107B8000A261029959437B43DF17FF0EFB185B117B
:107B900023626423CA17D20E51185B42039A5843DA
:107BA000C8335A435D43E2674911221DA067E16172
:107BB000201CD567FDF743FF201C4430FDF79BFFD9
:107BC00000E00026301C09B0F0BDC0460EFCFFFFEF
:107BD00008B4024B9C46443808BC6047D97A000080
:107BE000F7B51E1C041C08AB1B88151C019309ABC0
:107BF00000911A88311C0AAB1F88FDF713FD201C69
:107C0000311C3A1C4430FDF7B3FF134B201C1A1CE7
:107C10003C336364231C08322260009A8C331A6060
:107C2000AB8890308380AB796A4683710B4B928826
:107C30000360AB68032183602B7B03736B7B43730F
:107C4000AB7B8373231CA0331A80FFF703F8201C3F
:107C5000FFF79CFE201CFEBD18C4020058C20200A3
:107C600008B5C9B20D22FEF7C3FCC73843425841DC
:107C700008BD08B503685B6A984708BDF7B5FA25E3
:107C8000204F0189AD00041C6943381C00F0FDFB46
:107C9000291C18F02BFCA17A20811B4800F0F5FB71
:107CA000261C636CA072009321895836337869438F
:107CB000381C019300F0E4FB07231843C3B2019979
:107CC00000982022FEF762FC002801D00F4818E03F
:107CD0003178606C22221023FEF758FC0028F5D181
:107CE000A17A0948656C377800F0CAFB80235B42B3
:107CF0001843C3B2391C281C2322FEF747FC002876
:107D0000E4D1FEBD24C50200FCC402000EFCFFFF4E
:107D100010B5041C034B08330360FDF77BFC201CEB
:107D200010BDC04680C4020010B5041CFFF7F0FF70
:107D3000201C00F0BAFB201C10BD00007FB50425FC
:107D40008379041C2B4204D1FAF722FEA3792B433A
:107D5000A371201C4830FEF739FF002837D0231CC0
:107D600058331978062302AE0093606CA822331CA6
:107D7000FEF718FC051E01D0164828E00023F25E2D
:107D8000D317DB0E9A18521193B20222B15E3380E0
:107D9000CA17D20E511849118AB20421705E1BB263
:107DA000C117C90E0818401181B2A07A5B42434343
:107DB000728012B2B180524209B242434843E36139
:107DC00023682062A2619B6A201C9847281C04B08B
:107DD00070BDC0460EFCFFFFF8B5041C151C06AABA
:107DE000168807AA0F1C1288191CFDF71BFC0F4BE5
:107DF000676408332360231CAA8848339A80AA79D1
:107E0000201C9A710A4AA264AA6822652A7B1A7306
:107E10006A7B5A73AA7B9A730023A371231C58337D
:107E20001E80FFF72BFF201CF8BDC04680C4020057
:107E300058C2020008B5C9B20F22FEF7D9FB333889
:107E40004342584108BD08B50368DB69984708BD3F
:107E5000F7B5FA25041C144E0189AD006943301CA6
:107E600000F013FB291C18F041FB271CA36C208198
:107E700000935C373B7881B26943301C019300F07A
:107E8000FFFA0199C3B260220098FEF77FFB002839
:107E900001D0064807E03978A06C62220123FEF782
:107EA00075FB0028F5D1FEBD7CC502000EFCFFFF6E
:107EB00010B5041C034B08330360FDF715FE201CAE
:107EC00010BDC04630C5020010B5041CFFF7F0FF1E
:107ED000201C00F0EAFA201C10BD00007FB5082528
:107EE0008379041C2B4204D1FAF752FDA3792B436A
:107EF000A371201C4C30FEF769FE002822D0231C01
:107F00005C331978062302AE0093A06CE822331C80
:107F1000FEF748FB051E01D00B4813E00223F25E7A
:107F200096235B425A4362630021725E201C5343D6
:107F3000A3630423F25E96235343E36323681B6A1F
:107F40009847281C04B070BD0EFCFFFFF8B5041C58
:107F5000151C06AA168807AA0F1C1288191CFDF703
:107F600007FE0D4BA76408332360231CAA884C33FB
:107F70009A80AA79201C9A71084AE264AA6862650C
:107F80002A7B1A736A7B5A73AA7B1E829A73FFF745
:107F90005FFF201CF8BDC04630C5020058C2020079
:107FA00008B5C9B24F22FEF723FB4038434258417F
:107FB00008BD08B50368DB69984708BD10B5041C07
:107FC000034B08330360FDF78FFD201C10BDC04636
:107FD00088C5020010B5041CFFF7F0FF201C00F05C
:107FE00064FA201C10BD0000F0B5061C5C3687B09A
:107FF000041C3178806C10220023FEF7C7FA204F52
:10800000002807D01E4839E02B789B0710D0642049
:10801000FAF758FD0F2502ABED1801233178A06C5B
:10802000009308222B1CFEF7BDFAB842ECD1E9E719
:10803000FA25144F2189AD006943381C00F025FA58
:10804000291C18F053FA20813178A06C1122A0234A
:10805000FEF79CFA0028D5D1A36C218903936943CC
:10806000381C367800F00CFA01231843C3B2311CD7
:1080700003981022FEF78AFA0028C3D107B0F0BD9A
:108080000EFCFFFF0CC6020070B50825837986B090
:10809000041C2B4204D1FAF77BFCA3792B43A37178
:1080A000201C4C30FEF792FD002830D0231C5C339E
:1080B0001978062304AE0093A06C0122331CFEF74E
:1080C00071FA051E01D0134821E00E2332786B446B
:1080D0005A707278201C1A700022995E64224A43FA
:1080E000A263B2785A70F2781A700022995E642204
:1080F000524251436163317959707179197000218D
:108100005B5E5A432368E2631B6A9847281C06B0EB
:1081100070BDC0460EFCFFFFF8B5041C151C06AA76
:10812000168807AA0F1C1288191CFDF721FD0D4B9C
:10813000A76408332360231CAA884C339A80AA7949
:10814000201C9A71084AE264AA6862652A7B1A7345
:108150006A7B5A73AA7B1E829A73FFF745FF201C25
:10816000F8BDC04688C5020058C2020008B5C9B2B1
:108170000722FEF73DFAC4384342584108BD08B50E
:1081800003685B6A984708BDF8B5FA260189B6000E
:10819000041C7143264800F078F9311C18F0A6F948
:1081A000244F2081A17A381C00F06FF9251CA072A1
:1081B00058352978606C2A220023FEF7E7F9002859
:1081C00001D01D4832E02978606C2B221023FEF785
:1081D000DDF90028F5D12978606C2D220123FEF706
:1081E000D5F90028EDD12978606C2E220123FEF705
:1081F000CDF90028E5D1A17A381C00F041F92978A1
:10820000C3B20E22606CFEF7C1F90028D9D12189D2
:108210000748714300F034F901231843C3B22978A9
:10822000606C2A22FEF7B2F90028CAD1F8BDC04618
:10823000ACC6020054C602000EFCFFFF10B5041CC1
:10824000034B08330360FDF7E5F9201C10BDC04661
:1082500078C6020010B5041CFFF7F0FF201C00F0E8
:1082600024F9201C10BD00007FB504258379041C6F
:108270002B4204D1FAF78CFBA3792B43A371201C6A
:108280004830FEF7A3FC051E24D1231C583319786F
:10829000062302AE0093606C0122331CFEF782F9C4
:1082A000002801D00D4D16E0022300210420F356D2
:1082B000A27ADB00715630565B425343C000C900BE
:1082C00051434243A3612368E16122629B6A201CFF
:1082D000984700E00025281C04B070BD0EFCFFFF8D
:1082E000F8B5041C151C06AA168807AA0F1C1288CC
:1082F000191CFDF797F90F4B676408332360231CA3
:10830000AA8848339A80AA79201C9A710A4AA264E2
:10831000AA6822652A7B1A736A7B5A73AA7B9A73AE
:108320000023A371231C58331E80FFF72DFF201C50
:10833000F8BDC04678C6020058C2020008B5C9B2EE
:108340000D22FEF755F95A384342584108BD29DF3E
:10835000704728DF70470000034B1A78002A01D1CC
:1083600001321A707047C046AD0A002038B50C1CA7
:10837000FDF70CF8002811D0154B00221D1C1A70B7
:10838000A40A201CFFF7E5FF002803D00A20FCF711
:1083900084FFF6E72B78002BFCD018E002210D4A71
:1083A0000D4B9950111C8022D20098580028FAD009
:1083B000A120094DC0002C5098580028FCD0002066
:1083C000054A50508022D2009A58002AFAD038BD6F
:1083D000AC0A00200405000000E00140F8B50D1CC7
:1083E000161C1C1CFCF7D2FF002812D0184B0022D0
:1083F0001F1C1A70281C311C221CFFF7A8FF002824
:1084000003D00A20FCF749FFF4E73B78002BFCD0AF
:108410001CE0104A012194460F4B99508022D20053
:108420009A58002AFAD000228027FF00A24207DAD9
:10843000910070586850D9590029FCD00132F3E7F7
:10844000002261465A50DA59002AFCD0F8BDC046D5
:10845000AC0A00200405000000E001400CC80748F9
:1084600010B51B18DB00D318181C934205D31C68E9
:108470008C4202D3181C083BF7E710BDFFFFFF1F1B
:1084800008B5FFF7EBFF406808BD08B5FFF7E6FF4A
:10849000006808BD08B500F008F808BD08B5031C61
:1084A000081C191C1BF07CFA08BD08B5FAF7A6FCDD
:1084B00008BD10B5041E02D1013400E08047201C25
:1084C000FAF768FC002805D100F06CFE0028F5D111
:1084D0001BF012FA10BD08B5FFF7EBFF08BD000056
:1084E00008B503491B2202201EF036FB00F0E6FE11
:1084F000B4C60200F7B5344D01902B685A1C2A60AF
:10850000002B5ED10122314C314B324F1A7023685F
:10851000381C996800F0EEF923682F48596800F07C
:10852000E9F923682D4ED968301C00F0E3F9391CB5
:108530002B480CF08DFF28492A4801F00DF92A4FED
:10854000311C381C0CF084FF311C28480CF080FFD3
:10855000244B234A9A6780233A699B0113433B616A
:108560001F4B7B67224F2368381C996800F0D2F9B3
:1085700023682048596800F0CDF923681E4ED96859
:10858000301C00F0C7F9391C1C480CF0E3FF1C4CF0
:108590001849201C01F054F91A4F311C381C0CF0FA
:1085A000D9FF1948311C0CF0D5FF144B3A69A36769
:1085B00080239B0113433B61104B7B672B68013386
:1085C0002B600198FEBDC046C40A00202001002097
:1085D00036000020A41E0020381D0020F41B0020BF
:1085E0001C1C0020A81C00208C190020F01D00205D
:1085F000CC1B0020641900207C1E0020181A0020CB
:10860000A81A0020601D00203C1B00200D4A10B558
:108610001368041C591E1160022B11D10A480CF07A
:1086200074FF0A480CF071FF09480CF06EFF09480E
:108630000CF0EDFF08480CF0EAFF08480CF0E7FFEB
:10864000201C10BDC40A00201C1C00208C19002016
:10865000F01D0020181A0020601D00203C1B002087
:1086600082B037B506920022041C00920A9A079342
:108670000B6801921D69069A079BA847201C3EBC07
:1086800008BC02B0184782B037B506920022041C1D
:1086900000920A9A07930B6801921D69069A079B3C
:1086A000A847201C3EBC08BC02B0184710B5041CEB
:1086B000024B03600DF026F8201C10BD38C70200E5
:1086C00010B5041C024B03600DF010F8201C10BD07
:1086D000F8C6020010B5041CFFF7E8FF201CFFF7E6
:1086E000E4FE201C10BD10B5041CFFF7E9FF201CA0
:1086F000FFF7DBFE201C10BD10B5041C006A1BF048
:1087000055FD606210BD10B5041C006A1BF04EFDE3
:10871000216A1EF09BFC10BD38B50125041C6D427A
:10872000081C4B1C04D1636A281C5A1C03D0181C5B
:10873000216A1EF08BFC656238BD08B5006A1BF02B
:10874000F9F908BD08B5006A1BF0F4F908BDF8B5E1
:10875000041C002301267642F71706980D1C26609C
:108760006760111CA360E3601A1C984204D0431E8A
:108770005A4253410220C21A286A1BF069FB0028A2
:1087800005D1286A1BF00AFC2060C0176060201C1D
:10879000F8BDF8B5041C002301267642F7170698A9
:1087A0000D1C26606760111CA360E3601A1C9842D0
:1087B00004D0431E5A4253410220C21A286A1BF0B9
:1087C00047FB002805D1286A1BF0E8FB2060C01792
:1087D0006060201CF8BD10B5041C006A1BF018FD79
:1087E000606210BDF8B5061C0F1C141C0025A542C4
:1087F00005D0306A1BF00CFD431C07D12C1C002C4B
:1088000008D0074BE3189B00DB5905E0AB00F8509C
:108810000135ECE701235B427362201CF8BDC046C2
:10882000FFFFFF3F10B5041C006A1BF0F1FC216A3A
:108830001EF040FC10BD38B50125041C6D42081C1B
:108840004B1C04D1636A281C5A1C03D0181C216AD3
:108850001EF030FC656238BDF8B5061C0F1C151CF7
:108860000024AC420AD0A300F858316A1CF054FB33
:10887000431C01D1251C01E00134F2E7281CF8BD9E
:1088800008B5031C081C1B6A01211BF07FFC08BDF6
:1088900038B5051C0C1C081C2B6A01211BF0C8FAFA
:1088A000002803DD2418013C237801E001235B420A
:1088B0006B6238BD08B5031C4A1C06D1006A1BF068
:1088C00039F9431E9841404203E0081C196A1CF024
:1088D00017FB08BD08B5031C4A1C06D1006A1BF033
:1088E00029F9431E9841404203E0081C196A1CF014
:1088F00013FB08BD38B5041C0D1C0CF0F9FF044B2C
:108900002562236001235B42201C636238BDC046A0
:10891000F8C6020038B5041C0D1C0DF01DF8044B00
:108920002562236001235B42201C636238BDC04680
:1089300038C7020008B5031C1B68081C0C3B1B68E9
:10894000994204D9111C021C014800F06FFB08BDBC
:10895000F4C70200006808B50C380068091A04481A
:108960000918914202D2181C00F05DFB08BDC046F8
:10897000FEFFFF0F02680120914207D3131C0C3B3E
:1089800018688300D018884280414042704708B57B
:10899000012A02D10B68036001E01FF0FBFA08BD59
:1089A00008B5012A02D10B68036001E01FF0F7FA55
:1089B00008BD08B50B1E012B01D1026003E0111C9C
:1089C0001A1C1FF0F1FA08BD08B5521A9210FFF7F1
:1089D000DEFF08BDF8B5041C0E1C171C191C0B4A41
:1089E0001D1CFFF7A7FF21680B1C0C3B1C68641BB8
:1089F000BC4200D93C1C002C05D0AD004919301CEC
:108A0000221CFFF7C4FF201CF8BDC0466FC802003F
:108A1000044B984205D0002301608900411883600F
:108A2000CB607047B00A002038B5144D041EAC422C
:108A300002D9134800F0F7FA884203D94B00984254
:108A400000D21C1C631C9B00181C80221C330C30A1
:108A5000520193420BD98C4209D91B051B0DD31A25
:108A60009B081C19AC4200D9044CA0001030FFF741
:108A700020FD00234460836038BDC046FEFFFF0F29
:108A800098C80200F8B50B4D002810D00E1C00212C
:108A9000041CFFF7C9FF051C071C0C35281C211CF2
:108AA000321CFFF786FF381C211CFFF7B1FF281C82
:108AB000F8BDC046BC0A002010B5041C081C111CDF
:108AC0001A1CFFF7DFFF2060201C10BD08B5054B06
:108AD000984206D083685A1E8260002B01DCFFF7A3
:108AE000E4FC08BDB00A002013B5041C006801A90D
:108AF0000C38FFF7EBFF201C16BDF0B587B00093D4
:108B00000368171C1A1C0C1C0C3A00991568C91B29
:108B100049190191061C516801982D1BED1B8842D3
:108B200017D89268002A14DC002D0BD0009A9742C7
:108B300008D010193C198000A400181819192A1C13
:108B4000FFF72EFF306801990C38FFF761FF07B07F
:108B5000F0BD019805AAFFF767FF031C0C330290D4
:108B60000393002C04D003983168221CFFF70FFFF9
:108B7000002D0CD0009B391918198000029B0C3075
:108B8000181833688C0019192A1CFFF700FF306889
:108B900005A90C38FFF79AFF039B3360D2E700006A
:108BA00003680A4A0C3B10B593420DD09B68041C25
:108BB000002B04DD00210A1C0B1CFFF79EFF012285
:108BC000236852420C3B9A6010BDC046B00A002098
:108BD00008B503680C3B9B68002B01DBFFF7E0FF47
:108BE00008BD000070B5041C151C094A0E1CFFF7D7
:108BF000A1FE2368011C0C3B1A68921BAA4200D9F3
:108C00002A1C201C0023FFF778FF201C70BDC046E3
:108C1000B0C80200F8B51E1C051C0C1C171C111C4A
:108C20001A1C0A4BFFF796FE281C211C3A1C331C09
:108C3000FFF763FF002E06D02B68A4001819311C23
:108C4000069AFFF7B6FE281CF8BDC046C4C802004D
:108C500013B5046800920C3C0B1C22680021FFF73E
:108C6000D9FF16BD73B5151C064A1E1C041CFFF760
:108C700061FE0096011C2B1C201C0022FFF7CAFF7E
:108C800076BDC046E1C8020070B51E1C049B051CE1
:108C90000C1CFFF732FF049B002B06D02B68A400AE
:108CA0001819311C049AFFF772FE281C70BD0000D1
:108CB0000368F0B51F1C041C0E1C85B00C3F02930A
:108CC0003B68151C191C0393164BFFF743FE201C31
:108CD000311CFFF74FFE00281BD1BB68002B18DCAE
:108CE000029BF31A9B10AB4205D30298311C2A1C3D
:108CF000FFF74DFE06E0002B04D00298311C2A1C21
:108D0000FFF74EFE2068291C0C38FFF781FE201C5F
:108D100006E00095201C0021039A331CFFF7B4FFE6
:108D200005B0F0BD0CC90200034B984202D0836825
:108D3000013383600C307047B00A002070B50B1C03
:108D4000041C016850181A1C6168FFF76DFE051CB1
:108D50002268061C0C35002A04D0211C281C0C316A
:108D6000FFF715FE301C2168FFF752FE281C70BD6E
:108D7000036837B50C3B5A68914202D19A68002AC1
:108D800010DD1A68914200D2111C041C8A1A181CAA
:108D900001A9FFF7D3FF051C206801A90C38FFF7D4
:108DA00095FE256037BDF8B50B68041C0C3B1E68AA
:108DB0000F1C002E1ED003680C3B1A68B5185A68A9
:108DC000954212D89B68002B0FDC236839681A1C67
:108DD0000C3A1068321C80001818FFF7D8FD206884
:108DE000291C0C38FFF714FE04E0201C291CFFF797
:108DF000BFFFEAE7201CF8BD08B5FFF7D4FF08BDA8
:108E0000F7B5041C0E1C171E31D01A4B0021FFF7BA
:108E1000A1FD236801930C3B1A68BD185A6895425E
:108E200002D89B68002B09DD201C311CFFF7A2FD36
:108E3000002813D0201C291CFFF79AFF2368311C3F
:108E40001A1C0C3A10683A1C80001818FFF79FFD96
:108E50002068291C0C38FFF7DBFD08E0019B201C73
:108E6000291CF61AFFF784FF23689E19E6E7201CE9
:108E7000FEBDC04621C90200F8B50E1C051C124BF0
:108E8000171C0021321CFFF765FD2B680C3B1A688C
:108E9000B4185A68944202D89B68002B03DD281C42
:108EA000211CFFF765FF2B68311C1A1C0C3A106857
:108EB0003A1C80001818FFF77CFD2868211C0C382C
:108EC000FFF7A6FD0020F8BD21C9020010B5041C63
:108ED000002901D0FFF7D0FF201C10BDF8B50F1CF2
:108EE0000368161C0C3B1C683A1C211C0A4B051C11
:108EF000FFF730FDBC4205D2391B281C321CFFF79E
:108F0000E5FF07E0A74205D20122281C391C524286
:108F1000FFF768FEF8BDC04636C9020008B500225A
:108F2000FFF7DCFF08BD036870B50C3B1A68051C31
:108F3000541C5A680E1C94420CD89B68002B09DC08
:108F40002A68211C101C0C3803689B009E50FFF7F8
:108F50005FFD70BD281C211CFFF70AFFF0E708B574
:108F60008368002B02DBFFF7DFFE02E00022FFF741
:108F7000E5FE08BD13B5041C086801AA69460C3853
:108F8000FFF7EDFF2060201C16BD0000F7B58842FA
:108F900001D10F4E1AE00C1C051E04D1002C02D08A
:108FA0000C4800F03DF8631B9B10181C0021019336
:108FB000FFF73AFD061C071C0C36301C291C221C2E
:108FC000FFF702FD381C0199FFF722FD301CFEBDA2
:108FD000BC0A00204BC9020070B5051C0C1C161CF5
:108FE000002905D0081C1EF049FE8000211801E070
:108FF00004214942321C201C0023FFF7C7FF2860D0
:10900000281C70BD10B5041C081C111C1A1C002360
:10901000FFF7BCFF2060201C10BD08B51AF06CFCE7
:1090200008B51AF069FC08B51AF066FC0FB41823ED
:10903000B3B500AFFC1820CC281C1CF0BBFD80236E
:109040009B00C118074B2A1CC0186B46C008C00003
:109050001B1A9D46231C68467C6000F05DF81AF0E0
:109060004BFCC0460E02000008B51AF045FC08B5DE
:109070001AF042FCF0B50C1A9FB000AF631C7B6085
:109080000C23061C1049F8186C221BF07FFA231CD5
:109090006A467A33DB08DB00D31A9D460C236B2229
:1090A000F91868461BF072FA68466D46221C6B3050
:1090B000311C1BF06BFA00227B686846EB186A33A0
:1090C0001A70FFF7ADFFC046A5C90200F0B5114BFD
:1090D00087B01B6804AF88B0009304AC0223061C61
:1090E000201C0193013B029318300023796007F0A4
:1090F000D2FD7B68051C834206D3211A1831301C2F
:109100002A1C1BF043FA01E001256D42BD46281CD4
:10911000FEBDC046B0000020F7B5071C151C041C9E
:10912000013946182A78002A39D0B44234D2252A87
:1091300026D16A78732A06D07A2A11D0253A51426C
:109140004A41AD181CE0181D1A68231C11781C1C1C
:1091500000291AD09E421BD0197001320133F5E765
:10916000AA78752A0CD11A1D0192311B201C1A688D
:10917000FFF7ACFF00280FDD24180335019BD1E772
:109180002A78013522700134CCE70235031CC9E787
:10919000381C311CFFF76EFF381C211CFAE7E01B5E
:1091A0002270FEBD014B18687047C046C00A0020FF
:1091B00010B5041C034B0833036000F0C3F8201CF7
:1091C00010BDC04618CA020010B5041CFFF7F0FF1E
:1091D000201CFFF76AF9201C10BDF7B51D1C089B69
:1091E000061C0F1C141C934206D1291C00F073F8B6
:1091F000002801D0062008E0B068089A03680092B1
:109200001E6A391C221C2B1CB047FEBDF0B50C1C7D
:1092100087B0191C0593071C04920F9E00F05BF8A1
:109220000C9B051E15D033606B461B7C3371002CE4
:1092300009DB0C9B0E9A1C190623A24200D0053BA9
:10924000B371002521E00025A31C1ED10123B371B9
:109250001BE00E9A934205D1381C0D9900F03BF8A3
:1092600000280FD1B8680C9A036800920D9A0396F3
:1092700001920E9A211C0292DD69049A059BA8476F
:10928000051C02E06B461B7C7371281C07B0F0BD07
:10929000F8B5071C0E1C151C1C1C00F068F80028F3
:1092A00006D1B868311C03682A1C9F69231CB84783
:1092B000F8BD08B580471AF01FFB000008B5024B47
:1092C0001868FFF7F6FFC046B40000207047002082
:1092D00070470020704708B5012381420FD04068D5
:1092E000002302782A2A0AD049680B782A3B5A427E
:1092F0005341C9181BF0C2FF43424341DBB2181C63
:1093000008BD7FB500246B461C71102302930368CF
:10931000151C9E6912686B4600940394B0476B4617
:109320001A790623201C1340062B02D1009B013022
:109330002B6004B070BD009B0620934200D005381E
:109340007047000010B5041C034B08330360FFF79F
:10935000BDFF201C10BDC04690CA020010B5041C01
:10936000FFF7F0FF201CFFF7A0F8201C10BD38B558
:10937000151C1C1CFFF7AFFF002804D00823E36076
:10938000023B2560237138BDF8B5051C0C1C161C6A
:109390001F1CFFF7A0FF002807D1032F05D8236863
:1093A000201C5B69291C321C9847F8BDF8B5141CB9
:1093B0001F1C089A069B051C099E934204D107991D
:1093C000FFF789FF00280BD1281C391CFFF783FF0A
:1093D000002806D0069B347133600123B37100E08E
:1093E00074710020F8BD0000104B021C083310B54A
:1093F00003600023243243608360C36003614361E0
:109400008361C3610362131C041C64300021196072
:10941000596008338342F9D10823201C6366A26691
:109420006C3000F079FE201C10BDC04600CB02005D
:1094300070B5051C0E1C8469002C06D0A2686368F8
:10944000301C291C98472468F6E770BD38B5041C09
:109450008069002802D10023A36138BDC3685A1E69
:10946000C260002BF7D10568FFF71FF8281CF0E752
:1094700010B5041C0C4B002108330360FFF7D8FF24
:10948000201CFFF7E3FF231CA06E2433984205D075
:10949000002801D0FEF7FEFF0023A366201C6C30DD
:1094A00000F08BF8201C10BD00CB020010B5041C8E
:1094B000FFF7DEFF201CFEF7F8FF201C10BD7047F1
:1094C00008B543685A1E4260012B02D103685B68ED
:1094D000984708BD0B681A68036001321A6070472C
:1094E00008B50348034900220DF0DCFB08BDC04667
:1094F000CC0A00202CCB0200044B10B51A681C1CAF
:10950000002A01D1FFF7ECFF206810BDCC0A002033
:10951000004870472CCB020038B500254368041C76
:10952000AB420DD1606800280ED0FEF7B3FF0BE010
:109530006268AB009858002801D0FFF7C1FF0135E1
:10954000A3689D42F4D3EDE70025E368AB420DD15B
:10955000E06800280ED0FEF79DFF0BE0E268AB004C
:109560009858002801D0FFF7ABFF0135A3689D4252
:10957000F4D3EDE700252369AB4208D12069002828
:109580000CD0FEF787FF09E00435182DF6D02369CB
:1095900058590028F8D0FEF77DFFF5E7201C38BDAC
:1095A000036810B55A1E0260012B05D1041CFFF799
:1095B000B3FF201CFEF779FF10BD10B5041C006836
:1095C000FFF7EEFF201C10BD38B50D1C041C0A6807
:1095D0000068136801331360FFF7E2FF2B68201C5B
:1095E000236038BDF8B5104F061C3B680D1C141CD9
:1095F000DB0707D4381C0DF01AFA002802D0381CFB
:109600000DF022FAF268A40012191368002B06D09C
:10961000002D08D02B68281C5B68984703E06B6816
:1096200001336B601560F8BDD80A00200368002B79
:1096300004D1044A136801331360036000680138E1
:109640007047C046D00A0020F0B585B0002A70D01F
:10965000041C081C151CFFF7E9FFA3680190013BDF
:10966000984249D96368061D0293FE23B0005B054A
:109670009E4201D901204042FEF72DFF0022071C27
:10968000A36899008A4204D060688058B8500432B8
:10969000F8E7B34204D200219A00B9500133F8E749
:1096A000E368B0000393FE235B059E4201D90120CD
:1096B0004042FEF710FFA3689A00944600226245DC
:1096C00004D0E168895881500432F8E7B34204D2EB
:1096D00000219A0081500133F8E7029BA660676081
:1096E000E060002B02D0181CFEF7D4FE039B002B79
:1096F00002D0181CFEF7CEFE6B6801336B60019B35
:109700009E0063689E193068002801D0FFF7D8FEDC
:1097100035600025A3689D420BD2E368AE009859DE
:10972000002804D0FFF7CCFE0023E26893510135F6
:10973000F0E705B0F0BD10B5041C0B6803600C3BEE
:10974000186849682150002161601868111C2018B0
:109750000BF0EFFD201C10BD70B5051C041C083576
:10976000281C0E1C0BF0AEFD054B281C2360054B7E
:10977000311CA360002363600BF0DBFD201C70BD77
:1097800044CB020058CB020038B5041C0D1E0F4B11
:1097900000D1136823600821002D01D10C3B19680A
:1097A00061180B4B002D00D153680B6000236360E0
:1097B000AB0703D5201C08300BF046FDEB0702D5A4
:1097C000201CFEF772FE201C38BDC04644CB0200B0
:1097D00058CB020008B502210022FFF7D5FF08BDD3
:1097E00008B503680C3B1B68C018FFF7F3FF08BD02
:1097F00010B5041CFFF7EEFF201CFEF756FE201CE0
:1098000010BD08B503680C3B1B68C018FFF7F0FFDC
:1098100008BD08B50A1C0021FFF7B6FF08BD10B54A
:10982000041C0B6803600C3B186849682150002138
:1098300061601868111C20180BF0E5FD201C10BD9C
:1098400070B5051C041C0835281C0E1C0BF0A0FD6F
:10985000054B281C2360054B311CA360002363606B
:109860000BF0D1FD201C70BD74CB020088CB020030
:1098700038B5041C0D1E0F4B00D11368236008215E
:10988000002D01D10C3B196861180B4B002D00D144
:1098900053680B6000236360AB0703D5201C0830BE
:1098A0000BF0DCFCEB0702D5201CFEF7FEFD201CB4
:1098B00038BDC04674CB020088CB020008B5022137
:1098C0000022FFF7D5FF08BD08B503680C3B1B68F5
:1098D000C018FFF7F3FF08BD10B5041CFFF7EEFF3B
:1098E000201CFEF7E2FD201C10BD08B503680C3BF0
:1098F0001B68C018FFF7F0FF08BD08B50A1C00215F
:10990000FFF7B6FF08BD08B503689B68984708BD18
:109910002523C06830B50B70030501D44B1C02E051
:109920002B248B1C4C70410502D523211970013367
:109930002E21197004395970991C002A01D0D91CA4
:109940009A7082235B0003404C1C042B01D16233CC
:109950000BE080228025D2016D00AB4201D145236E
:1099600000E04723104200D120330B700023237006
:1099700030BD30B514680139231C0C3B1A68051C36
:10998000013A914200D9111C41180120A94212D07C
:10999000002810D0A35C2878013A181A4342584195
:1099A0000135C0B2F2E7002808D0A35C013A581B89
:1099B00043425841C0B20D78002AF4D16BB2002B5B
:1099C00004DD0023227895425B41184030BD000041
:1099D00010B5074C2368DB0707D4201C0DF027F8CF
:1099E000002802D0201C0DF02FF8024810BDC04600
:1099F00098180020100B0020F8B51C23836000236A
:109A0000071CFC4A01604260FB4A0361C2600021FE
:109A10007A68F868D218C15004331160702BF6D1FF
:109A2000F64BF74C3B611C60FFF772FD0222011CF4
:109A3000201C1AF0ABFD042300243A69D4500433EF
:109A4000182BF9D1EF4D173B211C221C281C0CF0C0
:109A5000F5F82A1C381CEC49FFF7F6FDEB4D012107
:109A6000281C0DF08DFD381C2A1CE949FFF7ECFD80
:109A70000122E84BE84D5A60E64AE84B94601360D7
:109A8000131C0533DC77131C0633DC77131C64339B
:109A90001C70D460147454619461D4611462111CFC
:109AA000281C012206F04AFB381C2A1CDC49FFF75F
:109AB000CBFD0123DB4A381C5360DB4BDB491360D1
:109AC000FFF7C2FD0123DA4A381C5360D94BDA494B
:109AD0001360FFF7B9FDD94D0121281C06F032FCB7
:109AE000381C2A1CD649FFF7AFFD0122D54BD64DB5
:109AF0005A60D44AD54B94601360131C43331C70D6
:109B0000D46014745474947454619461D461146274
:109B100054629462D46214635463111C281C0122A1
:109B200006F010FA381C2A1CC949FFF78DFD0122E6
:109B3000C84BC94D5A60C74AC84B94601360131C88
:109B400043331C70D46014745474947454619461DD
:109B5000D461146254629462D46214635463111C1D
:109B6000281C012206F052FA381C2A1CBC49FFF7B7
:109B70006BFD0123BB4A381C5360BB4BBB491360D0
:109B8000FFF762FD0123BA4A381C5360B94BBA494A
:109B90001360FFF759FD0123B84E01227360B84BE3
:109BA000B4603360331DF46034617461B461F46196
:109BB00034627462B462F46234637463B463F463F1
:109BC00034647464B464F46434657465B465F465D1
:109BD00034667466B466F46634677467B467F467B1
:109BE000DC67331C0833DC67331C88331C60331C90
:109BF0008C331C60331C90331C60331C94331C600A
:109C0000331C98331C60331C9C331C60331CA03302
:109C10001C60331CA4331C60331CA8331C60331C31
:109C2000AC331C60331CB0331C60331CB4331C6079
:109C3000331CB8331C60331CBC331C60331CC03372
:109C40001C60331C8F4DC4331C70311C281C06F063
:109C5000BBFA381C2A1C8C49FFF7F6FC01238B4AFF
:109C6000381C53608A4B8B491360FFF7EDFC0123CE
:109C7000894A381C5360894B89491360FFF7E4FC1B
:109C8000884D0121281C06F04FFB2A1C381C8649F0
:109C9000FFF7DAFC854D0121281C0BF0E3FE2A1C9E
:109CA000381C8349FFF7D0FC824D0121281C0DF0A0
:109CB00077FC381C2A1C8049FFF7C6FC01227F4B29
:109CC0007F4D5A607D4A7F4B9460136092235B0006
:109CD000D454D460147454619461D4611462546295
:109CE0009462111C281C012200F05AFE381C2A1C08
:109CF0007549FFF7A9FC0123744A381C5360744B63
:109D000074491360FFF7A0FC0123734A381C5360A9
:109D1000724B73491360FFF797FC724D0121281CA9
:109D200000F042FF381C2A1C6F49FFF78DFC01220E
:109D30006E4B6F4D5A606D4A6E4B94601360131CEE
:109D40006C331C70D460147454619461D4611462D7
:109D500054629462D462146354639463D463111C98
:109D6000281C012200F020FD381C2A1C6249FFF744
:109D70006BFC0122614B624D5A60604A614B9460FA
:109D80001360131C6C331C70D460147454619461A0
:109D9000D461146254629462D46214635463946311
:109DA000D463111C281C012200F062FD381C2A1CFF
:109DB0005549FFF749FC0123544A381C5360544B62
:109DC00054491360FFF740FC0123534A381C536089
:109DD000524B53491360FFF737FC0123514D0122C9
:109DE0006B60514BAC602B602B1DEC602C616C6187
:109DF000AC619BE04817002028180020DC0B0020F5
:109E0000040B0020300D0020D01E0020600B00202D
:109E1000F41E0020B81700203C0B002070D6020072
:109E2000501900209C18002090D402004C190020EA
:109E3000580B0020D0D4020048190020F00A00205E
:109E4000341900202C1600205C10002050D602008F
:109E500060190020F01600204410002060D6020097
:109E60005C190020640F0020E0D502005819002082
:109E7000480B0020F8D5020054190020741000206F
:109E800000D50200DC0A002044190020E81600205A
:109E900028D602003C1900203C10002010D60200F9
:109EA000401900202C0B0020381900203C11002004
:109EB000CC1E0020200B0020F81E0020080C0020E3
:109EC000140B002038D00200F01800206C0F002086
:109ED00058CE0200EC180020500B002098CE020053
:109EE000E818002050100020D41800206C0B00202F
:109EF000FC0B002018D00200001900207016002072
:109F00006810002028D00200FC180020FC0A002065
:109F1000A8CF0200F8180020E0160020C0CF0200F1
:109F2000F4180020740F0020C8CE0200EC612C62EF
:109F30006C62AC62EC622C636C63AC63EC632C64AB
:109F40006C64AC64EC642C656C65AC65EC652C668B
:109F50006C66AC66EC662C676C67AC67EC67DC67BC
:109F60002B1C0833DC672B1C88331C602B1C8C33A8
:109F70001C602B1C90331C602B1C94331C602B1C0E
:109F800098331C602B1C9C331C602B1CA0331C6062
:109F90002B1CA4331C602B1CA8331C602B1CAC3363
:109FA0001C602B1CB0331C602B1CB4331C602B1C9E
:109FB000B8331C602B1CBC331C602B1CC0331C60D2
:109FC0002B1CC4331C702F4C291C201C00F02EFDB0
:109FD000381C221C2C49FFF737FB01232B4A381C65
:109FE00053602B4B2B491360FFF72EFB01232A4AAA
:109FF000381C5360294B2A491360FFF725FB294C75
:10A000000121201C00F0C2FD221C2749381CFFF74B
:10A010001BFB2648FC68FFF709FB254B800003511A
:10A020002448FC68FFF702FB234B800003512348C0
:10A03000FC68FFF7FBFA224B800003512148FC68C3
:10A04000FFF7F4FA800006511F48FC68FFF7EEFAAC
:10A050001E4B800003511E48FC68FFF7E7FA1D4BBA
:10A06000800003511C48FC68FFF7E0FA1B4B80009E
:10A0700003510548FC68FFF7D9FA80000551381CE8
:10A08000F8BDC046500F0020E4180020F40B00205B
:10A09000F0CF0200DC18002020180020D8CF0200EA
:10A0A000E01800201C160020D818002050190020AD
:10A0B000B8170020601900202C1600205C19002021
:10A0C000F016002044190020F0180020080C002091
:10A0D000001900206C0B0020FC18002070160020D6
:10A0E00010B5054C0221201CFFF786FC034B1C60B9
:10A0F000034B1C6010BDC04634170020C80A002066
:10A10000D40A002008B5034B1B68002B01D1FFF7D0
:10A11000E7FF08BDC80A002038B50023041C03600F
:10A12000FFF7F0FF094D0A4A2B682360126893423B
:10A1300003D11A6801321A6006E0FFF749FC2B6868
:10A140001A6801321A602360201C38BDD40A00202E
:10A15000C80A002083685869704783689869704707
:10A160008368586B704713B58368FF249B6B181C7A
:10A17000190A1A0C21402040090222401204084307
:10A180001B0E1B061043184316BD13B58368FF242E
:10A19000DB6B181C190A1A0C2140204009022240CE
:10A1A000120408431B0E1B061043184316BD836898
:10A1B000586970478368986970478368586B70471F
:10A1C00013B58368FF249B6B181C190A1A0C2140D5
:10A1D000204009022240120408431B0E1B061043B4
:10A1E000184316BD13B58368FF24DB6B181C190ACE
:10A1F0001A0C2140204009022240120408431B0E81
:10A200001B061043184316BD8368586A704783685D
:10A21000986A704700207047002070477047002000
:10A22000914204D21923D84108C9C018F8E77047F1
:10A2300013B5041C8B6801AA99680CF0EBF8201C7C
:10A2400016BD13B5041C8B6801AA99680CF0E2F8DE
:10A25000201C16BD13B5041C8B6801AA99680CF06C
:10A26000D9F8201C16BD13B5041C8B6801AAD96946
:10A27000FEF7B2FE201C16BD13B5041C8B6801AAA4
:10A28000596AFEF7A9FE201C16BD13B5041C8B6885
:10A2900001AAD96AFEF7A0FE201C16BD13B5041C46
:10A2A0008B6801AAD969FEF797FE201C16BD13B56D
:10A2B000041C8B6801AA596AFEF78EFE201C16BD8D
:10A2C00013B5041C8B6801AAD96AFEF785FE201C11
:10A2D00016BD13B5041C8B6801AA5969FEF77CFEF4
:10A2E000201C16BD13B5041C8B6801AAD969FEF7A2
:10A2F00073FE201C16BD0000104B10B50360031C3C
:10A300006C331B78041C002B13D08068002801D00C
:10A31000FEF7C0F8E069002801D0FEF7BBF8606ADC
:10A32000002801D0FEF7B6F8E06A002801D0FEF759
:10A33000B1F8201CFFF7C3F8201C10BD18D0020094
:10A34000104B10B50360031C6C331B78041C002BEE
:10A3500013D08068002801D0FEF79CF8E06900283F
:10A3600001D0FEF797F8606A002801D0FEF792F856
:10A37000E06A002801D0FEF78DF8201CFFF79FF857
:10A38000201C10BD28D0020010B5041C024B036035
:10A39000FFF795F8201C10BDA8CF020010B5041CD3
:10A3A000024B0360FFF78BF8201C10BDC0CF0200EA
:10A3B0000E4B10B5036092235B00C35C041C002BA2
:10A3C0000ED08068002801D0FEF764F8606900288C
:10A3D00001D0FEF75FF8E069002801D0FEF75AF8D7
:10A3E000201CFFF76CF8201C10BDC04638D00200BE
:10A3F00010B5041C024B0360FFF761F8201C10BD70
:10A4000058CE020010B5041C024B0360FFF757F84A
:10A41000201C10BD98CE020010B5041C024B036036
:10A42000FFF74DF8201C10BDC8CE020010B5041C6B
:10A43000024B0360FFF743F8201C10BDD8CF020089
:10A4400010B5041C024B0360FFF739F8201C10BD47
:10A45000F0CF020010B5041CFFF74EFF201CFEF7E2
:10A4600024F8201C10BD10B5041CFFF769FF201C48
:10A47000FEF71BF8201C10BD10B5041CFFF784FF6D
:10A48000201CFEF712F8201C10BD10B5041CFFF7AD
:10A4900085FF201CFEF709F8201C10BD10B5041C18
:10A4A000FFF786FF201CFEF700F8201C10BD10B53A
:10A4B000041CFFF79DFF201CFDF7F7FF201C10BDBB
:10A4C00010B5041CFFF79EFF201CFDF7EEFF201CBB
:10A4D00010BD10B5041CFFF79FFF201CFDF7E5FF22
:10A4E000201C10BD10B5041CFFF7A0FF201CFDF7B9
:10A4F000DCFF201C10BD10B5041CFFF7A1FF201CC1
:10A50000FDF7D3FF201C10BD10B5041C044B0360E5
:10A5100008300CF0D9FB201CFEF7D1FF201C10BD29
:10A5200058CF020010B5041CFFF7EEFF201CFDF70A
:10A53000BCFF201C10BD000010B5041C044B0360C0
:10A5400008300CF0C1FB201CFEF7B9FF201C10BD29
:10A55000D0CD020010B5041CFFF7EEFF201CFDF764
:10A56000A4FF201C10BD000038B50E4B0569036028
:10A57000041CFEF7CDFF854204D0002D02D0281C1C
:10A58000FDF788FFA068002802D003685B68984741
:10A59000201C0C300CF098FB201CFEF790FF201CB8
:10A5A00038BDC046D8CE020010B5041CFFF7DCFF52
:10A5B000201CFDF77AFF201C10BDF0B51C1C87B0D5
:10A5C00005AB071C04A8FEF71DFD211C03AB05A865
:10A5D0000C9AFEF717FD049C059D231C0C3B1B6881
:10A5E0009B00E31801932B1C0C3B1E68B600AE19B0
:10A5F000381C211C2A1C0CF03CFA002816D1201C07
:10A600001DF03CFB80002418281C1DF037FB019B2B
:10A6100080002D189C4204D1AE1B751EAE417642BF
:10A6200007E0B54204D004340435E1E7061C00E03D
:10A63000012605A8FEF758FA04A8FEF755FA301CC3
:10A6400007B0F0BDF0B51C1C2B4B85B0036000912A
:10A65000171C111C02AB221C061C03A8FEF7D2FC1F
:10A66000039DE41B2B1C0C3B1B6864109B00EB1828
:10A670000193FE23A0005B059C4201D901204042CA
:10A68000FDF729FF071C2A1C0098391C231C0CF01D
:10A69000FBF9021EA24214D3441C381CFDF7FAFE3B
:10A6A000FE23A0005B059C4201D901204042FDF73A
:10A6B00012FF071C2A1C0098391C231C0CF0E4F91B
:10A6C000021C391C301CFEF79BFB281C1DF0D6FA1F
:10A6D000019B80002D189D4205D0301C00210435BF
:10A6E000FEF721FCCFE7381CFDF7D4FE03A8FEF7E8
:10A6F000FBF9301C05B0F0BDBC0A00200A2806D8C2
:10A700002F2915D93030814212D230390EE0081C81
:10A71000303809280ED90B1C613B052B01D857395D
:10A7200004E00B1C413B052B02D83739081C01E023
:10A73000012040427047000008B4FFB50420019199
:10A74000002119F059FE174F061C391C1AF096FD0E
:10A750000024A0420FD0301C1BF02CFA451C281CF2
:10A76000FDF7B9FE311C2A1C041C19F00FFF042050
:10A77000391C19F041FE0AAA0198099903921CF0AC
:10A78000DBFC051C002C06D00420211C19F034FE33
:10A79000201CFDF77FFE281C04B0F0BC08BC01B0F3
:10A7A0001847C046AFC3020010B5531E9A418160DE
:10A7B0000021041C034B426003600A1C0CF0ACFB3C
:10A7C000201C10BD20CF020008B503689B68984785
:10A7D00008BD08B50368DB68984708BD10B5041CC0
:10A7E0000B681B699847201C10BD10B5041C0B6832
:10A7F0005B699847201C10BD10B5041C0B689B6951
:10A800009847201C10BD10B5041C0B68DB699847E5
:10A81000201C10BD08B503681B6A984708BD036873
:10A8200013B55B6A9847FF22041C010A030C114010
:10A83000144009021A4012042143000E114303067A
:10A84000081C184316BD036813B59B6A9847FF227E
:10A85000041C010A030C1140144009021A4012049E
:10A860002143000E11430306081C184316BD0000C7
:10A8700010B5531E9A4181600021041C034B4260B5
:10A8800003600A1C0CF0F8FA201C10BDE8CE020090
:10A8900008B503689B68984708BD08B50368DB687E
:10A8A000984708BD10B5041C0B681B699847201C0D
:10A8B00010BD10B5041C0B685B699847201C10BDC7
:10A8C00010B5041C0B689B699847201C10BD10B57F
:10A8D000041C0B68DB699847201C10BD08B5036891
:10A8E0001B6A984708BD036813B55B6A9847FF2247
:10A8F000041C010A030C1140144009021A401204FE
:10A900002143000E11430306081C184316BD0368BB
:10A9100013B59B6A9847FF22041C010A030C1140DF
:10A92000144009021A4012042143000E1143030689
:10A93000081C184316BD00004B1E99410A4B021C0F
:10A94000036000236C3241608360C3600374436121
:10A950008361C361036243628362C36203634363CF
:10A960008363C3631370704718D002004B1E994174
:10A970000A4B021C036000236C3241608360C36099
:10A98000037443618361C361036243628362C36290
:10A99000036343638363C3631370704728D002006B
:10A9A000531E9A4110B5041C044B42600360816041
:10A9B00000210BF0D9F8201C10BDC04630CE02009B
:10A9C00008B503689B68984708BD08B50368DB684D
:10A9D000984708BD10B5041C0B681B699847201CDC
:10A9E00010BD10B5041C0B685B699847201C10BD96
:10A9F00010B5041C0B689B699847201C10BD000013
:10AA00004B1E9941084B9222036000235200416083
:10AA10008360C360037443618361C3610362436203
:10AA2000836283547047C04638D00200531E9A4157
:10AA3000074B10B5426003608160041CFEF768FD9F
:10AA400000212061201C0CF043FC201C10BDC046DE
:10AA5000D8CE020083689B680B608368DB684B601C
:10AA6000704783681B690B6083685B694B60704744
:10AA700083689B690B608368DB694B607047836800
:10AA8000DB6A0B6083681B6B4B6083685B6B8B605E
:10AA900083689B6BCB608368DB6B0B6183681B6C8B
:10AAA0004B6183685B6C8B61704783689B6C0B6048
:10AAB0008368DB6C4B6083681B6D8B6083685B6DA8
:10AAC000CB6083689B6D0B618368DB6D4B61836832
:10AAD0001B6E8B61704783685B6E0B6083689B6E37
:10AAE0004B608368DB6E8B6083681B6FCB60836811
:10AAF0005B6F0B6183689B6F4B618368DB6F8B615E
:10AB000083680433DB6FCB6183680833DB6F0B62D0
:10AB1000836888331B684B6283688C331B688B6245
:10AB2000836890331B68CB627047836894331B68DB
:10AB30000B60836898331B684B6083689C331B6889
:10AB40008B608368A0331B68CB608368A4331B6869
:10AB50000B618368A8331B684B618368AC331B6847
:10AB60008B618368B0331B68CB618368B4331B6827
:10AB70000B628368B8331B684B628368BC331B6805
:10AB80008B628368C0331B68CB6270474B1E994150
:10AB9000044B10B541600360041CFEF7ADFCA060DF
:10ABA000201C10BD58CF02004B1E9941044B10B51C
:10ABB00041600360041CFEF79FFCA060201C10BDD8
:10ABC000D0CD020010B5041C0B48FEF72FFD236802
:10ABD0005A689B68984203D280008058002801D1AF
:10ABE000FEF71BFA0549064A00230BF033FC002848
:10ABF00001D10BF019FF10BDCC1E002024CB0200A8
:10AC00007CDC020010B5041C0B48FEF70FFD236826
:10AC10005A689B68984203D280008058002801D16E
:10AC2000FEF7FBF90549064A00230BF013FC002848
:10AC300001D10BF0F9FE10BDF018002024CB02006A
:10AC4000C4D3020010B5041C0B48FEF7EFFC2368C8
:10AC50005A689B68984203D280008058002801D12E
:10AC6000FEF7DBF90549064A00230BF0F3FB002849
:10AC700001D10BF0D9FE10BDE818002024CB020052
:10AC800000D1020010B5041C0B48FEF7CFFC23686E
:10AC90005A689B68984203D280008058002801D1EE
:10ACA000FEF7BBF90549064A00230BF0D3FB002849
:10ACB00001D10BF0B9FE10BDEC18002024CB02002E
:10ACC000A0D1020010B5041C0B48FEF7AFFC2368AE
:10ACD0005A689B68984203D280008058002801D1AE
:10ACE000FEF79BF90549064A00230BF0B3FB002849
:10ACF00001D10BF099FE10BDFC18002024CB0200FE
:10AD0000DCD2020010B5041C0B48FEF78FFC236850
:10AD10005A689B68984203D280008058002801D16D
:10AD2000FEF77BF90549064A00230BF093FB002848
:10AD300001D10BF079FE10BD0019002024CB0200D8
:10AD4000E0D0020010B5041C0B48FEF76FFC23682E
:10AD50005A689B68984203D280008058002801D12D
:10AD6000FEF75BF90549064A00230BF073FB002848
:10AD700001D10BF059FE10BDE418002024CB0200D5
:10AD800044D3020010B5041C0A48FEF74FFC2368A8
:10AD900099685A68002388420AD2800080589842F5
:10ADA00006D00549054A0BF055FB431E9841C3B236
:10ADB000181C10BDCC1E002024CB02007CDC02003D
:10ADC00010B5041C0A48FEF731FC236899685A68DC
:10ADD000002388420AD280008058984206D0054954
:10ADE000054A0BF037FB431E9841C3B2181C10BD37
:10ADF000E818002024CB020000D1020010B5041C8A
:10AE00000A48FEF713FC236899685A6800238842B1
:10AE10000AD280008058984206D00549054A0BF0B6
:10AE200019FB431E9841C3B2181C10BDEC1800203A
:10AE300024CB0200A0D10200F0B500259C462C1CBA
:10AE400085B002910B9F0A990392039B1B191E78F0
:10AE500001937B1A9B10B34202DC061C0B1C0CE016
:10AE600073B2002BF9DD6346B600013BBF1B9C4269
:10AE700001D20134E9E70135E7E7BB4202D004CB58
:10AE800004C6FAE7591A890889004018013D12D30F
:10AE90000021029A0260019A1678B6000F1DB14295
:10AEA00004D05A5841184A60391CF7E7C0195B189A
:10AEB000ECE780195B18013C0DD30021029A026077
:10AEC000039A155DAD000E1DA942F2D05F584118DE
:10AED0004F60311CF7E705B0F0BDF7B5089F8C4611
:10AEE000141C0A990B9E002F02D07D1AAD1000E0B1
:10AEF0003568AA008A1800910192191C0998231C30
:10AF00006246FFF799FF099BC41AA410002F07D0CF
:10AF10003368391C5A1B1DF03DF833685D1B6419FA
:10AF20003460F7BD73B50E1C151C0898099C009081
:10AF30002268191C920082182B1C01920798321C5F
:10AF4000FFF77AFF079BC01A8010206073BDF8B529
:10AF5000171C06AA1278061C0D1C002A10D0041C0F
:10AF6000281C0A2115F048FB04318900CB59043C08
:10AF7000281C23600A2115F0B9FA051EF0D11CE047
:10AF80004A221A40402A0AD1041C07232B400433CA
:10AF90009B00DB59043C2360ED08F6D10DE0142240
:10AFA0005B0400D4103A341C0F232B409B189B00E9
:10AFB000DB59043C23602D09F6D1301B8010F8BD0D
:10AFC000F8B51E1C08AB1B78071C141C0799002B36
:10AFD00017D0051C201C311C0A22002315F080FC10
:10AFE000069B04329200D358043D2B60201C311C78
:10AFF0000A22002315F074FC041C0E1C0843E9D13E
:10B0000028E04A230B40402B10D1051C0723234086
:10B010000433069A9B009B58043D2B60E408730799
:10B020001C43231CF6083343F0D113E014224B04D5
:10B0300000D4103A3D1C0F2323409B1806999B0017
:10B040005B58043D2B60240933071C43231C36093D
:10B050003343F0D1781B8010F8BD10B50468E46A62
:10B06000A04710BD031CF7B501226C331A70041CF5
:10B07000081C0F1CFFF746FE051CFFF7A5FB6061CF
:10B08000281CFFF7A6FBA061281CFFF7C3FB291CA7
:10B09000606301A8FFF7A2FB019B01A80C3B1B68A2
:10B0A000E3600AF025FFE068FDF715FA061C291C8D
:10B0B00001A8FFF793FBE2680023311C01A80AF006
:10B0C0006BFE01A80AF014FF0023E268A6609A4212
:10B0D00004D00022B256D3179B1ADB0F237401A8A9
:10B0E000291CFFF782FB019B01A80C3B1B68236214
:10B0F000FDF7FAFCFE23206A5B05984201D8800028
:10B1000001E001204042FDF7E6F9061C291C01A8D8
:10B11000FFF76BFB226A0023311C01A8FDF75AFCE4
:10B1200001A8FDF7E1FC01A8291CE661FFF764FB1B
:10B13000019B01A80C3B1B68A362FDF7D5FCFE2315
:10B14000A06A5B05984201D8800001E001204042DE
:10B15000FDF7C1F9061C291C01A8FFF74DFBA26AE7
:10B160000023311C01A8FDF735FC01A8FDF7BCFC4C
:10B1700001A8291C6662FFF746FB019B01A80C3B56
:10B180001B682363FDF7B0FCFE23206B5B05984230
:10B1900001D8800001E001204042FDF79CF9061C27
:10B1A000291C01A8FFF72FFB311C226B002301A8EB
:10B1B000FDF710FC01A8FDF797FCE662281CFFF7DD
:10B1C0002EFBA063281CFFF73EFBE063381CFFF753
:10B1D000F9FC044B1968231C0A1C40330B32FFF79F
:10B1E0003CFFF7BDAC000020F7B5061C0E48FEF78B
:10B1F0001DFA32688300D4680190E4182768002F94
:10B200000FD17020FDF755F9051C391CFFF794FB91
:10B21000281C311CFFF726FF3068291C019AFEF715
:10B22000E1F92068FEBDC04600190020031CF7B5F7
:10B2300001226C331A70041C081C0F1CFFF742FD1E
:10B24000051CFFF725FB6061281CFFF726FBA061AA
:10B25000281CFFF743FB291C606301A8FFF722FBB2
:10B26000019B01A80C3B1B68E3600AF041FEE0680B
:10B27000FDF731F9061C291C01A8FFF713FBE26852
:10B280000023311C01A80AF087FD01A80AF030FE56
:10B290000023E268A6609A4204D00022B256D31777
:10B2A0009B1ADB0F237401A8291CFFF702FB019BEB
:10B2B00001A80C3B1B682362FDF716FCFE23206AE5
:10B2C0005B05984201D8800001E001204042FDF773
:10B2D00002F9061C291C01A8FFF7EBFA226A0023D9
:10B2E000311C01A8FDF776FB01A8FDF7FDFB01A8C5
:10B2F000291CE661FFF7E4FA019B01A80C3B1B68DF
:10B30000A362FDF7F1FBFE23A06A5B05984201D81A
:10B31000800001E001204042FDF7DDF8061C291CF9
:10B3200001A8FFF7CDFAA26A0023311C01A8FDF79E
:10B3300051FB01A8FDF7D8FB01A8291C6662FFF7A5
:10B34000C6FA019B01A80C3B1B682363FDF7CCFBED
:10B35000FE23206B5B05984201D8800001E00120AC
:10B360004042FDF7B8F8061C291C01A8FFF7AFFA08
:10B37000311C226B002301A8FDF72CFB01A8FDF76F
:10B38000B3FBE662281CFFF7AEFAA063281CFFF7A8
:10B39000BEFAE063381CFFF715FC044B1968231C48
:10B3A0000A1C40330B32FFF758FEF7BDAC000020FB
:10B3B000F7B5061C0E48FEF739F932688300D468E9
:10B3C0000190E4182768002F0FD17020FDF771F865
:10B3D000051C391CFFF7CAFA281C311CFFF726FF91
:10B3E0003068291C019AFEF7FDF82068FEBDC046B2
:10B3F000FC1800209223F7B501225B00C254041C04
:10B40000081C0F1CFFF7FEFB051C01A8291CFFF7F9
:10B41000E1FA019B01A80C3B1B68E3600AF068FDA0
:10B42000E068FDF758F8061C291C01A8FFF7D2FABE
:10B43000E2680023311C01A80AF0AEFC01A80AF062
:10B4400057FD0023E268A6609A4204D00022B2565B
:10B45000D3179B1ADB0F237401A8291CFFF7C1FA2D
:10B46000019B01A80C3B1B68A361FDF73DFBFE237C
:10B47000A0695B05984201D8800001E001204042AC
:10B48000FDF729F8061C291C01A8FFF7AAFAA269F2
:10B490000023311C01A8FDF79DFA01A8FDF724FB4C
:10B4A00001A8291C6661FFF7A3FA019B01A80C3BC8
:10B4B0001B682362FDF718FBFE23206A5B05984298
:10B4C00001D8800001E001204042FDF704F8061C8D
:10B4D000291C01A8FFF78CFA311C226A002301A85D
:10B4E000FDF778FA01A8FDF7FFFAE661281CFFF7DF
:10B4F00067FA6062281CFFF768FAA062381CFFF741
:10B5000061FB094B051C1968231C0A1C2C332432CF
:10B51000FFF7A3FD054B281C1968231C0A1CBC332C
:10B520001A32FFF79AFDF7BDB0000020A8000020F6
:10B53000F7B5061C0E48FEF779F832688300D46828
:10B540000190E4182768002F10D194204000FCF7E8
:10B55000B0FF051C391CFFF753FA281C311CFFF7FC
:10B5600049FF3068291C019AFEF73CF82068FEBDAF
:10B57000F018002010B5041C0068002804D00AF060
:10B58000CEF901235B426360201C10BD73B5D5B2B8
:10B59000061C6C4600910192002D08D1081C069AE9
:10B5A000191C0AF0D4F9069B984200D00135331CCF
:10B5B0002571301C06CC06C376BD0000F0B591B0F5
:10B5C000169F07903C1C6C34201C08920993FFF7CF
:10B5D000F9FA061C201CFFF7EBFE189B016C1D6896
:10B5E000041C2B1C2A680C3B8A4206D0826B0B92EF
:10B5F000426A0492826A029209E0C26B0B92C26AAA
:10B600000492026B02921A68002A00D00435326854
:10B610001B6852699B00EB189446301C04212A1CBD
:10B62000E047401B8310039300D1D4E06E4B0CA87D
:10B630000C93039B5900FDF79BFB636B039AD61A8F
:10B64000002E2ADD002B00DA161CE368002B1FD029
:10B65000710000220CA8FDF7FBFA0CA8FDF7B8FA60
:10B66000B300EB1800950193A169A268E3680C98F8
:10B67000FFF7E2FB05900CA8FDF7AAFA0C9A059BD0
:10B680000CA8991A012289105242FDF7ABFA04E086
:10B690000CA8291C321CFDF70BFB636B002B14DD7F
:10B6A0000CA86169FDF73FFC002E04DBB600A91968
:10B6B0000CA8626B07E07142626C0CA8FDF706FCF7
:10B6C000291C039A0CA8FDF79BFBB023FA681340D2
:10B6D00006930C9B0C3B1E68029B9E19002392054F
:10B6E00000D5236AF618404B71000DA80D93FDF7A5
:10B6F0003FFB00230593069BBD68102B03D1AE4290
:10B700009B415B42059300230393039A0BABD05CF0
:10B71000042829D814F0D6FE2018030C1300FB6867
:10B720009B0521D50DA8E169226AFDF769FB1BE0A5
:10B73000029B002B18D0049B0DA8196809E00DA8E6
:10B740000CA9FDF759FB0FE0059B002B07D11799BA
:10B750000DA8FDF7E8FB07E0059B002B04D0A91B13
:10B760000DA8179AFDF7B2FB039B01330393042B3B
:10B77000CBD1029B012B06D91A1C0499013A043142
:10B780000DA8FDF73DFB0D9B0C3B1A6895420ED9A9
:10B79000069BAA1A0DA8202B04D1111C179AFDF79D
:10B7A00095FB05E00021179BFDF75CFA00E0151CF6
:10B7B0000EAE301C0899099A0D9B0095FFF7E6FE26
:10B7C0000E9B08AC089333790DA82371FDF78CF913
:10B7D0000CA8FDF789F90023079ABB6008AB03CBDF
:10B7E00003C2079811B0F0BDBC0A0020F0B591B0BB
:10B7F000169F07903C1C6C34201C08920993FFF79D
:10B80000E1F9061C201CFFF7EFFC189B016C1D687A
:10B81000041C2B1C2A680C3B8A4206D0826B0B92BC
:10B82000426A0492826A029209E0C26B0B92C26A77
:10B830000492026B02921A68002A00D00435326822
:10B840001B6852699B00EB189446301C04212A1C8B
:10B85000E047401B8310039300D1D4E06E4B0CA84B
:10B860000C93039B5900FDF783FA636B039AD61A76
:10B87000002E2ADD002B00DA161CE368002B1FD0F7
:10B88000710000220CA8FDF7E3F90CA8FDF7A0F960
:10B89000B300EB1800950193A169A268E3680C98C6
:10B8A000FFF7CAFA05900CA8FDF792F90C9A059BD0
:10B8B0000CA8991A012289105242FDF793F904E06D
:10B8C0000CA8291C321CFDF7F3F9636B002B14DD67
:10B8D0000CA86169FDF727FB002E04DBB600A9194F
:10B8E0000CA8626B07E07142626C0CA8FDF7EEFADF
:10B8F000291C039A0CA8FDF783FAB023FA681340B9
:10B9000006930C9B0C3B1E68029B9E19002392051C
:10B9100000D5236AF618404B71000DA80D93FDF772
:10B9200027FA00230593069BBD68102B03D1AE4276
:10B930009B415B42059300230393039A0BABD05CBE
:10B94000042829D814F0BEFD2018030C1300FB684E
:10B950009B0521D50DA8E169226AFDF751FA1BE08C
:10B96000029B002B18D0049B0DA8196809E00DA8B4
:10B970000CA9FDF741FA0FE0059B002B07D11799A1
:10B980000DA8FDF7D0FA07E0059B002B04D0A91BFA
:10B990000DA8179AFDF79AFA039B01330393042B22
:10B9A000CBD1029B012B06D91A1C0499013A043110
:10B9B0000DA8FDF725FA0D9B0C3B1A6895420ED990
:10B9C000069BAA1A0DA8202B04D1111C179AFDF76B
:10B9D0007DFA05E00021179BFDF744F900E0151CF6
:10B9E0000EAE301C0899099A0D9B0095FFF7CEFD0D
:10B9F0000E9B08AC089333790DA82371FDF774F8FA
:10BA00000CA8FDF771F80023079ABB6008AB03CBC5
:10BA100003C2079811B0F0BDBC0A0020F0B591B088
:10BA200004AFBA611822FB613023BA18D3181B780F
:10BA300018227B601023F960F96CBA186C317861B8
:10BA4000D018FDF747FD18221023BA18D018FFF7B9
:10BA5000B9F8D0B004AB3B61B860FDF74DFD1822DA
:10BA600014230026BA18D418F862BA6DFB6D00963C
:10BA7000029203933969321C1F4B201CFEF75CFEB7
:10BA80000C23051C321C1836BE19291CF318201C67
:10BA9000FDF712F83B69201C5D19FDF799F8FB6A68
:10BAA000B86839692A1CFFF7D8FA7B68002B0BD0DD
:10BAB000FB6C029400933B6D78690193F968BA6955
:10BAC000FB69FFF77BFD0AE0FB6C029400933B6D82
:10BAD00078690193F968BA69FB69FFF787FE201C52
:10BAE000FDF702F818221023BA18D018FDF765FDEB
:10BAF000BD4678690DB0F0BDD6D3020030B5041C48
:10BB000087B005930AAB1D7804920B980C9A0D9B95
:10BB1000009001920293201C049A059B002D02D0F4
:10BB2000FFF74CFD01E0FFF761FE201C07B030BDC0
:10BB300008B503681B6B984708BD08B503689B6A86
:10BB4000984708BDF7B5141C1D1C099A089B019164
:10BB50009F1AB023C2681340202B0CD1291C099ACC
:10BB6000201C1CF017FA099B01999A00A0183A1C96
:10BB70001CF01AFA45E00026102B13D16C30FFF7A9
:10BB800021F82D21061CFFF7D8FF2B68984206D01C
:10BB9000301C2B21FFF7D1FF2B68984210D10126D2
:10BBA0002B6808C401993A1C201C1CF0FDF9099B64
:10BBB000B800B100201869189A1B1CF0EBF920E0BE
:10BBC000301C3021FFF7B9FF2B68984217D1099B31
:10BBD000012B14DD301C7821FFF7AFFF6B68984212
:10BBE00006D0301C5821FFF7A8FF6B68984206D199
:10BBF0002B68022623606B6863600834D2E7002656
:10BC0000D0E7F7BDF0B58FB004AF3D6C7860281C6D
:10BC10006C30BA61FB613960FFF78AFC031C2C337E
:10BC2000BB60EB6896B07B614A237A69041C1A40BA
:10BC300004AEFA60402A01D0082A03D100233B61F8
:10BC4000B96C06E001233B61BB6C002BF8DCBB6CDC
:10BC50005942301C3B6950300093BA687B69FFF74A
:10BC600076F9142378621B1A227C9B00F318002AB1
:10BC700014D06A46C0001030121A9546182202935A
:10BC80000C23BA18D31806AE009501960393A36A45
:10BC90003868A168E268FFF745F9331C39697A6AA8
:10BCA000002909D0B96C002903DB7969090528D47A
:10BCB00011E0043BE16A26E0796989050BD5B96C8E
:10BCC000002908D0F968181F402920D1E36B013200
:10BCD0000360031C7A62AC68796A8C4224DD684692
:10BCE000A2000E32D208D200821A954604AE009409
:10BCF0000191281C796C321CFFF724FF7C62331CF5
:10BD000012E0216B043B196001327A62E3E7796942
:10BD1000BE684904C90F023189008959083B016096
:10BD2000E16B02321960F0E70022AA607A6A0092A1
:10BD30007868B969FA69FFF729FCBD4678680BB0E5
:10BD4000F0BDF0B58DB004AF3A6110227B613023B5
:10BD5000BD6BBA18D3181C78EB6838607B60DB07C2
:10BD60000CD40095FB6B1022019308230294BA189F
:10BD7000D0183A697B69FFF745FF5FE0281C6C30FB
:10BD8000FFF7D6FB002C02D04669846901E0C66942
:10BD9000046AAB68A34245DD6A461B1BFB609B003F
:10BDA0000E33DB08DB00D31A9D4604AB181CFA687F
:10BDB000F96BBB601CF0F8F800237A68AB60B03315
:10BDC0001A40131E202B17D110220094183BBA18CA
:10BDD000D01839697A69331CFFF7D8FBBB69102288
:10BDE0003B613B7FBA183B75FB6800930823B96938
:10BDF000D0187A69BB681FE0FB6810220093082303
:10BE0000BA18D01839697A69BB68FFF7BFFBBB69FC
:10BE100010223B613B7FBA183B7508230094D01871
:10BE2000B96907E000231022AB6000940833BA1808
:10BE30003969D018331C7A69FFF7A8FBBB69BD4686
:10BE40003B613B7F3A683B751023FB1803CB03C271
:10BE5000386809B0F0BD10B5041C86B00898009091
:10BE6000099801900A980290201CFFF7CBFE201C35
:10BE700006B010BDF0B58FB004AF3D6C7860281CE3
:10BE80006C30BA61FB613960FFF752FB031C2C3345
:10BE9000BB60EB6896B07B614A237A69041C1A4048
:10BEA000002304AEFB603A61131E402B04D0083B14
:10BEB0005A1E9341DBB2FB60301CFB68503000938C
:10BEC000BA687B69B96CFFF742F8142378621B1AD1
:10BED000227C9B00F318002A14D06A46C000103060
:10BEE000121A9546182202930C23BA18D31806AEDC
:10BEF000009501960393A36A3868A168E268FFF78A
:10BF000011F8331CFA68002A0FD17A6992050CD512
:10BF1000BA6C002A09D03A69181F796A402A1AD1E6
:10BF2000E36B01310360031C7962AC68796A8C426F
:10BF30001FDD6846A2000E32D208D200821A954652
:10BF400004AE00940191281C796C321CFFF7FAFDB5
:10BF50007C62331C0DE07A69BE685204D20F023253
:10BF600092009259083B0260E26B02311A607962DA
:10BF7000DBE70022AA607A6A00927868B969FA69F8
:10BF8000FFF704FBBD4678680BB0F0BD10B5041C8C
:10BF900086B008980090099801900A980290201C99
:10BFA000FFF768FF201C06B010BD0000F0B58BB095
:10BFB000109E05930793F368944604930692104BE2
:10BFC000049A051C1340822292001343F360119BD4
:10BFD00008AF0193129B381C02936246059B0096A2
:10BFE000FFF748FF089B06AC06933B79281C23719A
:10BFF000049BF3602B1C06CC06C30BB0F0BDC046FF
:10C00000B5BFFFFFF0B58FB004AF3E6C7860301C59
:10C010006C30BA61FB613960FFF78AFA031C2C337C
:10C02000FB60F368AAB07B6104ABBB604A237A690A
:10C03000041C1A403A61402A01D0082A01D1002587
:10C0400003E0FB6C002B03DD0125BA6CFB6C07E001
:10C05000002B61D0B86CF96C0125002342428B4162
:10C06000F968B86800917969A03001910295FEF7EE
:10C07000A7FF2823BA681B1A78629B00D318227C7A
:10C08000002A16D06A46C0001030121A954606AA39
:10C09000BA600096BA680293019218220C23BA186B
:10C0A000D3180393A36A3868A168E268FEF73AFFE1
:10C0B000BB687A6A002D09D0F96C002903DB796925
:10C0C00009052DD412E0043BE16A2BE0796989056A
:10C0D0000CD5B96CF86C014308D03969181F402998
:10C0E00024D1E36B01320360031C7A62B468796A7D
:10C0F0008C4228DD6846A2000E32D208D200821A95
:10C10000954604AD00940191301C796C2A1CFFF710
:10C1100019FD7C622B1C16E0BB6C002B94D199E7B7
:10C12000216B043B196001327A62DFE77969FD68AF
:10C130004904C90F023189004959083B0160E16B8C
:10C1400002321960F0E70022B2607A6A00927868E1
:10C15000B969FA69FFF71AFABD4678680BB0F0BD05
:10C1600070B5041C86B00A980C9D0D9E00900B982B
:10C17000029503960190201CFFF744FF201C06B097
:10C1800070BDF0B591B004AFBD6CF860281C7B6247
:10C190003B6D6C30BB607B6D3A627B603960FFF752
:10C1A000C7F9031C2C333B61EB68AAB0FB614A233F
:10C1B000FA69041C1A40002304AE7B61BA61131EA5
:10C1C000402B04D0083B5A1E9341DBB27B61301CEC
:10C1D0003B69A0300093FB6901937B690293BA68C5
:10C1E0007B68FEF7EDFE2823F8621B1A227C9B0079
:10C1F000F318002A14D06A46C0001030121A95466F
:10C20000202202930C23BA18D31806AE009501968B
:10C210000393A36A3868A168E268FEF783FE331CC3
:10C220007A69002A10D1FA6992050DD5BA68796841
:10C230000A4309D0BA69181FF96A402A1AD1E36B78
:10C2400001310360031CF962AC68F96A8C421FDD9E
:10C250006846A2000E32D208D200821A954604AE79
:10C2600000940191281CF96C321CFFF76BFCFC62F6
:10C27000331C0DE0FA693E695204D20F023292007B
:10C280009259083B0260E26B02311A60F962DBE707
:10C290000022AA60FA6A0092F868396A7A6AFFF79F
:10C2A00075F9BD46F8680DB0F0BD70B5041C86B0D8
:10C2B0000A980C9D0D9E00900B9802950396019094
:10C2C000201CFFF75EFF201C06B070BDF0B591B0DA
:10C2D00004AF3A6110227B614023BA18D3181E784C
:10C2E000BB6C78606C33181CFB603960FFF720F979
:10C2F000BB6C051C5B680624002B00DB1C1C102398
:10C30000FA18D118B86C321CFDF702FBBB6CDB6865
:10C31000BB60231CBA681E33520701D51B33FF33A1
:10C320006A460E33DB08DB00D31A9D46FDF7E4F8BE
:10C330001022F8610094BB6DFC6D029303940C23F2
:10C34000BA18D018043304AEFC18E318311C0022CC
:10C35000FEF7F2F9B861F868FEF734FC6946BA698D
:10C3600093000E33DB08DB00CB1A9D4604ACB218F9
:10C37000311C231CFEF771FEBB69301C1A1C2E21D8
:10C38000FB6018F0E9F8021E04D0801B80006B6A85
:10C39000221813602B7C002B38D0002A0BD1FB68AD
:10C3A000022B08DD7178392930D8B3782F292DD99F
:10C3B000303B092B2AD86946FB68DB000833CB1ACF
:10C3C0009D46FD2104ABBB60337800262B3B0B421E
:10C3D00006D1BB68216801361960FB68013BBB616F
:10C3E0000092BA68B300D21801921022E418082310
:10C3F000BA18D31802940393AB6A3868A968EA683C
:10C40000FEF76BFDBB69BC689E19BE61BB6CBA6967
:10C410009D68954211DD6946AB000E33DB08DB00F9
:10C42000CB1A9D4604AE231C341C01920095B86CB7
:10C43000F96C321CFFF786FBBD610023BA6C936078
:10C44000BB690093786839697A69231CFFF79EF805
:10C45000BD4678680DB0F0BD70B588B0041C0E9D67
:10C460000F9E0C980495059600900D980190002061
:10C470000290201CFFF72AFF201C08B070BDF0B509
:10C4800091B004AF3A6110227B614023BA18D318EF
:10C490001E78BB6C78606C33181CFB603960FFF74A
:10C4A00047F8BB6C051C5B680624002B00DB1C1CDA
:10C4B0001023FA18D118B86C321CFDF729FABB6C9E
:10C4C000DB68BB60231CBA681E33520701D51B33DF
:10C4D000FF336A460E33DB08DB00D31A9D46FDF7B7
:10C4E0000BF81022F8610094BB6DFC6D029303946D
:10C4F0000C23BA18D018043304AEFC18E318311C0E
:10C500000022FEF719F9B861F868FEF75BFB69468F
:10C51000BA6993000E33DB08DB00CB1A9D4604ACEE
:10C52000B218311C231CFEF798FDBB69301C1A1C85
:10C530002E21FB6018F010F8021E04D0801B800032
:10C540006B6A221813602B7C002B38D0002A0BD189
:10C55000FB68022B08DD7178392930D8B3782F2990
:10C560002DD9303B092B2AD86946FB68DB000833FC
:10C57000CB1A9D46FD2104ABBB60337800262B3BD4
:10C580000B4206D1BB68216801361960FB68013B8C
:10C59000BB610092BA68B300D21801921022E4186D
:10C5A0000823BA18D31802940393AB6A3868A968B1
:10C5B000EA68FEF792FCBB69BC689E19BE61BB6C61
:10C5C000BA699D68954211DD6946AB000E33DB0800
:10C5D000DB00CB1A9D4604AE231C341C019200954F
:10C5E000B86CF96C321CFFF7ADFABD610023BA6C70
:10C5F0009360BB690093786839697A69231CFEF7F8
:10C60000C5FFBD4678680DB0F0BD70B588B0041C9C
:10C610000E9D0F9E0C980495059600900D98019024
:10C620004C200290201CFFF72AFF201C08B070BD90
:10C63000F0B51C4C061CA544909C05936C3493AB40
:10C640001F78201C94AB04921D78FEF7BBFA039070
:10C65000201CFEF777FB2521041C0398FFF76DFAD9
:10C660000690002D02D10797089503E00023079557
:10C6700008970993929B0AA90093201C06AB80227D
:10C680000AF0F8FD0AA81BF0F9FA04990090059A3F
:10C69000301C0AABFEF77AFF301C8B239B009D44B5
:10C6A000F0BDC046D4FDFFFF026810B5002A0ED0D1
:10C6B0004368591C0DD1041C101C09F03DF9031CE2
:10C6C000421C01D0606004E00022226001E00123EE
:10C6D0005B42181C10BD38B50D1CFFF7E5FF041CAC
:10C6E000281CFFF7E1FF01340130634263414442FB
:10C6F0006041181A44426041C0B238BD08B5FFF726
:10C70000EAFF01235840C0B208BDF0B585B00090E3
:10C71000109803936C300292119FFEF753FA0F9B0F
:10C7200001900A25022B04D0093D042B01D1FA25E2
:10C73000AD000024261C02A80AA9FFF7DFFF0F9B0B
:10C74000002802D09E4203D11CE09E4214D119E081
:10C7500002A8FFF7A9FF2A22011C0198FFF7E8F9B8
:10C760003038C3B2092B07D80A212B1C4C4324189C
:10C7700063430E9A93420DDD0F9B042B05D1022ECD
:10C7800003D1643C0C9B1C6011E004233A68134302
:10C790003B600CE00D9A5B199A42EDDA281C13F00D
:10C7A00035FF051C02A8FEF7E5FE0136C3E7009A37
:10C7B00002AB03CB03C2009805B0F0BDF0B589B061
:10C7C00000AFB860F86CBA616C30FB61FEF7FAF943
:10C7D0006A46BB6C051C9B000E33DB08DB00D31ADA
:10C7E0009D463B611823F8180833C118FFF786FFF0
:10C7F000002803D1061C00237B6155E01823002488
:10C80000F818FFF751FF261C7861BB6C9C42F2D0F0
:10C810007A6CA300D35819687B698B4200D180E001
:10C820002B68281C9B6998477B69834279D0013427
:10C83000EBE73A69A300D3587A6C9B0098581BF039
:10C840001DFA854200D9051C0134B442F1D11823E8
:10C85000F818FEF78FFE7B6901337B61AB4265D22E
:10C860001823F8180833C118FFF748FF00285DD0D7
:10C8700000257B699B00FB603B69AC001C192368A9
:10C880007A6C9B009B58FA689B587B601823F818B9
:10C89000FFF70AFF7B68834213D0013E3A69B30079
:10C8A0009B582360B542E7D3012E0CD93B697A6CC3
:10C8B0001B680124FB609B0098581BF0DFF9051CE6
:10C8C000B7E70135EEE7012E30D11823F818FEF74F
:10C8D00051FE7B697A6C5D1C3B691B68FB609B00A9
:10C8E0009C58201C1BF0CAF97B6938619E00A41972
:10C8F0003B699D4223D21823F8180833C118FFF76B
:10C90000FDFE00281BD01823F8186668FFF7CCFE40
:10C910000434864213D11823F818FEF72BFE013594
:10C92000E6E73A69B3009C50013680E73B6D1B682F
:10C930007B6104237A6913433A6D136005E03B6918
:10C94000AB42F3D13B6CFA681A601823BD46BA6853
:10C95000FB1803CB03C2B86809B0F0BDF0B58BB0CB
:10C9600000AFF860786D3A626C307B62FEF72AF9AE
:10C970006A463B6D051CDB000833D31A9D46FB61FC
:10C980002023F818C118FFF7B9FE002803D10026AC
:10C99000351C341C3EE020230024F818FFF784FEE9
:10C9A000261C3B6DB8615B007B617B699C4211D0AA
:10C9B000FA6CA300D3581968BB698B4200D191E08F
:10C9C0002B68281C9B699847BB69834200D189E08A
:10C9D0000134EAE7002EDAD02023F818FEF7CAFD6A
:10C9E0006A46B3000E33DB08DB00D31A9D460025F0
:10C9F0006C46AB00BB61BA69FB6901359B58FA6CA8
:10CA00007B619B0098581BF039F9BB69E050B54237
:10CA1000EFD10125AB00BB612023F818C118FFF747
:10CA20006DFE002839D02023F818FFF73DFE0023C3
:10CA3000B8607B61B34224D2F8699A00844694447A
:10CA400060460068F96CA2188000405811683A618D
:10CA50008D4203D37A6901327A6110E0B969405896
:10CA6000B96888420BD0013EF969B0000958796075
:10CA700061467A680A60225839690A60DAE7013348
:10CA8000D8E7BB690433BB617B69B34205D020237F
:10CA9000F818FEF76FFD0135BEE7012E01D12368BE
:10CAA00005E0022E0DD12368AB4202D06368AB4291
:10CAB00007D1FB693A6D1B68934200D39B1ABA6C8D
:10CAC00006E0BB6D1B68FB610423FA691343BA6D72
:10CAD00013602023BD46FA68FB1803CB03C2F86835
:10CAE0000BB0F0BDFA69B3009C50013670E700004E
:10CAF000F0B5A1B0289C0D906C34201C0F1C109236
:10CB00001193FEF71FF90990201CFEF75BF80890BF
:10CB10002B981BF0B3F800240C90129410AD281C35
:10CB200026A9FFF7EBFD129B0A93002800D15CE2D7
:10CB30000C9B9C4200D358E20A9B002B00D054E28D
:10CB40002B9BA6009E19089831680A9AFEF7F0FF01
:10CB5000252800D005E2631C089871680A9A0B9397
:10CB6000FEF7E6FF0A9B1393452801D04F2806D114
:10CB7000A31C0898B16800220B93FEF7D9FF413837
:10CB8000382800D9E7E110AC13F0A6FC3F006100A3
:10CB90007C01C200E501E501E501C700D500E50122
:10CBA000E501E5010501E501E501E501E5012201F8
:10CBB00037015901E501E501E50163017C01A201AD
:10CBC000E501E501E501E501E501E50139005B006D
:10CBD000720077008500E501E5015B00E501E501F4
:10CBE000E501E501E3001301E501E501E501E501EA
:10CBF000E5014D01E501E501E5015E017C0114AEB1
:10CC00000998311CFDF751FF04E014AE0998311C5E
:10CC1000FDF735FF6B4626AA03CA03C32A9B10AD56
:10CC20001833029307230EAC03960493289B201C11
:10CC3000059312AB0693391C109A119BFFF7BEFDAA
:10CC4000D0E114AE0998311CFDF76FFF04E014AE7B
:10CC50000998311CFDF73FFF6B4626AA03CA03C3A0
:10CC60002A9B10AD103302930EAC03960C23DCE725
:10CC7000099814A9FDF7FCFEEFE06B4626AA03CA4B
:10CC800003C32A9B0EAD0C330293012303931E337F
:10CC900004931D3BBDE0201CFFF706FD0821021C8C
:10CCA0000898FCF730FE0EAD00281CD0201CFEF7C3
:10CCB00061FC6A4626A9031C41C941C209212A9A7E
:10CCC00004910C3202920122281C391C0392059215
:10CCD000289A069212AA07921A685B68FFF715FD58
:10CCE0000CCD0CC43BE16B4626AA03CA03C32A9BA6
:10CCF000281C0C3302930A230393153304931D3B22
:10CD00000593289B391C069312AB0793226888E091
:10CD100014AE0898BF49C04A5EE06B4626AA03CA13
:10CD200003C32A9B0EAD08330293002303931733EA
:10CD30000493153B6DE06B4626AA03CA03C32A9BE6
:10CD40000EAD08330293012303930B3304930A3B84
:10CD50005FE06B4626AA03CA03C313AB0293012309
:10CD600003930B3304930A3B0593289B0EAD069364
:10CD700012AB07936368281C109A391CFFF7C5FC97
:10CD80000CCD0CC4129B002B00D0E8E0139B2A9A18
:10CD9000013B1361E3E06B4626AA03CA03C32A9B47
:10CDA0000EAD04330293002303933B330493393BCA
:10CDB0002FE0201CFFF778FC0022011C0898FEF7EA
:10CDC000B7FE0A2800D0C6E010A8FEF7D3FBC6E0E5
:10CDD00008989249924A14AE331CFEF73EF96B460E
:10CDE00026AA03CA03C3289B10AD029312AB039378
:10CDF0002A9B0EAC049305963DE06B4626AA03CA17
:10CE000003C32A9B0EAD0293002303933D33049387
:10CE10003B3B281C391C0593289B109A069312ABA8
:10CE2000079363685AE7201CFFF73EFC0022011CB1
:10CE30000898FEF77DFE092800D08CE0C4E714AE08
:10CE400008987849784AC7E7099814A9FDF702FEBF
:10CE500003E0099814A9FDF704FE6B4626AA03CA4D
:10CE600003C3289B10AD029312AB03932A9B0EAC15
:10CE70000493149B0593201C391C109A119BFFF7F7
:10CE800037FEAFE06B4626AA03CA03C313AB029377
:10CE900000230393654B0EAD049304230593289B55
:10CEA000281C069312AB07936368109A391CFFF78E
:10CEB0002CFC0CCD0CC4129B002B50D1139B5C4A54
:10CEC0009A18002B01DA64331A1C2A9B5A6146E037
:10CED000201CFFF7E9FB0121021C0898FCF713FD59
:10CEE000002838D06B4626AA03CA03C314AB0293AA
:10CEF000504B0EAD03930E230493289B281C0593DF
:10CF000012AB0693391C22686368FFF757FC231C99
:10CF1000201C06CD06C326A9FFF7F0FB00281ED073
:10CF2000129B002B1BD1149B002B18D1201CFFF748
:10CF3000BBFB2D21051C0898FEF7FFFD854220D084
:10CF4000201CFFF7B1FB2B21041C0898FEF7F5FD10
:10CF5000844204D115E00423129A134312930B9CCC
:10CF60000DE0281C3668FFF79FFB864203D1281C82
:10CF7000FEF700FB03E00423129A134312930134DB
:10CF8000CCE56B4626AA03CA03C314AB0293002365
:10CF90000226039317330493289B0EAC069312AB1F
:10CFA000201C391C0793109A119B10AD0596FFF7B2
:10CFB000ACFB2B1C221C03CA03C36B4626AA03CA64
:10CFC00003C314AB0293002303933B330493289BC6
:10CFD0000596069312AB0793201C391C0E9A6368C2
:10CFE000FFF793FB0CCC0CC5B9E70A9B002B02D1D1
:10CFF0000C9B9C4207D0299B1B6808930423089A2A
:10D000001343299A13600D9B06CD06C30D9821B0DA
:10D01000F0BDC046DCD30200E5D30200E5D3020038
:10D02000EBD30200EBD30200F4D302000F27000081
:10D0300094F8FFFF70000020F0B58FB0051C169823
:10D040000AAC6C300A9263600791179EFDF77AFE76
:10D050000CA9FDF706FD6B4614AA03CA03C3169B71
:10D0600008AF0293189B039604930C9B381C0593FE
:10D0700007990A9A6368FFF73BFD231C201C06CF23
:10D0800006C314A9FFF727FB002803D00223326848
:10D09000134333602B1C281C06CC06C30FB0F0BD15
:10D0A000F0B58FB0051C16980AAC6C300A9263601C
:10D0B0000791179EFDF746FE0CA9FDF7CBFC6B46CA
:10D0C00014AA03CA03C3169B08AF0293189B0396C6
:10D0D00004930C9B381C059307990A9A6368FFF721
:10D0E00007FD231C201C06CF06C314A9FFF7F3FA83
:10D0F000002803D002233268134333602B1C281C02
:10D1000006CC06C30FB0F0BDF0B59FB0269F0CACA7
:10D110006C37061C381C0C9263600991279DFDF743
:10D1200011FE0890381C10AFFDF74CFD0898391C13
:10D13000FDF7BBFC089817A9FDF7A1FC00230F938E
:10D140006B4624AA03CA03C30EAB029307230493BE
:10D15000269B039705930FAB06930AA809990C9A8F
:10D160006368FFF7FBFB231C0AAA03CA03C30F9BD8
:10D17000002B03D1289B0E9A9A6103E004232A68AE
:10D1800013432B60201C24A9FFF7A5FA002803D025
:10D1900002232A6813432B60331C301C06CC06C3C1
:10D1A0001FB0F0BDF0B5A9B0309F0CAC6C37061CB9
:10D1B000381C0C9263600991319DFDF7C3FD089006
:10D1C000381C10AFFDF7FEFC0898391CFDF7ADFCCC
:10D1D00008981CA9FDF77FFC00230F936B462EAA2D
:10D1E00003CA03C30EAB02930C230493309B039733
:10D1F00005930FAB06930AA809990C9A6368FFF789
:10D20000ADFB231C0AAA03CA03C30F9B002B03D147
:10D21000329B0E9A1A6103E004232A6813432B60A1
:10D22000201C2EA9FFF757FA002803D002232A68F2
:10D2300013432B60331C301C06CC06C329B0F0BD51
:10D24000F0B591B0051C18980CAC6C3009910C929B
:10D250006360199EFDF7B6FC00236A460F9316A97A
:10D2600081C981C204270393194B0EAA0493189B0A
:10D27000029206930FAB059707930AA809990C9A97
:10D280006368FFF742FA231C0AAA03CA03C30F9B71
:10D29000002B09D10E9B0F4A9A18002B01DA643338
:10D2A0001A1C1A9B5A6102E033683B433360201C0E
:10D2B00016A9FFF710FA002803D00223326813439F
:10D2C00033602B1C281C06CC06C311B0F0BDC04631
:10D2D0000F27000094F8FFFFF0B593B01A9C099057
:10D2E0006C34201C0D930C921B9FFDF76BFC089077
:10D2F000201CFDF779FF031C40330A93002306939B
:10D30000836A041C002B04D0036B5A1E9341DBB2CA
:10D310000693C04B0F93237C002B03D00FA8202132
:10D3200008F046FFBB4B10A82021109308F040FFE7
:10D33000231C002644330B93E36B0496119307964A
:10D3400001960296039611ABF05C042800D95FE1C8
:10D3500013F0B8F8AD9803325C001A9BDB680593B4
:10D360009B0500D54CE1039B012B00D948E1002E21
:10D3700000D145E1012E0ED1069B002B00D03FE1EC
:10D3800011AB1A78032A00D13AE19B78012B00D126
:10D3900036E10136D7E70125022E00D0BFE011AB00
:10D3A000DB78042B00D12BE1069A002A00D195E00E
:10D3B000032B00D092E023E1A36A002B00D12DE1E2
:10D3C0000CA818A9FFF79AF9002800D126E10CA8AB
:10D3D000FFF76AF9636A1B68984200D01EE1A36AEE
:10D3E0000CA80393FEF7C6F812E163699D422AD1A7
:10D3F000049B002B27D1636B002B38DD019B019030
:10D400000793012304930CA8FEF7B4F80CA818A9FD
:10D41000FFF774F900282AD00CA8FFF745F9051C7E
:10D420000A220B98291C1AF0A9FD0028DDD00A9BBE
:10D43000C01A794B80101B68195C10A808F091FF86
:10D44000019B013311E0237C002B10D0A3699D4286
:10D450000DD1049B002B0AD1019B002B09D06B46F8
:10D460000FA8197908F07DFF049B0193CBE70125F4
:10D4700000E0019D109B0C3B1B685A1E93415B42D0
:10D480001D404CE00CA818A9FFF738F9002800D17E
:10D49000E9E00CA8FFF708F90821021C0898FCF73E
:10D4A00032FA002800D1DEE00CA8FEF763F801256F
:10D4B000032E3BD00CA818A9FFF720F900282ED086
:10D4C0000CA8FFF7F1F80821021C0898FCF71BFADA
:10D4D000002824D00CA8FEF74DF8EBE7032632E72E
:10D4E000AB4200D194E00CA8FFF7DEF8059BE2699F
:10D4F0009B009B5898420ED10CA8FEF73BF8059B69
:10D5000001330CA818A90593FFF7F8F8059B00282C
:10D51000E6D1AB427CD00025059BAB4273D00136EF
:10D52000042E03D0002D00D00DE7AAE0039B012BB1
:10D5300020D9002D00D1A4E0029B002B01D0E66A87
:10D5400000E0666A01250CA818A9FFF7D7F8039B2D
:10D55000002800D189E09D420FD00CA8FFF7A4F865
:10D56000AB00F358984200D08BE00CA8FEF702F80D
:10D570000135E8E7002D00D183E0109B0C3B1B68D0
:10D58000012B11D910A83021002208F035FC002809
:10D590000AD0021C431C03D1109B0C3B1A68013AB1
:10D5A00010A8002108F02CFD029B002B06D010A82B
:10D5B00008F00EFD109B1B78302B59D10F9B0C3BB4
:10D5C0001B68002B14D06B461979049B002B01D0EB
:10D5D0006B46197F0FA808F0C4FEA068E1680FAA87
:10D5E000FCF7C7F9002803D104233A6813433B60D2
:10D5F000049B002B55D0636B019A9A4241D150E0B5
:10D60000256A00237DE71A9BDB6805939B0586D47A
:10D61000012584E7E01E0020AC000020236B002BD6
:10D6200015D00CA818A9FFF769F800280FD00CA88E
:10D63000FFF73AF8E36A1B68984208D1236B0CA8FD
:10D640000393FDF797FF012302931D1C67E7A36A6D
:10D650000125002B02D0236B002B02D0069B5D40DE
:10D660005DE702955BE7002522E79D4209D184E74B
:10D6700010A808F0B6FC2D22011C10A808F014FD1B
:10D680009CE704233A6813433B600CAC201C18A9A8
:10D69000FFF721F8002809D002233A6813433B60C2
:10D6A00004E01C9810A908F093FBEEE7099B10A872
:10D6B00006CC06C308F01CFC0FA808F019FC09985A
:10D6C00013B0F0BDF0B593B01A9C09906C34201CD7
:10D6D0000D930C921B9FFDF775FA0890201CFDF727
:10D6E00067FE031C40330A9300230693836A041CDD
:10D6F000002B04D0036B5A1E9341DBB20693C04B40
:10D700000F93237C002B03D00FA8202108F050FD9D
:10D71000BB4B10A82021109308F04AFD231C0026C3
:10D7200044330B93E36B049611930796019602968C
:10D73000039611ABF05C042800D95FE112F0C2FE41
:10D74000AD9803325C001A9BDB6805939B0500D5FE
:10D750004CE1039B012B00D948E1002E00D145E1AB
:10D76000012E0ED1069B002B00D03FE111AB1A78A1
:10D77000032A00D13AE19B78012B00D136E1013632
:10D78000D7E70125022E00D0BFE011ABDB78042BD8
:10D7900000D12BE1069A002A00D195E0032B00D09E
:10D7A00092E023E1A36A002B00D12DE10CA818A977
:10D7B000FEF7A4FF002800D126E10CA8FEF774FFB5
:10D7C000636A1B68984200D01EE1A36A0CA8039309
:10D7D000FDF7D0FE12E163699D422AD1049B002B24
:10D7E00027D1636B002B38DD019B01900793012348
:10D7F00004930CA8FDF7BEFE0CA818A9FEF77EFF47
:10D8000000282AD00CA8FEF74FFF051C0A220B980F
:10D81000291C1AF0B3FB0028DDD00A9BC01A794BF3
:10D8200080101B68195C10A808F09BFD019B013358
:10D8300011E0237C002B10D0A3699D420DD1049BE5
:10D84000002B0AD1019B002B09D06B460FA8197938
:10D8500008F087FD049B0193CBE7012500E0019DC3
:10D86000109B0C3B1B685A1E93415B421D404CE0D1
:10D870000CA818A9FEF742FF002800D1E9E00CA887
:10D88000FEF712FF0821021C0898FCF73CF800285C
:10D8900000D1DEE00CA8FDF76DFE0125032E3BD084
:10D8A0000CA818A9FEF72AFF00282ED00CA8FEF716
:10D8B000FBFE0821021C0898FCF725F8002824D05C
:10D8C0000CA8FDF757FEEBE7032632E7AB4200D189
:10D8D00094E00CA8FEF7E8FE059BE2699B009B58CC
:10D8E00098420ED10CA8FDF745FE059B01330CA80C
:10D8F00018A90593FEF702FF059B0028E6D1AB426D
:10D900007CD00025059BAB4273D00136042E03D09A
:10D91000002D00D00DE7AAE0039B012B20D9002D9C
:10D9200000D1A4E0029B002B01D0E66A00E0666A09
:10D9300001250CA818A9FEF7E1FE039B002800D1E1
:10D9400089E09D420FD00CA8FEF7AEFEAB00F35865
:10D95000984200D08BE00CA8FDF70CFE0135E8E7FB
:10D96000002D00D183E0109B0C3B1B68012B11D9CB
:10D9700010A83021002208F03FFA00280AD0021C2B
:10D98000431C03D1109B0C3B1A68013A10A80021DC
:10D9900008F036FB029B002B06D010A808F018FBFD
:10D9A000109B1B78302B59D10F9B0C3B1B68002B15
:10D9B00014D06B461979049B002B01D06B46197F5C
:10D9C0000FA808F0CEFCA068E1680FAAFBF7D1FF12
:10D9D000002803D104233A6813433B60049B002BC7
:10D9E00055D0636B019A9A4241D150E0256A0023D9
:10D9F0007DE71A9BDB6805939B0586D4012584E7A8
:10DA0000E01E0020AC000020236B002B15D00CA8DA
:10DA100018A9FEF773FE00280FD00CA8FEF744FEED
:10DA2000E36A1B68984208D1236B0CA80393FDF7A7
:10DA3000A1FD012302931D1C67E7A36A0125002BAA
:10DA400002D0236B002B02D0069B5D405DE7029560
:10DA50005BE7002522E79D4209D184E710A808F082
:10DA6000C0FA2D22011C10A808F01EFB9CE704231D
:10DA70003A6813433B600CAC201C18A9FEF72BFE40
:10DA8000002809D002233A6813433B6004E01C9845
:10DA900010A908F09DF9EEE7099B10A806CC06C373
:10DAA00008F026FA0FA808F023FA099813B0F0BD81
:10DAB000F0B58DB008AC636014AB061C08921E482C
:10DAC0001A788C460AAF0A9006AD002A0FD06A4633
:10DAD00012A80AC80AC2159B04970293169B281C19
:10DAE00003936146089A6368FFF7ECFD0EE06A460F
:10DAF00012A80AC80AC2159B04970293169B281CF9
:10DB000003936146089A6368FFF7E6FB231C06CD82
:10DB100006C30A9DFBF7F0FC1799169A0B900BAB06
:10DB2000281C09F065F8331C381C06CC06C308F025
:10DB3000DFF9301C0DB0F0BDE01E0020F0B58FB055
:10DB40000AAD6B60061C16AB17981B786C300A92F6
:10DB50000F1C0793FDF736F8244A06900D92079A9A
:10DB600008AC002A10D06A4614A909C909C2179A3C
:10DB70000DAB0292189A04930392201C391C0A9A46
:10DB80006B68FFF79FFD0FE06A4614A909C909C237
:10DB9000179A0DAB0292189A04930392201C391C19
:10DBA0000A9A6B68FFF798FB0CCC0CC50D9B0C3BDD
:10DBB0001C68002C0FD0211C1998FBF7AFF90D9DA4
:10DBC0001998FBF705F8199B2C190698291C221C9B
:10DBD0001B68FDF742FA321C0AAB03CB03C20DA847
:10DBE00008F086F9301C0FB0F0BDC046E01E0020E2
:10DBF000F0B58BB00590129806926C300793FDF744
:10DC000097FC10A9051C06A8FEF765FD00240190ED
:10DC1000A04230D106A8FEF747FD2B1CC0331B687D
:10DC2000041CC31A59425941CBB2002B04D12A1CFF
:10DC3000BC32126890421ED12A7C002A02D0AA6A05
:10DC4000944218D06A6A944215D02B21002B00D13F
:10DC50000231149808F085FB06A8FDF78BFC10A98B
:10DC6000FEF74CFD002804D006A8FEF71DFD041C9D
:10DC700001E00123019300270397019B002B27D18B
:10DC80002B7C002B02D0AB6A9C4221D06B6A9C4259
:10DC90001ED02B1CCC331B689C4219D1039B002B3C
:10DCA00003D11498302108F05CFB06A8FDF762FC54
:10DCB00010A90137FEF722FD002804D006A8FEF7C0
:10DCC000F3FC041C01E00123019301230393D4E737
:10DCD000A14B09932B7C002B03D009A8202108F02D
:10DCE00067FA92235B00EE5C002E01D1029631E0D0
:10DCF0002B1C0026CC330493029693E06B6A9C4263
:10DD00003AD02B1CFC339A68944241D1002E00D0AB
:10DD1000F9E0039B002B00D1F5E06521149808F091
:10DD200020FB06A8FDF726FC10A9FEF7E7FC00285B
:10DD300000D1E7E006A8FEF7B7FC2B1CC0331B6838
:10DD4000041E9C4228D02B1CBC331B6801362D219D
:10DD5000984222D0019B002B00D0D4E00A20211C45
:10DD6000FCF7CCFC431CC9D03030C1B2149808F089
:10DD7000F8FA0123039314E0029B002BC1D1002E7B
:10DD8000BFD114982E2108F0ECFA0123029308E089
:10DD90001B6A9C42BAD0B6E02B21149808F0E1FA35
:10DDA000012606A8FDF7E6FB10A9FEF7A7FC002850
:10DDB00004D006A8FEF778FC041CCBE701230193EE
:10DDC000C8E72B1CFC339A68944270D1002E00D017
:10DDD00099E0039B002B00D195E0099B0C3B1B684D
:10DDE000002B68D16521149808F0BBFA06A8FDF74E
:10DDF000C1FB10A9FEF782FC002800D182E006A832
:10DE0000FEF752FC2B1CC0331B68041CC31A59427A
:10DE10005941CBB2002B52D12A1CBC3212680126C8
:10DE200090424CD0019B002B6DD12B7C002B13D04A
:10DE3000AB6A9C4210D1029B002B64D1002E62D1B0
:10DE4000002F05D0F9B209A808F08BFA371C49E079
:10DE5000149808F0CCF856E06B6A9C4214D1029BEF
:10DE6000002B50D1002E4ED1099B0C3B1B68002B80
:10DE700003D0F9B209A808F074FA14982E2108F01A
:10DE800070FA012302932DE00498211C0A221AF053
:10DE900075F8002895D0049B0137C11A89103031DC
:10DEA000C9B2149808F05DFA012303931AE01B6AC3
:10DEB0009C428BD027E0029B002B3DD092E72A7C2E
:10DEC000002A03D0AA6A01269442ABD06A6A0126CE
:10DED0009442A7D02B21002B00D10231149808F0D6
:10DEE00040FA012606A8FDF745FB10A9FEF706FC3F
:10DEF000002804D006A8FEF7D7FB041C92E70123F4
:10DF000001938FE70126099B0C3B1B68002B18D05F
:10DF1000029B002B05D1002E03D1F9B209A808F00D
:10DF200020FAA868E96809AAFBF723FD002808D1B0
:10DF30000422139B1A6004E0F9B209A808F011FA50
:10DF400050E7059A06AB03CB03C209A807F0D0FF40
:10DF500005980BB0F0BDC046E01E0020F0B58FB0B4
:10DF60000AAC63600CAF1D4B0791051C2021381CC7
:10DF7000179E0A920C9308F01BF96B4614AA03CA69
:10DF800003C3169B039602930497079908A80A9A5D
:10DF90006368FFF72DFE231C08AA03CA03C30C9B6A
:10DFA0000793FBF7A9FA18990D90321C07980DAB4F
:10DFB00008F072FD201C14A9FEF78DFB002803D089
:10DFC00002233268134333602B1C381C06CC06C373
:10DFD00007F08EFF281C0FB0F0BDC046E01E0020E9
:10DFE000F0B58FB00AAC63600CAF1D4B0791051CF8
:10DFF0002021381C179E0A920C9308F0D9F86B4622
:10E0000014AA03CA03C3169B0396029304970799A5
:10E0100008A80A9A6368FFF7EBFD231C08AA03CA45
:10E0200003C30C9B0793FBF767FA18990D90321CFA
:10E0300007980DAB08F07EFD201C14A9FEF74BFBE2
:10E04000002803D002233268134333602B1C381C92
:10E0500006CC06C307F04CFF281C0FB0F0BDC0462D
:10E06000E01E0020F0B58FB00AAC63600CAF1D4B12
:10E070000791051C2021381C179E0A920C9308F06A
:10E0800097F86B4614AA03CA03C3169B0396029320
:10E090000497079908A80A9A6368FFF7A9FD231C4B
:10E0A00008AA03CA03C30C9B0793FBF725FA189928
:10E0B0000D90321C07980DAB08F09AFD201C14A996
:10E0C000FEF709FB002803D00223326813433360B4
:10E0D0002B1C381C06CC06C307F00AFF281C0FB007
:10E0E000F0BDC046E01E0020F0B58FB0169C099030
:10E0F000201C6C300B930A92FDF71AFA4A23E4684D
:10E10000061C1C40423B0093402C05D00233009378
:10E11000082C01D1063300930AA814A9FEF7DBFAF4
:10E120000290002828D10AA8FEF7BEFA331CBC339F
:10E130001B68071CC31A59425941CBB20493002BE8
:10E1400004D1331CC0331B6898421AD1337C002B96
:10E1500002D0B36A9F4214D0736A9F4211D00AA8BA
:10E16000FDF708FA14A9FEF7C9FA002807D00AA893
:10E17000FEF79AFA071C04E00027049701E0012348
:10E18000029300250195029B002B56D1337C002B76
:10E1900002D0B36A9F4250D0736A9F424DD0331C65
:10E1A000CC331B689F420DD1019B002B03D0009BF9
:10E1B0000A2B0AD127E0002C19D0009B082B1AD07B
:10E1C000013519E0019B002B37D0331CC4331B6889
:10E1D0009F4204D0331CC8331B689F422BD1002CB4
:10E1E0000DD0009B102B2ED10025019510E00123AE
:10E1F000251C01930AE0019D0123019308E0251CE1
:10E200000194102303E0002CDAD1251C082300938D
:10E210000AA8FDF7AFF914A9FEF770FA002807D095
:10E220000AA8FEF741FA019B071C002BABD104E0C2
:10E2300001230293A7E70123019316230593009B73
:10E24000102B02D103E001230193009B0593704B37
:10E250000D93337C002B03D00DA8202107F0A8FFDD
:10E260006C4A049B94466344181C0099069312F070
:10E270003DF9922307905B00F45C002C01D10394DC
:10E2800026E0331C0024CC330893039443E0059824
:10E29000391CFCF733FA431C69D0079B9C421BD8FE
:10E2A000009B039A5C43069B01351B1AA3429B41CA
:10E2B0005B421A43039204190AA8FDF75BF914A9FB
:10E2C000FEF71CFA00280AD00AA8FEF7EDF9071C91
:10E2D000029B002BDBD04AE001230393ECE70123F0
:10E2E0000293F5E7337C002B19D0B36A9F4216D115
:10E2F000002D3AD0E9B20DA808F033F8029D0AA823
:10E30000FDF738F914A9FEF7F9F900282AD00AA870
:10E31000FEF7CAF9071C029B002BE3D027E0736AC3
:10E320009F4224D00898391C059A19F027FE00282E
:10E330001FD0089BC01A80100F2800DD0638079BED
:10E340009C420CD8009B039A5C43069B01351B1A28
:10E35000A3429B415B421A4303920419CFE7012376
:10E360000393CCE701230293D5E7012702E00027BE
:10E3700000E0071C0D9B0C3B1B68002B0DD0E9B285
:10E380000DA807F0EEFFB068F1680DAAFBF7F1FAEF
:10E39000002802D10423179A1360002D07D1019B96
:10E3A000002B04D10D9B0C3B1B68002B01D0002FD0
:10E3B00006D00023189A13600423179A136008E00C
:10E3C000039B002B11D1049B002B00D06442189BAF
:10E3D0001C60029B002B10D0179B1B68009302232C
:10E3E000009A1343179A136007E0049B002B02D096
:10E3F00080231B06DEE7074BDCE7099A0AAB03CB59
:10E4000003C20DA807F074FD09980FB0F0BDC04617
:10E41000E01E0020FFFFFF7FF0B589B0041C6846B6
:10E420000EADC0CDC0C01098029011980390129804
:10E430000490201CFFF758FE201C09B0F0BDF0B579
:10E44000012493B00EAE73601A9B0B909C46DB6860
:10E4500007910E921B9D23422BD101235B42119306
:10E460006B4618AA03CA03C36346029311AB0CAFF1
:10E4700003950493381C07990E9A7368FFF734FECE
:10E48000331C06CF06C3119BA34203D81C401C9B20
:10E490001C70AFE01C9B301C1C70042318A92B605F
:10E4A000FEF719F9002800D1A4E002232A681343DB
:10E4B0009FE060466C30FDF73BF8036A061C5A4249
:10E4C0005341DBB20893836900275A425341DBB2C0
:10E4D00009930794089B002B45D10EA818A9FEF7B5
:10E4E000FAF8002844D10EA8FEF7DEF8089B002BAE
:10E4F00006D1F269BB009C58041B62426241D4B24F
:10E50000099B002C02D1002B02D04CE0002B62D1E1
:10E510007269BB009B58984205D0089B002B2BD1F9
:10E52000002C01D14FE0012307930EA87B1C0A9316
:10E53000FDF720F801230893002C06D000230A9A47
:10E54000316A8A425B41DBB2089301230993079B3E
:10E55000002B06D000230A9AB1698A425B41DBB2E4
:10E5600009930137B6E7099B002BB6D0002300E0E2
:10E570000123002C04D112E0002C24D000230793A7
:10E58000326A97420BD1002F09D000221C990A70E1
:10E59000079A002A13D0B269974210D128E0079A4F
:10E5A000002A11D003E0079B002B1DD0231CB26969
:10E5B000974209D1002F07D001221C990A705A1ED8
:10E5C00093415B0015E0231C00221C990A709342C2
:10E5D0000ED006230DE0079B002B9ED07B1C0EA8BF
:10E5E0000A93FCF7C7FFA9E76A461C9B127F1A70C3
:10E5F00004232B600B9A0EAB03CB03C20B9813B012
:10E60000F0BD0000F0B58FB0169C0990201C6C3056
:10E610000B930A92FCF78CFF4A23E468061C1C400B
:10E62000423B0193402C05D002330193082C01D1C9
:10E63000063301930AA814A9FEF74DF802900028AA
:10E6400028D10AA8FEF730F8331CBC331B68071C1E
:10E65000C31A59425941CBB20593002B04D1331C44
:10E66000C0331B6898421AD1337C002B02D0B36AA6
:10E670009F4214D0736A9F4211D00AA8FCF77AFF18
:10E6800014A9FEF73BF8002807D00AA8FEF70CF8FB
:10E69000071C04E00027059701E0012302930025F1
:10E6A0000395029B002B56D1337C002B02D0B36A1A
:10E6B0009F4250D0736A9F424DD0331CCC331B68AD
:10E6C0009F420DD1039B002B03D0019B0A2B0AD143
:10E6D00027E0002C19D0019B082B1AD0013519E036
:10E6E000039B002B37D0331CC4331B689F4204D0DC
:10E6F000331CC8331B689F422BD1002C0DD0019BCB
:10E70000102B2ED10025039510E00123251C039327
:10E710000AE0039D0123039308E0251C03941023C2
:10E7200003E0002CDAD1251C082301930AA8FCF78A
:10E7300021FF14A9FDF7E2FF002807D00AA8FDF782
:10E74000B3FF039B071C002BABD104E00123029312
:10E75000A7E70123039316230693019B102B02D1F5
:10E7600003E001230393019B0693724B0D93337CCB
:10E77000002B03D00DA8202107F01AFD6E48019947
:10E7800011F044FF83B2079392235B00F45C002CEA
:10E7900001D104942BE0331C0024CC33089304945F
:10E7A00048E00698391CFBF7A9FF431C72D0079B71
:10E7B0009C4220D8019B604A5C43A4B2121A0123F8
:10E7C000944201DC6B461B7A049A24181A43D3B294
:10E7D0000493A4B201350AA8FCF7CCFE14A9FDF7F6
:10E7E0008DFF00280AD00AA8FDF75EFF071C029BD8
:10E7F000002BD6D04EE001230493ECE701230293D3
:10E80000F5E7337C002B19D0B36A9F4216D1002D57
:10E810003ED0E9B20DA807F0A4FD029D0AA8FCF7BE
:10E82000A9FE14A9FDF76AFF00282ED00AA8FDF75B
:10E830003BFF071C029B002BE3D02BE0736A9F4237
:10E8400028D00898391C069A19F098FB002823D084
:10E85000089BC31A9B100F2B00DD063B079A9442BE
:10E8600010D8019A34495443A4B2C91A01228C42E7
:10E8700000DC00220499E4181143CAB20492A4B245
:10E880000135CBE701230493C8E701230293D1E7C5
:10E89000012702E0002700E0071C0D9B0C3B1B68D2
:10E8A000002B0DD0E9B20DA807F05BFDB068F16850
:10E8B0000DAAFBF75EF8002802D10423179A136013
:10E8C000002D07D1039B002B04D10D9B0C3B1B6833
:10E8D000002B01D0002F11D00023189A138004338D
:10E8E000179A1360029B002B19D0179B1B6801938A
:10E8F0000223019A1343179A136010E0049B002B24
:10E9000005D00123189A5B4213800533E8E7059B85
:10E91000002B01D06442A4B2189B1C80E2E7099A44
:10E920000AAB03CB03C20DA807F0E2FA09980FB0B7
:10E93000F0BDC046E01E0020FFFF0000F0B589B02A
:10E94000041C68460EADC0CDC0C01098029011984E
:10E95000039012980490201CFFF754FE201C09B06D
:10E96000F0BD0000F0B58FB0169C0990201C6C30F3
:10E970000B930A92FCF7DCFD4A23E468061C1C405A
:10E98000423B0193402C05D002330193082C01D166
:10E99000063301930AA814A9FDF79DFE03900028F1
:10E9A00028D10AA8FDF780FE331CBC331B68071C66
:10E9B000C31A59425941CBB20593002B04D1331CE1
:10E9C000C0331B6898421AD1337C002B02D0B36A43
:10E9D0009F4214D0736A9F4211D00AA8FCF7CAFD67
:10E9E00014A9FDF78BFE002807D00AA8FDF75CFEEE
:10E9F000071C04E00027059701E00123039300258D
:10EA00000295039B002B56D1337C002B02D0B36AB6
:10EA10009F4250D0736A9F424DD0331CCC331B6849
:10EA20009F420DD1029B002B03D0019B0A2B0AD1E0
:10EA300027E0002C19D0019B082B1AD0013519E0D2
:10EA4000029B002B37D0331CC4331B689F4204D079
:10EA5000331CC8331B689F422BD1002C0DD0019B67
:10EA6000102B2ED10025029510E00123251C0293C6
:10EA70000AE0029D0123029308E0251C0294102362
:10EA800003E0002CDAD1251C082301930AA8FCF727
:10EA900071FD14A9FDF732FE002807D00AA8FDF782
:10EAA00003FE029B071C002BABD104E00123039360
:10EAB000A7E70123029316230693019B102B02D193
:10EAC00003E001230293019B06936C4B0D93337C6F
:10EAD000002B03D00DA8202107F06AFB012001992B
:10EAE000404211F003FD922307905B00F45C002C80
:10EAF00001D1049425E0331C0024CC330893049402
:10EB000042E00698391CFBF7F9FD431C67D0079BD0
:10EB10009C421AD8019B049A5C43C343A3429B4185
:10EB20005B421A430492041901350AA8FCF722FD3E
:10EB300014A9FDF7E3FD00280AD00AA8FDF7B4FDEB
:10EB4000071C039B002BDCD049E001230493ECE776
:10EB500001230393F5E7337C002B19D0B36A9F425E
:10EB600016D1002D39D0E9B20DA807F0FAFB039DAC
:10EB70000AA8FCF7FFFC14A9FDF7C0FD002829D066
:10EB80000AA8FDF791FD071C039B002BE3D026E0AC
:10EB9000736A9F4223D00898391C069A19F0EEF93F
:10EBA00000281ED0089BC01A80100F2800DD0638F0
:10EBB000079B9C420BD8019B049A5C43C343A3422E
:10EBC0009B415B421A43049204190135D0E70123AB
:10EBD0000493CDE701230393D6E7012702E0002742
:10EBE00000E0071C0D9B0C3B1B68002B0DD0E9B20D
:10EBF0000DA807F0B6FBB068F1680DAAFAF7B9FEE8
:10EC0000002802D10423179A1360002D07D1029B1C
:10EC1000002B04D10D9B0C3B1B68002B01D0002F57
:10EC200011D00023189A13600433179A1360039BC2
:10EC3000002B18D0179B1B6801930223019A1343E2
:10EC4000179A13600FE0049B002B05D00123189A3C
:10EC50005B4213600533E8E7059B002B00D064425C
:10EC6000189B1C60E3E7099A0AAB03CB03C20DA80B
:10EC700007F03EF909980FB0F0BDC046E01E002035
:10EC8000F0B589B0041C68460EADC0CDC0C0109868
:10EC900002901198039012980490201CFFF762FED6
:10ECA000201C09B0F0BD0000F0B58FB0169C099093
:10ECB000201C6C300B930A92FCF73AFC4A23E46860
:10ECC000061C1C40423B0193402C05D002330193AB
:10ECD000082C01D1063301930AA814A9FDF7FBFC07
:10ECE0000390002828D10AA8FDF7DEFC331CBC33B2
:10ECF0001B68071CC31A59425941CBB20593002B1C
:10ED000004D1331CC0331B6898421AD1337C002BCA
:10ED100002D0B36A9F4214D0736A9F4211D00AA8EE
:10ED2000FCF728FC14A9FDF7E9FC002807D00AA885
:10ED3000FDF7BAFC071C04E00027059701E001235A
:10ED4000039300250295039B002B56D1337C002BA7
:10ED500002D0B36A9F4250D0736A9F424DD0331C99
:10ED6000CC331B689F420DD1029B002B03D0019B2B
:10ED70000A2B0AD127E0002C19D0019B082B1AD0AE
:10ED8000013519E0029B002B37D0331CC4331B68BC
:10ED90009F4204D0331CC8331B689F422BD1002CE8
:10EDA0000DD0019B102B2ED10025029510E00123E0
:10EDB000251C02930AE0029D0123029308E0251C12
:10EDC0000294102303E0002CDAD1251C08230193C0
:10EDD0000AA8FCF7CFFB14A9FDF790FC002807D088
:10EDE0000AA8FDF761FC029B071C002BABD104E0D5
:10EDF00001230393A7E70123029316230693019BA4
:10EE0000102B02D103E001230293019B06936C4B6C
:10EE10000D93337C002B03D00DA8202107F0C8F9F7
:10EE200001200199404211F061FB922307905B00A1
:10EE3000F45C002C01D1049425E0331C0024CC3375
:10EE40000893049442E00698391CFBF757FC431CD6
:10EE500067D0079B9C421AD8019B049A5C43C3432A
:10EE6000A3429B415B421A430492041901350AA84C
:10EE7000FCF780FB14A9FDF741FC00280AD00AA882
:10EE8000FDF712FC071C039B002BDCD049E001239B
:10EE90000493ECE701230393F5E7337C002B19D0AF
:10EEA000B36A9F4216D1002D39D0E9B20DA807F000
:10EEB00058FA039D0AA8FCF75DFB14A9FDF71EFC98
:10EEC000002829D00AA8FDF7EFFB071C039B002BA5
:10EED000E3D026E0736A9F4223D00898391C069A33
:10EEE00019F04CF800281ED0089BC01A80100F287B
:10EEF00000DD0638079B9C420BD8019B049A5C43BB
:10EF0000C343A3429B415B421A4304920419013557
:10EF1000D0E701230493CDE701230393D6E701272C
:10EF200002E0002700E0071C0D9B0C3B1B68002B38
:10EF30000DD0E9B20DA807F014FAB068F1680DAA77
:10EF4000FAF717FD002802D10423179A1360002D49
:10EF500007D1029B002B04D10D9B0C3B1B68002B9F
:10EF600001D0002F11D00023189A13600433179A90
:10EF70001360039B002B18D0179B1B68019302237F
:10EF8000019A1343179A13600FE0049B002B05D0DE
:10EF90000123189A5B4213600533E8E7059B002BB9
:10EFA00000D06442189B1C60E3E7099A0AAB03CBCC
:10EFB00003C20DA806F09CFF09980FB0F0BDC04633
:10EFC000E01E0020F0B589B0041C68460EADC0CD2F
:10EFD000C0C0109802901198039012980490201CC1
:10EFE000FFF762FE201C09B0F0BDF0B58FB0169E91
:10EFF0000793F76894460A920B933A1C4A239A4364
:10F00000131C08221343F3606B46069114AA051CD7
:10F0100003CA03C3179B08A803930DAB06990AAC58
:10F0200004936246079B0296FFF73EFE231C08AA44
:10F0300003CA03C3189B0D9AF7601A602B1C281C87
:10F0400006CC06C30FB0F0BDF0B597B01E9D109072
:10F05000281C6C3013931292FCF76AFA4A23ED686D
:10F06000041C1D40423B0093402D05D00233009309
:10F07000082D01D10633009312A81CA9FDF72BFB24
:10F080000490002828D112A8FDF70EFB231CBC33E6
:10F090001B68061CC31A59425941CBB20893002B76
:10F0A00004D1231CC0331B6898421AD1237C002B47
:10F0B00002D0A36A9E4214D0636A9E4211D012A865
:10F0C000FCF758FA1CA9FDF719FB002807D012A875
:10F0D000FDF7EAFA061C04E00026089601E0012389
:10F0E000049300270197049B002B56D1237C002B0F
:10F0F00002D0A36A9E4250D0636A9E424DD0231C28
:10F10000CC331B689E420DD1019B002B03D0009B8A
:10F110000A2B0AD127E0002D19D0009B082B1AD00A
:10F12000013719E0019B002B37D0231CC4331B6827
:10F130009E4204D0231CC8331B689E422BD1002D55
:10F140000DD0009B102B2ED10027019710E001233A
:10F150002F1C01930AE0019F0123019308E02F1C5B
:10F160000195102303E0002DDAD12F1C0823009312
:10F1700012A8FCF7FFF91CA9FDF7C0FA002807D078
:10F1800012A8FDF791FA019B061C002BABD104E0FD
:10F1900001230493A7E70123019316230E93009BF9
:10F1A000102B02D103E001230193009B0E93A34B8C
:10F1B0001593237C002B03D015A8202106F0F8FF1F
:10F1C000089B002B03D101229D4B524202E0802379
:10F1D00000221B060692079306980799009B009A47
:10F1E000DB170F9311F07CFB9223119009915B00C8
:10F1F000E35C002B05D100210022059302910392CC
:10F2000044E0231CCC330A93002200230292039390
:10F210000023059369E00E98311CFBF76FFA051C7B
:10F22000431C00D1AEE0039B099A93423ED831D0F3
:10F2300002980399009A0F9B11F072FBEB170A9545
:10F240000B9302900391069A079B0A980B99121A46
:10F250008B4103990125994221D902980399059B75
:10F2600001372B43DBB205930A9A0B9B12184B41D3
:10F270000292039312A8FCF77DF91CA9FDF73EFA50
:10F28000002816D012A8FDF70FFA061C049B002BCD
:10F29000C1D077E0029B119A934207D8C8E7994200
:10F2A00002D102999142D8D80025D6E701230593CF
:10F2B000E0E701230493E9E7237C002B19D0A36A3C
:10F2C0009E4216D1002F5BD0F9B215A807F049F87D
:10F2D000049F12A8FCF74EF91CA9FDF70FFA0028AD
:10F2E0004BD012A8FDF7E0F9061C049B002BE3D0DD
:10F2F00048E0636A9E4245D00A98311C0E9A18F085
:10F300003DFE002840D00A9BC51AAD100F2D00DD30
:10F31000063D039B099A93422CD803D1029B119A74
:10F32000934227D802980399009A0F9B11F0F8FA9C
:10F33000EB170C950D9302900391069A079B0C987E
:10F340000D99121A8B4103990125994204D802D1D3
:10F350000299914200D8002502980399059B013734
:10F360002B43DBB205930C9A0D9B12184B41029272
:10F370000393AEE701230593ABE701230493B4E7BE
:10F38000012502E0002500E0051C159B0C3B1B68D5
:10F39000002B0DD0F9B215A806F0E3FFA068E168D4
:10F3A00015AAFAF7E6FA002802D104231F9A13607F
:10F3B000002F07D1019B002B04D1159B0C3B1B6830
:10F3C000002B01D0002D08D00022002320990A60D4
:10F3D0004B6004231F9A13600FE0059B002B18D18C
:10F3E00002980399089B002B04D0031C0C1C0021DD
:10F3F0005842A141209B18605960049B002B13D0F8
:10F400001F9B1B6800930223009A13431F9A1360EB
:10F410000AE0089B002B03D0802300221B06D5E7BF
:10F420000122074B5242D1E7109A12AB03CB03C221
:10F4300015A806F05DFD109817B0F0BDE01E002085
:10F44000FFFFFF7FF0B589B0041C68460EADC0CD4C
:10F45000C0C0109802901198039012980490201C3C
:10F46000FFF7F2FD201C09B0F0BD0000F0B595B02B
:10F470001C9C0E90201C6C3011931092FCF758F8D5
:10F480004A23E768051C1F40423B0093402F05D0EC
:10F4900002330093082F01D10633009310A81AA954
:10F4A000FDF719F90490002828D110A8FDF7FCF801
:10F4B0002B1CBC331B68061CC31A59425941CBB2E2
:10F4C0000B93002B04D12B1CC0331B6898421AD11C
:10F4D0002B7C002B02D0AB6A9E4214D06B6A9E42FA
:10F4E00011D010A8FCF746F81AA9FDF707F9002873
:10F4F00007D010A8FDF7D8F8061C04E000260B96EC
:10F5000001E00123049300240194049B002B56D1B5
:10F510002B7C002B02D0AB6A9E4250D06B6A9E427D
:10F520004DD02B1CCC331B689E420DD1019B002B70
:10F5300003D0009B0A2B0AD127E0002F19D0009B93
:10F54000082B1AD0013419E0019B002B37D02B1C5B
:10F55000C4331B689E4204D02B1CC8331B689E42D8
:10F560002BD1002F0DD0009B102B2ED10024019405
:10F5700010E001233C1C01930AE0019C012301934C
:10F5800008E03C1C0197102303E0002FDAD13C1C5B
:10F590000823009310A8FBF7EDFF1AA9FDF7AEF8BA
:10F5A000002807D010A8FDF77FF8019B061C002B50
:10F5B000ABD104E001230493A7E7012301931623B1
:10F5C0000C93009B102B02D103E001230193009BBD
:10F5D0000C93914B13932B7C002B03D013A8202169
:10F5E00006F0E6FD009B01204042C117DB17009AA0
:10F5F0000D9311F075F992230F900A915B00EB5C6B
:10F60000002B05D1002100220593029103923CE0DA
:10F610002B1CCC3306930022002302920393002379
:10F62000059360E00C98311CFBF768F8071C431C3D
:10F6300000D19CE0039B0A9A934235D829D00298C6
:10F640000399009A0D9B11F06BF9FB170793079B29
:10F650000697DA43FF43012391421FD9059A0134EB
:10F660001A43D3B20593069A079B12184B41029294
:10F67000039310A8FBF77EFF1AA9FDF73FF80028B7
:10F6800015D010A8FDF710F8061C049B002BC9D05C
:10F690006DE0029B0F9A934206D8D0E7914201D1C8
:10F6A000B842DBD80023D9E701230593E1E7012322
:10F6B0000493EAE72B7C002B19D0AB6A9E4216D14B
:10F6C000002C52D0E1B213A806F04BFE049C10A807
:10F6D000FBF750FF1AA9FDF711F8002842D010A837
:10F6E000FCF7E2FF061C049B002BE3D03FE06B6AB3
:10F6F0009E423CD00698311C0C9A18F03FFC002822
:10F7000037D0069BC71ABF100F2F00DD063F039BA3
:10F710000A9A934223D803D1029B0F9A93421ED890
:10F7200002980399009A0D9B11F0FAF8FB170993C0
:10F73000099B0897DA43FF430123914203D801D183
:10F74000B84200D80023059A01341A43D3B2059376
:10F75000089A099B12184B4102920393B7E70123C1
:10F760000593B4E701230493BDE7012702E00027D6
:10F7700000E0071C139B0C3B1B68002B0DD0E1B273
:10F7800013A806F0EEFDA868E96813AAFAF7F1F8E5
:10F79000002802D104231D9A1360002C07D1019B7D
:10F7A000002B04D1139B0C3B1B68002B01D0002FB6
:10F7B00013D0002200231E990A604B6004231D9A77
:10F7C0001360049B002B1DD01D9B1B68009302231C
:10F7D000009A13431D9A136014E0059B002B03D07D
:10F7E00001225242D317E6E70B9B02980399002BA4
:10F7F00004D0031C0C1C00215842A1411E9B186020
:10F800005960DEE70E9A10AB03CB03C213A806F0D3
:10F810006FFB0E9815B0F0BDE01E0020F0B589B06A
:10F82000041C68460EADC0CDC0C01098029011985F
:10F83000039012980490201CFFF718FE201C09B0BA
:10F84000F0BD00000123244A1168194200D1136061
:10F85000224A1168194201D1012313600123204A71
:10F860001168194200D113601E4A1168194201D172
:10F870000123136001231C4A1168194200D113604F
:10F880001A4A1168194201D1012313600123184A51
:10F890001168194200D11360164A1168194201D14A
:10F8A000012313600123144A1168194200D1136027
:10F8B000124A1168194201D1012313600123104A31
:10F8C0001168194200D113600E4A1168194201D122
:10F8D000012313607047C046D0180020CC180020C8
:10F8E000C8180020C4180020C0180020BC18002030
:10F8F000B8180020B4180020B0180020AC18002060
:10F90000A8180020A41800208368587C70478368DA
:10F91000987C70478368D86A704713B58368FF2462
:10F920001B6B181C190A1A0C2140204009022240A6
:10F93000120408431B0E1B061043184316BD13B5D3
:10F940008368FF245B6B181C190A1A0C21402040A5
:10F9500009022240120408431B0E1B0610431843E1
:10F9600016BD8368587C70478368987C70478368AD
:10F97000D86A704713B58368FF241B6B181C190ADB
:10F980001A0C2140204009022240120408431B0E99
:10F990001B061043184316BD13B58368FF245B6B29
:10F9A000181C190A1A0C2140204009022240120496
:10F9B00008431B0E1B061043184316BD836805330E
:10F9C000D87F704783680633D87F70470020704720
:10F9D0000020704770470020914205D21923D8417A
:10F9E0000B7801311818F7E7704713B5041C8B68C2
:10F9F00001AA996806F00EFD201C16BD13B5041C63
:10FA00008B6801AA596906F005FD201C16BD13B5C7
:10FA1000041C8B6801AAD96906F0FCFC201C16BDE9
:10FA200013B5041C8B6801AA596A06F0F3FC201C6C
:10FA300016BD13B5041C8B6801AA996806F0EAFC90
:10FA4000201C16BD13B5041C8B6801AA596906F069
:10FA5000E1FC201C16BD13B5041C8B6801AAD969F2
:10FA600006F0D8FC201C16BD13B5041C8B6801AA37
:10FA7000596A06F0CFFC201C16BD13B5041C8B6818
:10FA800001AA996806F0C6FC201C16BD13B5041C1B
:10FA90008B6801AA596906F0BDFC201C16BD13B580
:10FAA000041C8B6801AAD96906F0B4FC201C16BDA1
:10FAB000104B10B50360031C43331B78041C002B50
:10FAC00013D08068002801D0F8F7E4FC60690028B2
:10FAD00001D0F8F7DFFCE069002801D0F8F7DAFC84
:10FAE000606A002801D0F8F7D5FC201CF9F7E7FC84
:10FAF000201C10BD50D60200104B10B50360031C33
:10FB000043331B78041C002B13D08068002801D0DD
:10FB1000F8F7C0FC6069002801D0F8F7BBFCE06989
:10FB2000002801D0F8F7B6FC606A002801D0F8F789
:10FB3000B1FC201CF9F7C3FC201C10BD60D60200EC
:10FB400010B5041C024B0360F9F7B9FC201C10BD72
:10FB5000E0D5020010B5041C024B0360F9F7AFFCBE
:10FB6000201C10BDF8D502000E4B10B50360031C1D
:10FB700064331B78041C002B0ED08068002801D051
:10FB8000F8F788FC6069002801D0F8F783FCE06989
:10FB9000002801D0F8F77EFC201CF9F790FC201C0F
:10FBA00010BDC04670D6020010B5041C024B0360A5
:10FBB000F9F785FC201C10BD90D4020010B5041C80
:10FBC000024B0360F9F77BFC201C10BDD0D402006F
:10FBD00010B5041C024B0360F9F771FC201C10BD2A
:10FBE00000D5020010B5041C024B0360F9F767FC56
:10FBF000201C10BD10D6020010B5041C024B03607F
:10FC0000F9F75DFC201C10BD28D6020010B5041CBD
:10FC1000FFF74EFF201CF8F748FC201C10BD10B564
:10FC2000041CFFF769FF201CF8F73FFC201C10BDE7
:10FC300010B5041CFFF784FF201CF8F736FC201CCD
:10FC400010BD10B5041CFFF785FF201CF8F72DFC34
:10FC5000201C10BD10B5041CFFF786FF201CF8F710
:10FC600024FC201C10BD10B5041CFFF79DFF201CB8
:10FC7000F8F71BFC201C10BD10B5041CFFF79EFFFD
:10FC8000201CF8F712FC201C10BD10B5041CFFF757
:10FC90009FFF201CF8F709FC201C10BD10B5041CA8
:10FCA000FFF7A0FF201CF8F700FC201C10BD10B5CA
:10FCB000041CFFF7A1FF201CF8F7F7FB201C10BD68
:10FCC00010B5041C044B0360083006F0FDFF201C37
:10FCD000F9F7F5FB201C10BD90D5020010B5041CEF
:10FCE000FFF7EEFF201CF8F7E0FB201C10BD000022
:10FCF00010B5041C044B0360083006F0E5FF201C1F
:10FD0000F9F7DDFB201C10BD48D4020010B5041C1F
:10FD1000FFF7EEFF201CF8F7C8FB201C10BD000009
:10FD200038B50E4B05690360041CF9F7F1FB8542F9
:10FD300004D0002D02D0281CF8F7ACFBA0680028E6
:10FD400002D003685B689847201C0C3006F0BCFFAB
:10FD5000201CF9F7B4FB201C38BDC04610D50200AA
:10FD600010B5041CFFF7DCFF201CF8F79EFB201CDD
:10FD700010BDF0B51C1C87B005AB071C04A806F02D
:10FD80005EFB211C03AB05A80C9A06F058FB049CF3
:10FD9000059D231C0C3B1B68E31801932B1C0C3B9B
:10FDA0001E68AE19381C211C2A1C06F050FE0028C3
:10FDB00014D1201C15F0FEFE2418281C15F0FAFEA4
:10FDC000019B2D189C4204D1AE1B751EAE4176429C
:10FDD00007E0B54204D001340135E3E7061C00E03A
:10FDE000012605A806F084F804A806F081F8301C66
:10FDF00007B0F0BDF0B51C1C244B85B0171C036088
:10FE0000009102AB111C061C221C03A806F017FB74
:10FE1000039DE41B2B1C0C3B1B686400EB18201C8F
:10FE20000193F8F758FB071C2A1C0098391C231C67
:10FE300006F018FE021EA2420ED3441C381CF8F72E
:10FE400029FB201CF8F747FB071C2A1C0098391CCB
:10FE5000231C06F007FE021C391C301C06F0F0F9CA
:10FE6000281C15F0A7FE019B2D189D4205D0301CC3
:10FE70000021013506F075FAD6E7381CF8F70AFBC1
:10FE800003A806F035F8301C05B0F0BDE01E0020D8
:10FE90000A2807D82F2915D93030C0B2814211D293
:10FEA00030390DE00B1C303B092BF9D9313B052BC8
:10FEB00001D8573904E00B1C413B052B02D83739D8
:10FEC000081C01E001204042704738B5037F002B39
:10FED00002D04018407F08E0041C0D1C05F0A1FD75
:10FEE0002368201C9B69291C984738BDF8B51F1C46
:10FEF000037F051C0E1C141C012B05D1521A381C43
:10FF000014F044FB201C0BE0002B01D105F089FD0F
:10FF10002B68281CDB69311C9C46221C3B1CE047DB
:10FF2000F8BD38B54418FF34A37F002B07D1036810
:10FF3000151C1B6A9847031EAB4200D0A077181C03
:10FF400038BD000010B5531E9A4181600021041C89
:10FF5000034B426003600A1C06F008FF201C10BD22
:10FF600058D5020008B503689B68984708BD08B5D6
:10FF70000368DB68984708BD10B5041C0B681B6953
:10FF80009847201C10BD10B5041C0B685B6998478E
:10FF9000201C10BD10B5041C0B689B699847201CE1
:10FFA00010BD10B5041C0B68DB699847201C10BD00
:10FFB00008B503681B6A984708BD036813B55B6AF8
:10FFC0009847FF22041C010A030C11401440090247
:10FFD0001A4012042143000E11430306081C184363
:10FFE00016BD036813B59B6A9847FF22041C010ADB
:10FFF000030C1140144009021A4012042143000E60
:020000021000EC
:1000000011430306081C184316BD000010B5531E0B
:100010009A4181600021041C034B426003600A1C6A
:1000200006F056FE201C10BD20D5020008B503685E
:100030009B68984708BD08B50368DB68984708BD0A
:1000400010B5041C0B681B699847201C10BD10B527
:10005000041C0B685B699847201C10BD10B5041C7C
:100060000B689B699847201C10BD10B5041C0B68D9
:10007000DB699847201C10BD08B503681B6A9847C8
:1000800008BD036813B55B6A9847FF22041C010A88
:10009000030C1140144009021A4012042143000EBF
:1000A00011430306081C184316BD036813B59B6A69
:1000B0009847FF22041C010A030C11401440090256
:1000C0001A4012042143000E11430306081C184372
:1000D00016BD00004B1E99410A4B021C0360002311
:1000E000433241608360C36003744374837443612B
:1000F0008361C361036243628362C36203634363D8
:100100001370704750D602004B1E99410A4B021CD7
:1001100003600023433241608360C360037443740F
:10012000837443618361C361036243628362C36218
:10013000036343631370704760D60200531E9A41F5
:1001400010B5041C044B426003608160002105F07F
:100150009DFC201C10BDC04668D4020008B5036891
:100160009B68984708BD08B50368DB68984708BDD9
:1001700010B5041C0B681B699847201C10BD10B5F6
:10018000041C0B685B699847201C10BD10B5041C4B
:100190000B689B699847201C10BD00004B1E9941BD
:1001A000084B421D0360002341608360C3600374F9
:1001B00043618361C3610362D377821DD3775E326B
:1001C0001370704770D60200531E9A41074B10B54A
:1001D000426003608160041CF9F79AF900212061F4
:1001E000201C06F04FFF201C10BDC04610D5020099
:1001F00083689B680B608368DB684B60704783682B
:100200001B690B6083685B694B60704783689B69FF
:100210000B608368DB694B6070478368DB6A0B6047
:1002200083681B6B4B6083685B6B8B6083689B6B25
:10023000CB608368DB6B0B6183681B6C4B618368ED
:100240005B6C8B61704783689B6C0B608368DB6CB5
:100250004B6083681B6D8B6083685B6DCB608368CC
:100260009B6D0B618368DB6D4B6183681B6E8B61DB
:10027000704783685B6E0B6083689B6E4B6083681E
:10028000DB6E8B6083681B6FCB6083685B6F0B6179
:1002900083689B6F4B618368DB6F8B61836804337A
:1002A000DB6FCB6183680833DB6F0B628368883355
:1002B0001B684B6283688C331B688B628368903346
:1002C0001B68CB627047836894331B680B6083683C
:1002D00098331B684B6083689C331B688B60836812
:1002E000A0331B68CB608368A4331B680B618368F1
:1002F000A8331B684B618368AC331B688B618368D0
:10030000B0331B68CB618368B4331B680B628368AE
:10031000B8331B684B628368BC331B688B6283688D
:10032000C0331B68CB6270474B1E9941044B10B51C
:1003300041600360041CF9F7DFF8A060201C10BDC9
:1003400090D502004B1E9941044B10B541600360EB
:10035000041CF9F7D1F8A060201C10BD48D402009D
:1003600010B5041C0B48F9F761F923685A689B68BB
:10037000984203D280008058002801D1F8F74DFE42
:100380000549064A002306F065F8002801D106F069
:100390004BFB10BDD01E002024CB02005CDC020011
:1003A00010B5041C0B48F9F741F923685A689B689B
:1003B000984203D280008058002801D1F8F72DFE22
:1003C0000549064A002306F045F8002801D106F049
:1003D0002BFB10BD5019002024CB0200A0D8020036
:1003E000031CF7B5012264331A70041C081C0F1C8F
:1003F000FFF7D6FF051C01A8291CFFF7B9FE019BDA
:1004000001A80C3B1B68E36005F072FDE068F8F79B
:1004100062F8061C291C01A8FFF7AAFEE268002367
:10042000311C01A805F0B8FC01A805F061FD00230E
:10043000E268A6609A4204D00022B256D3179B1AF3
:10044000DB0F291C237401A8FFF799FE019B01A86B
:100450000C3B1B68A36105F04BFDA069F8F73BF866
:10046000061C291C01A8FFF78AFEA269311C002383
:1004700001A805F091FC01A805F03AFD291C666170
:1004800001A8FFF783FE019B01A80C3B1B682362B8
:1004900005F02EFD206AF8F71EF8061C291C01A89D
:1004A000FFF774FE311C226A002301A805F074FCDA
:1004B00001A805F01DFDE661281CFFF74FFE631D36
:1004C000D877281CFFF74FFEA31DD877381CFFF7FD
:1004D00047FF094B051C1968231C0A1C26332432CC
:1004E000FFF704FD054B281C1968231C0A1C4A331E
:1004F0001A32FFF7FBFCF7BDB0000020A800002077
:10050000F7B5061C0E48F9F791F832688300D468F5
:100510000190E4182768002F0FD16820F7F7C9FF72
:10052000051C391CFFF73AFE281C311CFFF758FF49
:100530003068291C019AF9F755F82068FEBDC046BD
:100540005019002010B5041C0B48F9F76FF8236808
:100550005A689B68984203D280008058002801D1D5
:10056000F8F75BFD0549064A002305F073FF0028F4
:1005700001D106F059FA10BD4819002024CB020021
:10058000F0D6020010B5041C0B48F9F74FF82368A9
:100590005A689B68984203D280008058002801D195
:1005A000F8F73BFD0549064A002305F053FF0028F4
:1005B00001D106F039FA10BD4C19002024CB0200FD
:1005C00000D8020010B5041C0B48F9F72FF8236877
:1005D0005A689B68984203D280008058002801D155
:1005E000F8F71BFD0549064A002305F033FF0028F4
:1005F00001D106F019FA10BD5C19002024CB0200CD
:1006000074D80200031CF7B5012243331A70041C8E
:10061000081C0F1CFFF7D6FF051CFFF707FD6074D1
:10062000281CFFF708FDA074281CFFF725FD291CD6
:10063000E06201A8FFF704FD019B01A80C3B1B68C9
:10064000E36005F055FCE068F7F745FF061C291C40
:1006500001A8FFF7F5FCE2680023311C01A805F0B2
:100660009BFB01A805F044FC0023E268A6609A42C7
:1006700004D00022B256D3179B1ADB0F291C237417
:1006800001A8FFF7E4FC019B01A80C3B1B68A361D8
:1006900005F02EFCA069F7F71EFF061C291C01A817
:1006A000FFF7D5FCA269311C002301A805F074FBFB
:1006B00001A805F01DFC291C666101A8FFF7CEFC0E
:1006C000019B01A80C3B1B68236205F011FC206A0A
:1006D000F7F701FF061C291C01A8FFF7BFFC226ADF
:1006E000311C002301A805F057FB01A805F000FC10
:1006F000291CE66101A8FFF7B8FC019B01A80C3B8F
:100700001B68A36205F0F4FBA06AF7F7E4FE061C81
:10071000291C01A8FFF7A9FC311CA26A002301A82B
:1007200005F03AFB01A805F0E3FB6662281CFFF721
:10073000A8FC2063281CFFF7B8FC6063381CFFF797
:100740000FFE044B1968231C0A1C38330B32FFF7C9
:10075000CDFBF7BDAC000020F7B5061C0E48F8F73E
:1007600065FF32688300D4680190E4182768002F81
:100770000FD14420F7F79DFE051C391CFFF7C4FC80
:10078000281C311CFFF73EFF3068291C019AF8F73E
:1007900029FF2068FEBDC0465C19002010B5041C6E
:1007A0000B48F8F743FF23685A689B68984203D2C6
:1007B00080008058002801D1F8F72FFC0549064A2F
:1007C000002305F047FE002801D106F02DF910BDE9
:1007D0006019002024CB0200E0D80200031CF7B50A
:1007E000012243331A70041C081C0F1CFFF7D6FFAC
:1007F000051CFFF7B7FB6074281CFFF7B8FBA0745B
:10080000281CFFF7D5FB291CE06201A8FFF7B4FB09
:10081000019B01A80C3B1B68E36005F069FBE068E5
:10082000F7F759FE061C291C01A8FFF7A5FBE26893
:100830000023311C01A805F0AFFA01A805F058FB10
:100840000023E268A6609A4204D00022B256D31771
:100850009B1ADB0F291C237401A8FFF794FB019B53
:1008600001A80C3B1B68A36105F042FBA069F7F7E8
:1008700032FE061C291C01A8FFF785FBA269311C6A
:10088000002301A805F088FA01A805F031FB291C16
:10089000666101A8FFF77EFB019B01A80C3B1B686A
:1008A000236205F025FB206AF7F715FE061C291CBC
:1008B00001A8FFF76FFB226A311C002301A805F095
:1008C0006BFA01A805F014FB291CE66101A8FFF7EB
:1008D00068FB019B01A80C3B1B68A36205F008FBA9
:1008E000A06AF7F7F8FD061C291C01A8FFF759FBC1
:1008F000311CA26A002301A805F04EFA01A805F0F8
:10090000F7FA6662281CFFF758FB2063281CFFF7E4
:1009100068FB6063381CFFF723FD044B1968231C38
:100920000A1C38330B32FFF7E1FAF7BDAC000020A8
:10093000F7B5061C0E48F8F779FE32688300D468D4
:100940000190E4182768002F0FD14420F7F7B1FD7C
:10095000051C391CFFF7BEFB281C311CFFF73EFFAE
:100960003068291C019AF8F73DFE2068FEBDC0469C
:100970006019002010B5041C0B48F8F757FE2368D7
:100980005A689B68984203D280008058002801D1A1
:10099000F8F743FB0549064A002305F05BFD0028F4
:1009A00001D106F041F810BD4419002024CB02000B
:1009B0002CD8020010B5041C0A48F8F737FE23684B
:1009C00099685A68002388420AD280008058984269
:1009D00006D00549054A05F03DFD431E9841C3B2C6
:1009E000181C10BDD01E002024CB02005CDC0200CD
:1009F00010B5041C0A48F8F719FE236899685A686C
:100A0000002388420AD280008058984206D00549C7
:100A1000054A05F01FFD431E9841C3B2181C10BDC6
:100A20004819002024CB0200F0D6020010B5041CA7
:100A30000A48F8F7FBFD236899685A680023884242
:100A40000AD280008058984206D00549054A05F030
:100A500001FD431E9841C3B2181C10BD4C19002063
:100A600024CB020000D80200F0B5002585B0029129
:100A70009C46291C0A9C0B9E0392039B5B181F78C3
:100A80000193331BBB4202DC071C231C0BE07BB22F
:100A9000002BF9DD6346013BF61B994201D201317F
:100AA000EBE70135E9E7B34205D001335A1E12786E
:100AB0003A700137F7E71C1B0019013D12D36A4653
:100AC0000024127A0270019A1778661CBC4204D086
:100AD0001A5D04196270341CF7E780191B19ECE7E2
:100AE00040191B1901390DD36A460024127A02708D
:100AF000039A565C651CB442F2D01F5D04196770FE
:100B00002C1CF7E705B0F0BDF7B5089F141C0A9A36
:100B10008C460B9DBE1A002F00D12E6800929219B0
:100B20000192191C0998231C6246FFF79DFF099B3F
:100B3000C41A002F07D02B68391C9A1B13F026FD0E
:100B40002B689E1BA4192C60F7BD73B50E1C151CD9
:100B5000089A099C00922168079852180192191C62
:100B6000321C2B1CFFF780FF079BC01A206073BD4F
:100B7000F7B5141C1D1C099A089B01919F1AB023FC
:100B8000C2681340202B0BD1291C099A201C13F09A
:100B9000FDFC099B0199E0183A1C13F014FD44E098
:100BA0000026102B14D16C30FFF7DAFB2D21061C28
:100BB000FFF78BF92B78834206D0301C2B21FFF7EF
:100BC00084F92B7883420FD101262B7823700134CE
:100BD00001993A1C201C13F0F6FC099BE0199A1BA2
:100BE000A91913F0D3FC20E0301C3021FFF76DF978
:100BF0002B78834217D1099B012B14DD301C7821FF
:100C0000FFF763F96B78834206D0301C5821FFF759
:100C10005CF96B78834206D12B78022623706B78BF
:100C200063700234D4E70026D2E7F7BDF8B5171C8D
:100C300006AA1278061C0D1C002A0FD0041C281CC2
:100C40000A210FF0D9FC79180B79013C281C23707C
:100C50000A210FF04BFC051EF1D11AE04A221A407E
:100C6000402A09D1041C07232B40FB181B79013CA7
:100C70002370ED08F7D10CE014225B0400D4103A85
:100C8000341C0F23B9182B40CB5C013C23702D0979
:100C9000F7D1301BF8BDF8B51E1C08AB1B78071C3C
:100CA000141C0799002B16D0051C201C311C0A228D
:100CB00000230FF015FE069B013D9A181379201CA6
:100CC0002B70311C0A2200230FF00AFE041C0E1C9C
:100CD0000843EAD126E04A230B40402B0FD1051CE4
:100CE0000723069A2340D3181B79013D2B70E40893
:100CF00073071C43231CF6083343F1D112E014227E
:100D00004B0400D4103A3D1C0F2306992340891848
:100D1000CB5C013D2B70240933071C43231C36098F
:100D20003343F1D1781BF8BD10B5041C00680028CE
:100D300004D004F0BFFD01235B426360201C10BDA2
:100D400073B5D5B2061C6C4600910192002D08D1F6
:100D5000081C069A191C04F0C6FD069B984200D098
:100D60000135331C2571301C06CC06C376BDF0B5A9
:100D7000A9B02E9C05936C3431AB1F78061C32ABA6
:100D8000201C1D780492FFF7EBFA0390201CFFF75C
:100D9000F1FD2521041C0398FFF797F807AB1870A5
:100DA000002D02D15F709D7003E000225D709F7086
:100DB000DA70309A08A90092201C802206F033F9DC
:100DC00008A814F0F7FE04990090059A301C08ABAF
:100DD000FFF7B6FF301C29B0F0BDF0B591B004AFFD
:100DE0003A6220227B622823BA18D31840CBF860DD
:100DF000301C1B786C307B60B960FFF781FB031CF3
:100E000088B026337B6104AB3B614A23F468051C40
:100E10002340BB61402B01D0082B03D10023FB6191
:100E2000396D06E00123FB613B6D002BF8DC3B6D67
:100E30005942FB69386900937A69231C1430FFF723
:100E4000F5FE3B69F8622A7C1B1A1433002A1CD079
:100E50006A4640001030C008C000121A954612229F
:100E60006A443A61AA1DD27F009694463A69029379
:100E7000019220220C23BA18D3180393B868634652
:100E8000A968EA68FFF761FE3B69F969FA6A002917
:100E900008D0396D002902DB21052BD414E0013B79
:100EA000073529E0A1050FD5396D002928D10BE0C0
:100EB00078696104C90F41188878591E087029782B
:100EC000023B19700232FA62B568F96A8D421EDD82
:100ED0002A1C68460E32D208D200821A954604AC0B
:100EE00000950191301C7968221CFFF741FEFD62DC
:100EF000231C0CE0013B0835E97F19700132E2E761
:100F0000B9692A354029D3D1013B2978F5E7002278
:100F1000B260FA6A0092F868396A7A6AFFF710FFDD
:100F2000BD46F8680DB0F0BD30B5041C87B00AA806
:100F300020C80078009501900C980290201CFFF7C3
:100F40004CFF201C07B030BDF0B58FB004AFBA61C4
:100F50001822FB612823BA18D31810CB18221B784B
:100F6000BA187B603023D3181D78E368B860FB6043
:100F7000DB070CD400947B681822019308230295A8
:100F8000BA18D018BA69FB69FFF727FF62E0201C86
:100F90006C30FFF7B5FA002D02D04569866901E093
:100FA000C569066AA368B34248DD6A469B1B7B613C
:100FB0000E33DB08DB00D31A9D4604AB181C7A699C
:100FC00079683B6113F0FFFA0023FA68A360B0333D
:100FD0001A40131E202B19D118220096183BBA185C
:100FE000D018B969FA692B1CFFF7AAFE3B6A1822D0
:100FF000BB612423FB181B78BA183B777B690093ED
:101000000823396AD018FA693B6921E07B69182204
:1010100000930823BA18D018B969FA693B69FFF739
:101020008FFE3B6A1822BB612423FB181B78BA1879
:101030003B7708230096D018396A07E0002318226E
:10104000A36000960833BA18B969D0182B1CFA6946
:10105000FFF776FE3B6ABD46BB612423FB181B7875
:10106000BA683B771823FB1803CB03C2B8680BB0F0
:10107000F0BDF0B591B004AF3A6220227B62282324
:10108000BA18D31840CBF860301C1B786C307B60EA
:10109000B960FFF735FA031C26333B61F36888B06B
:1010A000FB614A23FA69051C1A40002304AC7B61EA
:1010B000BA61131E402B04D0083B5A1E9341DBB289
:1010C0007B61201C7B69143000933A69FB69396DA0
:1010D000FFF7ACFDF8622A7C231A1433002A1AD0D9
:1010E0006A4640001030C008C000121A9546AA1D7A
:1010F000D27F12249446202202930C23BA18D318CC
:101100006C440393009601946346B868A968EA6842
:10111000FFF71BFD231C7A69002A10D1FA6992059A
:101120000DD53A6D002A0AD0BA69591E2A35402ACF
:101130001BD12B780B70FB6A0133FB620B1CB5686B
:10114000F96A8D421FDD2A1C68460E32D208D20091
:10115000821A954604AC00950191301C7968221CD6
:10116000FFF706FDFD62231C0DE0FA6938695204A1
:10117000D20F82189278023B0A702A781A70FA6AA3
:101180000232FA62DBE70022B260FA6A0092F86883
:10119000396A7A6AFFF7D4FDBD46F8680DB0F0BD34
:1011A00030B5041C87B00AA820C8007800950190CB
:1011B0000C980290201CFFF75CFF201C07B030BD8C
:1011C000F0B58BB00593079310AB40CB94460692D5
:1011D0001A78F368051C049304980E4B08AF03407B
:1011E000822080000343F360129B01920293381C1B
:1011F0006246059B0096FFF73CFF089B06AC0693F2
:101200003B79281C2371049BF3602B1C06CC06C37E
:101210000BB0F0BDB5BFFFFFF0B591B004AF3A62BF
:1012200020227B622823BA18D31820CBF860281C10
:101230001B786C307B60B960FFF762F9031C8CB0DF
:1012400026337B6104AB3B614A23EE68041C3340C8
:10125000BB61402B01D0082B01D1002303E07B6D43
:10126000002B04DD0123FB613A6D7B6D08E0002B50
:1012700069D0386D796D002342428B410121F961BB
:101280007969386900910196F96928300291FFF770
:1012900002FD3B69F862227C1B1A2833002A1CD00D
:1012A0006A4640001030C008C000121A954612224B
:1012B0006A443A61A21DD27F009594463A6902932E
:1012C000019220220C23BA18D3180393B8686346FE
:1012D000A168E268FFF739FC3B69F969FA6A0029FD
:1012E00008D0796D002902DB310530D415E0013BCF
:1012F00007342EE0B10510D5396D786D01432CD13E
:101300000BE078697104C90F41188878591E08707C
:101310002178023B19700232FA62AC68F96A8C4299
:1013200022DD221C68460E32D208D200821A95466F
:1013300004AE00940191281C7968321CFFF718FC58
:10134000FC62331C10E03B6D002B8BD191E7013B1D
:101350000834E17F19700132DEE7B9692A34402987
:10136000CFD1013B2178F5E70022AA60FA6A00920A
:10137000F868396A7A6AFFF7E3FCBD46F8680DB091
:10138000F0BD70B5041C86B00AA820C8007800958E
:1013900001900C9D0D9E201C02950396FFF73CFFCB
:1013A000201C06B070BDF0B593B004AFFB622823DB
:1013B000BA62FA18D31840CB7861301C1B786C30B5
:1013C0007B60BB6DB9603B61FB6DFB60FFF798F81C
:1013D000031C2633BB61F3688CB07B624A237A6AB4
:1013E000051C1A40002304ACFB613A62131E402B1B
:1013F00004D0083B5A1E9341DBB2FB61201CBB6941
:10140000283000937B6A0193FB6902933A69FB6879
:10141000FFF741FC78632A7C231A2833002A1AD06C
:101420006A4640001030C008C000121A9546AA1D36
:10143000D27F12249446282202930C23BA18D31880
:101440006C440393009601946346B868A968EA68FF
:10145000FFF77BFB231CFA69002A11D17A6A9205F7
:101460000ED53A69F9680A430AD03A6A591E2A35F4
:10147000402A1BD12B780B707B6B01337B630B1CD9
:10148000B568796B8D421FDD2A1C68460E32D20882
:10149000D200821A954604AC00950191301C7968FF
:1014A000221CFFF765FB7D63231C0DE07A6AB86997
:1014B0005204D20F82189278023B0A702A781A706E
:1014C0007A6B02327A63DBE70022B2607A6B0092B9
:1014D0007869B96AFA6AFFF733FCBD4678690FB0DC
:1014E000F0BD70B5041C86B00AA820C8007800952D
:1014F00001900C9D0D9E201C02950396FFF753FF53
:10150000201C06B070BDF0B593B004AFBA611822CC
:10151000FB613823BA18D31840CB18221B78BA18AD
:101520003B604023D3181C78331C6C33B860181C04
:101530003B617960FEF7E4FF736878610625002B54
:1015400000DB1D1C18221023BA18D118301C221CD5
:10155000F8F7DEF92B1CF2681E33520701D51B3356
:10156000FF336A460E33DB08DB00D31A9D46F7F7DC
:10157000C3FF786200953A6E7B6E02920393182245
:101580000C231825BA1804ACD0187D190433EB18B5
:10159000211C0022F9F7D0F838623869FEF7E0FE26
:1015A0003A6A6946131C0E33DB08DB00CB1A9D46F2
:1015B00004ADA218211C2B1CFEF798FC3B6A201CD2
:1015C0001A1C2E213B6112F0C7FF021E05D07B6959
:1015D000001B0533DB7F2A1813707B691B7C002BF3
:1015E0003CD0002A0BD13B69022B08DD61783929F8
:1015F00034D8A3782F2931D9303B092B2ED869460E
:101600003B695B000E33DB08DB00CB1A9D46FD21F6
:1016100004ABFB60237800242B3B0B4206D12B78D4
:10162000F96801340B703B69013B3B627B6918210F
:101630000633DB7F0092FA687918121901922A1991
:10164000029208228A1803927A6978689168D268AF
:10165000FFF75AFA3B6A1D193D62FD68B4683A6AA1
:10166000944212DD231C69460E33DB08DB00CB1AE3
:101670009D4604AB7B61009401922B1C301C3968A1
:101680007A69FFF775FA7D693C620023B3603B6AB3
:101690000093B868B969FA692B1CFFF751FBBD4686
:1016A000B8680FB0F0BD70B588B0041C0CA820C895
:1016B00000780095019000200E9D0F9E02900495E9
:1016C0000596201CFFF71FFF201C08B070BDF0B569
:1016D00093B004AFBA611822FB613823BA18D3184B
:1016E00040CB18221B78BA183B604023D3181C78D3
:1016F000331C6C33B860181C3B617960FEF700FF47
:10170000736878610625002B00DB1D1C182210234E
:10171000BA18D118301C221CF8F7FAF82B1CF26802
:101720001E33520701D51B33FF336A460E33DB08E5
:10173000DB00D31A9D46F7F7DFFE786200953A6E1C
:101740007B6E0292039318220C231825BA1804AC5E
:10175000D0187D190433EB18211C0022F8F7ECFF98
:1017600038623869FEF7FCFD3A6A6946131C0E338D
:10177000DB08DB00CB1A9D4604ADA218211C2B1CF4
:10178000FEF7B4FB3B6A201C1A1C2E213B6112F0B1
:10179000E3FE021E05D07B69001B0533DB7F2A18A0
:1017A00013707B691B7C002B3CD0002A0BD13B695A
:1017B000022B08DD6178392934D8A3782F2931D953
:1017C000303B092B2ED869463B695B000E33DB08A2
:1017D000DB00CB1A9D46FD2104ABFB60237800247F
:1017E0002B3B0B4206D12B78F96801340B703B6917
:1017F000013B3B627B6918210633DB7F0092FA686C
:101800007918121901922A19029208228A18039251
:101810007A6978689168D268FFF776F93B6A1D1992
:101820003D62FD68B4683A6A944212DD231C694641
:101830000E33DB08DB00CB1A9D4604AB7B610094C2
:1018400001922B1C301C39687A69FFF791F97D6988
:101850003C620023B3603B6A0093B868B969FA69D7
:101860002B1CFFF76DFABD46B8680FB0F0BD70B520
:1018700088B0041C0CA820C80078009501904C206A
:101880000E9D0F9E029004950596201CFFF71FFFEA
:10189000201C08B070BD0000F0B593B00B9318ABDE
:1018A0000A9204CB0890141C1B786C34201C0493FF
:1018B000FEF756FD061C201CFEF74EFF021C1A9B6D
:1018C00038321B6812781978041C914207D0026BD9
:1018D0001D1C0D92C2690592026A03920BE0426BD5
:1018E0000D92426A0592826A03921A1C0C3A15689C
:1018F000691E8D415D190C3B1A682B1CAA18934276
:1019000006D21978B069415C490701D50133F6E781
:101910005F1B00D1D1E06E4B79000EA80E9304F04E
:1019200047FCE36AFE1A002E28DD002B00DA3E1C7D
:10193000E368002B1DD0710000220EA804F098FB74
:101940000EA804F045FBAB19A17C00950193A26899
:10195000E3680E98FFF788F806900EA804F038FBAD
:101960000E9A069B0EA8991A0122524204F048FBD7
:1019700004E00EA8291C321C04F0BAFBE36A002B19
:1019800015DD617C0EA804F0ECFC002E03DBA91928
:101990000EA8E26A09E0231C393371421A780EA8B6
:1019A00004F0B2FC291C3A1C0EA804F049FC189B58
:1019B000DA68B023134007930E9B0C3B1F68039B10
:1019C000DF190023920500D5A369FF18404B790069
:1019D0000FA80F9304F0ECFB189B9D68002306935F
:1019E000079B102B03D1AF429B415B42069300261D
:1019F0000DABF05C04282BD80EF064FD221A030E08
:101A00001500189BDB6809939B0521D50FA8616918
:101A1000A26904F015FC1BE0039B002B18D0059B6A
:101A20000FA8197809E00FA80EA904F004FC0FE034
:101A3000069B002B07D104990FA804F092FC07E045
:101A4000069B002B04D0E91B0FA8049A04F05CFC51
:101A50000136042ECCD1039B012B06D91A1C059903
:101A6000013A01310FA804F0EBFB0F9B0C3B1A6805
:101A700095420ED9079BAA1A0FA8202B04D1111C3E
:101A8000049A04F041FC05E00021049B04F0FAFAFA
:101A900000E0151C10AE301C0A990B9A0F9B0095A4
:101AA000FFF74EF9109B0AAC0A9333790FA8237104
:101AB00004F01EFA0EA804F01BFA0023189A936093
:101AC000089A0AAB03CB03C2089813B0F0BDC04616
:101AD000E01E0020F0B593B00B9318AB0A9204CB34
:101AE0000890141C1B786C34201C0493FEF738FCFF
:101AF000061C201CFEF71CFF021C1A9B38321B68B8
:101B000012781978041C914207D0026B1D1C0D92AB
:101B1000C2690592026A03920BE0426B0D92426A1F
:101B20000592826A03921A1C0C3A1568691E8D414F
:101B30005D190C3B1A682B1CAA18934206D219781F
:101B4000B069415C490701D50133F6E75F1B00D15D
:101B5000D1E06E4B79000EA80E9304F029FBE36AE6
:101B6000FE1A002E28DD002B00DA3E1CE368002B55
:101B70001DD0710000220EA804F07AFA0EA804F01D
:101B800027FAAB19A17C00950193A268E3680E982F
:101B9000FEF76AFF06900EA804F01AFA0E9A069B4A
:101BA0000EA8991A0122524204F02AFA04E00EA863
:101BB000291C321C04F09CFAE36A002B15DD617CC1
:101BC0000EA804F0CEFB002E03DBA9190EA8E26AD2
:101BD00009E0231C393371421A780EA804F094FBF3
:101BE000291C3A1C0EA804F02BFB189BDA68B023C2
:101BF000134007930E9B0C3B1F68039BDF190023C8
:101C0000920500D5A369FF18404B79000FA80F93E8
